:020000040800F2
:1000000000040020A10200087D10000881100008F3
:10001000D510000881100008A9100008A3020008EC
:10002000A3020008A3020008A30200080529000893
:10003000A3020008A3020008A3020008A30200080C
:10004000A3020008A3020008A3020008A3020008FC
:10005000A3020008A30200083D3E0008693E000814
:10006000953E0008C13E0008ED3E0008A3020008CE
:10007000A3020008A3020008A3020008A3020008CC
:10008000A3020008A3020008A3020008A3020008BC
:10009000A3020008A3020008A3020008193F0008F9
:1000A000A3020008A3020008A3020008A30200089C
:1000B000B93A0008A3020008A3020008A30200083E
:1000C000A3020008A3020008A3020008A30200087C
:1000D000A3020008A3020008A3020008A30200086C
:1000E000813F0008A3020008A3020008A302000841
:1000F000A3020008A3020008A3020008A30200084C
:10010000A3020008A3020008A3020008A30200083B
:10011000A3020008A3020008A3020008A30200082B
:10012000A3020008A3020008A3020008A30200081B
:10013000A3020008A3020008A3020008A30200080B
:10014000A3020008A3020008A3020008A3020008FB
:10015000A3020008A3020008A3020008A3020008EB
:10016000A3020008A3020008A3020008A3020008DB
:10017000A30200083D340008A3020008A3020008FF
:10018000A3020008A302000865110008A3020008EA
:10019000A3020008A3020008A3020008A3020008AB
:1001A000A3020008A3020008A3020008A30200089B
:1001B000A3020008A3020008A3020008A30200088B
:1001C000A3020008A3020008A3020008A30200087B
:1001D000A302000829340008A3020008A3020008B3
:1001E000A3020008A3020008A3020008A30200085B
:1001F000A3020008A3020008A3020008A30200084B
:10020000A3020008A3020008A3020008A30200083A
:10021000A3020008A3020008A3020008A30200082A
:10022000A3020008A3020008A3020008A30200081A
:10023000A3020008A3020008A3020008A30200080A
:10024000A3020008A3020008A3020008A3020008FA
:10025000A3020008A3020008A3020008A3020008EA
:10026000A3020008A3020008A3020008A3020008DA
:10027000A3020008A3020008A3020008A3020008CA
:10028000A3020008A3020008A3020008A3020008BA
:10029000A3020008A3020008A3020008A3020008AA
:1002A00002E000F000F8FEE772B6394880F30888F3
:1002B000384880F3098838484EF60851CEF20001DC
:1002C000086040F20000CCF200004EF63471CEF22D
:1002D00000010860BFF34F8FBFF36F8F40F2000043
:1002E000C0F2F0004EF68851CEF200010860BFF374
:1002F0004F8FBFF36F8F4FF00000E1EE100A4EF604
:100300003C71CEF200010860062080F31488BFF330
:100310006F8F02F035FB03F04DFB4FF055301F4956
:100320001B4A91423CBF41F8040BFAE71C49194AA9
:1003300091423CBF41F8040BFAE71A491A4A1B4B99
:100340009A423EBF51F8040B42F8040BF8E7002034
:100350001749184A91423CBF41F8040BFAE702F0F2
:1003600053FB03F09BFB144C144DAC4203DA54F8DE
:10037000041B8847F9E700F03FF8114C114DAC42DF
:1003800003DA54F8041B8847F9E702F03BBB00008E
:1003900000040020002400200000000800000020CD
:1003A00000040020E0430008002400204424002032
:1003B0004824002060350020A0020008A0020008A8
:1003C000A0020008A00200082DE9F04F2DED108AD0
:1003D000C1F80CD0D0F80CD0BDEC108ABDE8F08F7D
:1003E000002383F311882846A047002001F0E6FE91
:1003F00001F096FE00DFFEE738B5204C6FF00D03EC
:10040000002523700323A57063701E23E5702571FA
:100410006571A571E57125726572A372E57200F0D0
:1004200047FD20B10E2325726572A372E57202F0BA
:100430002BFA044602F060FA0546D0B9104B9C42F4
:1004400019D001339C4241F2883412BF0546002482
:100450000125002002F022FA0DB100F0B7F800F0FB
:10046000B3FD00F07DFC204600F070F900F0AEF81E
:10047000F9E70024EDE70446EBE700BF482400203D
:10048000010007B008B500F0E9FBA0F120035842D5
:10049000584108BD054B07B51B88022101A8ADF8DE
:1004A000043000F047FC03B05DF804FB884000080E
:1004B000064991F8243033B100230822086A81F8F4
:1004C000243000F071BC0120704700BF6824002078
:1004D0002DE9F84F234C05468846174694F82430FA
:1004E0008BBB2E46DFF87C90002F38D094F824A0E8
:1004F000BAF1000F05D12022FF214846266200F004
:1005000051FDCAF10805414604EB8A00BD4228BFEF
:100510003D465FFA85FBAD00A7EB0B072A462E444C
:1005200000F018FD94F82430A844FFB29B445FFA11
:100530008BFBBBF1080F84F824B0D5D1FFF7B8FFCF
:100540000028D1D108E0266A06EB8306B042C9D064
:10055000FFF7AEFF0028C4D10020BDE8F88F0120CE
:10056000BDE8F88F6824002010B5202383F311889C
:100570001248C3680BB101F0A7FE0023104A4FF4E4
:100580007A710E4801F064FE002383F311880D4C4C
:10059000236813B12368013B2360636813B1636868
:1005A000013B6360084B1B7833B9636823B90220B1
:1005B00000F0BEFC3223636010BD00BF5424002055
:1005C000690500089825002090240020554B5649C5
:1005D0002DE9F04153F8042F013201D1BDE8F0813B
:1005E0008B42F7D1514C524B22689A4240F298808C
:1005F000504B9B6803F1006303F500339A4280F08F
:100600008F80002000F0C8FB02204B4B187000F0D8
:1006100083FC4A4BD3F8E8200022C3F8E820D3F843
:100620001011C3F81021D3F81011D3F8EC10C3F84F
:10063000EC20D3F81411C3F81421D3F81411D3F813
:10064000F010C3F8F020D3F81811C3F81821D3F82C
:100650001811D3F8801041F00061C3F88010D3F86E
:10066000801021F00061C3F88010D3F88010D3F817
:10067000801041F00071C3F88010D3F8801021F091
:100680000071C3F88010D3F8803072B62C4B2D491E
:100690000B601D682468BFF34F8FBFF36F8F2A4B29
:1006A000C3F88420BFF34F8F5A6922F480325A6115
:1006B000BFF34F8FD3F8802043F6E07EC2F3C90624
:1006C000C2F34E32B707520102EA0E0838463146ED
:1006D000013948EA000C00F14040B1F1FF3FC3F896
:1006E00074C2F5D1203A12F1200FEDD1BFF34F8F34
:1006F000BFF36F8FBFF34F8FBFF36F8F5A6922F431
:1007000000325A610022C3F85022BFF34F8FBFF36B
:100710006F8F202383F31188AD4685F30888204727
:10072000BDE8F081FCFF01081C000208040002087B
:10073000FFFF0108482400209024002000440258B4
:100740000000020808ED00E000ED00E02DE9F04FA8
:1007500099B0B34C2022FF21019010A8A66800F0A8
:1007600021FCB04AA3461378A3B90121AE48117009
:10077000C360202383F31188C3680BB101F0A4FD8B
:100780000023AA4A4FF47A71A74801F061FD0023C3
:1007900083F31188019B13B1A54B019A1A600023C2
:1007A000A44AA349019F99461C461D4698461370CA
:1007B0004B600292012000F0AFFB002F00F012828C
:1007C0009B4B1B68002B40F00D8219B0BDE8F08FE9
:1007D0000220FFF757FE002840F0FB81019BB9F192
:1007E000000F08BF1F46944B1B8802210BA8ADF8D1
:1007F0002C3000F09FFADDE74FF47A7000F02EFA0B
:10080000031E0393EADB0220FFF73CFE824600282A
:10081000E4D0039B581E042800F2DD81DFE800F0DD
:10082000030E1114170018A80523042140F8343DC5
:1008300000F080FA54464FF0000856E00421784852
:10084000F6E704217D48F3E704217D48F0E71C2406
:100850002046043400F0A2FA04210B900BA800F00B
:1008600069FA2C2CF4D1E5E7002DB7D0002CB5D0D7
:100870000220FFF707FE0546002800F0AF810120A7
:100880006C4C00F089FA4FF000090220207000F053
:1008900043FB5FFA89FA504600F08EFA074658B1DA
:1008A000504609F1010900F097FA0028F1D12C46D1
:1008B000A9460027634B97E701233E460220237099
:1008C00000F01CFBDBF808309E4206D2304600F0F8
:1008D00065FA0130EBD10436F4E70026029BA94605
:1008E0002C461E703746524B5E6000F063FB15B11C
:1008F000002C18BF0027FFF7CDFD5BE7002D3FF46C
:100900006DAF002C3FF46AAF0220029B187000F01C
:1009100003FB322000F0A2F9B0F1000AC0F25E81C0
:100920001AF0030540F05A8106EB0A03DBF80820B1
:10093000934200F25381BAF5807F00F24F81554512
:100940000DDA4FF47A7000F089F90490049B002BC3
:10095000C0F24481049B3C4AAB540135EFE7C82008
:10096000FFF790FD0546002800F038811F2E11D8B2
:10097000C6F1200410AB26F0030033495445184457
:1009800028BF5446224600F0E5FA2246FF212E48B1
:1009900000F008FB4FEAAA0A2B4930465FFA8AF2B8
:1009A000FFF796FD0446002800F01A8106EB8A0640
:1009B00005469AE70220FFF765FD00283FF40EAFD9
:1009C000FFF776FD00283FF409AF4FF0000A5346C9
:1009D000DBF8082092451CD2BAF11F0F12D8109AEA
:1009E00001320FD02AF0030218A90A4452F8202C31
:1009F0000B92184604220BA90AF1040A00F07EFBB0
:100A00000346E5E75046039300F0C8F9039B0B90BB
:100A1000EFE718A8042140F84C3D00F08BF964E79B
:100A20004824002094250020542400206905000853
:100A300098250020902400208A4000084C240020A3
:100A4000502400208C4000089424002018A8002383
:100A5000642140F8343D00F039F900287FF4BEAE3F
:100A60000220FFF70FFD00283FF4B8AE0B9800F00E
:100A7000C5F918AB43F8480D04211846CDE718A86E
:100A80000023642140F8343D00F020F900287FF471
:100A9000A5AE0220FFF7F6FC00283FF49FAE0B98AE
:100AA00000F0AEF918AB43F8440DE5E70220FFF77C
:100AB000E9FC00283FF492AE00F0A8F918AB43F827
:100AC000400DD9E70220FFF7DDFC00283FF486AE99
:100AD0000BA9142000F0A0F9824618A8042140F8C0
:100AE0003CAD00F027F951460BA896E7322000F004
:100AF000B5F8B0F1000AFFF671AE1AF0030F7FF4FB
:100B00006DAE0AEB0803DBF8082093423FF666AEB1
:100B10000220FFF7B7FC00283FF460AE2AF0030A7A
:100B2000C244D0453FF4E1AE404608F1040800F06D
:100B300035F904210A900AA800F0FCF8F1E74FF417
:100B40007A70FFF79FFC00283FF448AEFFF7B0FC37
:100B500000283FF4AFAE109B01330CD0082210A93F
:100B60000020FFF7B5FC00283FF4A4AE2022FF21AF
:100B700010A800F017FAFFF78DFC374801F024FBAE
:100B800023E6002D3FF42AAE002C3FF427AE18A830
:100B90000023642140F8343D00F098F88246002894
:100BA0007FF41CAE0220FFF76DFC00283FF416AE68
:100BB0000390FFF76FFC41F28830574601F004FBC9
:100BC0000B9800F03BFA00F0F5F9039B1C461D461C
:100BD000F0E5054689E64FF00008FFE52546FDE50E
:100BE0002C4667E6002000F039F80490049B002BA7
:100BF000FFF6E3AD012000F081F9049B213B122BAD
:100C00003FF6D8AD01A252F823F000BFD10700088B
:100C1000F907000869080008B5070008B5070008CB
:100C2000B5070008FD080008ED0A0008B50900082E
:100C30004D0A00087F0A0008AD0A0008B507000841
:100C4000C50A0008B50700083F0B0008EB080008BC
:100C5000B5070008830B0008A08601002DE9F347C3
:100C60004FF47A75002402AE154F4543DFF85880E3
:100C700006F8014D97F900305FFA84F95A1C01D04B
:100C8000A34212D158F82400012231460368D3F858
:100C900020A02B46D047012807D10A4B9DF807001A
:100CA00083F8009002B0BDE8F0870134022CE1D156
:100CB0004FF4FA7001F088FA4FF0FF30F2E700BF0E
:100CC00000240020BC250020A04000082DE9F047AA
:100CD0004FF47A7506460024134F4D43DFF85080D9
:100CE00097F900305FFA84F95A1C01D0A34210D161
:100CF00058F82400042231460368D3F820A02B467C
:100D0000D047042805D1094B002083F80090BDE8A6
:100D1000F0870134022CE3D14FF4FA7001F054FA59
:100D20004FF0FF30BDE8F08700240020BC250020F4
:100D3000A0400008074B30B41A78074B53F8224004
:100D40000A46014623682046DD69044BAC4630BCA8
:100D5000604700BFBC250020A0400008A08601001D
:100D6000F8B50A4C00250A4E01F076FC094F2070B8
:100D700030682378834207D901F06AFC3368054460
:100D80000133BD423360F3D9F8BD00BFBD2500205B
:100D9000A0250020FFFF010001F02ABD00F1006046
:100DA00000F500300068704700F10060920000F527
:100DB000003001F0ADBC0000054B1A68054B1B78F4
:100DC0009B1A834202D9104401F042BC00207047B4
:100DD000A0250020BD25002038B5074D0446286811
:100DE000204401F03BFC28B928682044BDE8384085
:100DF00001F046BC38BD00BFA02500200020704790
:100E0000014BC058704700BF00E8F11F014B186844
:100E1000704700BF0010005C234BF0B5234C1B68EB
:100E20002788C3F30B0665681B0C94F90820BE42A3
:100E300028D0A789BE4206D101220C2505FB024419
:100E4000656894F9082041F20104A3421CD041F2E4
:100E50000304A3421AD042F20104A34218D042F282
:100E60000304A34208BF5622441E013D0B460C4416
:100E7000A34217D215F9016F581C5EB1034600F862
:100E8000016CF5E70022D8E75A22EDE75922EBE79B
:100E90005822E9E72C2584421D7001D9981C5A700C
:100EA000401AF0BD1846FBE70010005C0424002047
:100EB000104B41F201015B888B429AB211D041F292
:100EC00003018B420FD042F201039A420DD042F24D
:100ED00003039A420BD10323074A02EB8303D8781A
:100EE00070470023F8E70123F6E70223F4E7002028
:100EF000704700BF0010005C90400008022804D139
:100F00004FF48002034B9A6170470128FCD14FF4E3
:100F10000002F7E700200258022803D14022034BC9
:100F20009A6170470128FCD18022F8E7002002581E
:100F3000022805D1064A536983F040035361704784
:100F40000128FCD1024A536983F08003F6E700BF11
:100F500000200258002310B5934203D0CC5CC45447
:100F60000133F9E710BD000030B5441E14F9010F3C
:100F70000B4658B193F900500131854206D11AB998
:100F800093F90020801A30BD013AEFE7002AF7D12B
:100F9000104630BD02460346981A13F9011B00297A
:100FA000FAD1704702440346934202D003F8011B72
:100FB000FAE77047024B1A78024B1A70704700BF6D
:100FC000BC2500200024002038B5164C164D2046C4
:100FD00000F02CFC2946204600F054FC2D681348F4
:100FE000D5F89020D2F8043843F00203C2F8043850
:100FF00001F0EAF80E49284600F054FDD5F890209B
:101000000C48D2F804380C49A04223F00203C2F87D
:1010100004384FF4E1330B6003D0BDE8384000F0F2
:1010200063BB38BDEC2A00208041000840420F001D
:10103000A841000840260020A425002038B50B4B0D
:1010400005461A780A4B53F822400A4B9C420CD0B2
:10105000094B002118221846FFF7A4FF056001463E
:101060002046BDE8384000F03FBB38BDBC2500201D
:10107000A0400008EC2A0020A4250020FEE7000084
:1010800000B59BB0EFF3098168226846FFF762FF65
:10109000EFF30583034B9A6B9A6A9A6A9A6A9A6A83
:1010A0009B6AFEE700ED00E000B59BB0EFF309811D
:1010B00068226846FFF74EFFEFF30583044B9A6BF7
:1010C0009A6A9A6A9A6A9A6A9A6A9B6AFEE700BF63
:1010D00000ED00E000B59BB0EFF30981682268469F
:1010E000FFF738FFEFF30583034B5A6B9A6A9A6A4E
:1010F0009A6A9A6A9B6AFEE700ED00E030B50A44FE
:10110000074D91420BD011F8013B09245840013C96
:10111000F7D040F300032B4083EA5000F7E730BDDF
:101120002083B8ED002304491A465A50C8180833E2
:101130004260802BF9D17047C0250020024A136815
:1011400043F0C0031360704700780040044B5A68B6
:1011500010439A6858600AB1181D1047704700BFC5
:10116000402600202DE9F84F414EF56D2F68EC69BF
:1011700021072C6219D014F0080F0CBF002080202A
:10118000E20748BF40F02000A3074FF0200348BF0C
:1011900040F04000610748BF40F4807083F311883D
:1011A000FFF7D4FF002383F31188E20509D520233C
:1011B00083F311884FF40070FFF7C8FF002383F317
:1011C00011884FF02009DFF8A8A04FF0000B14F0B1
:1011D000200832D13B0615D54FF02009DFF894A046
:1011E00020060FD589F31188504600F0F1F9002848
:1011F00030DA0820FFF7AAFF27F080032B600023D6
:1012000083F3118879060DD562060BD5202383F36D
:101210001188F26C336D9A4201D1336C03BB002309
:1012200083F31188E30604D5B26E13690BB15069DC
:101230009847BDE8F84F01F075BB89F31188AB8C76
:10124000504696F86410194000F05CFA8BF3118850
:10125000EC69BCE780B2288588F31188EC69BFE7A8
:1012600027F040071020FFF771FF2F60D7E700BF7E
:10127000402600207826002013B5104C204600F0B0
:1012800027FA04F11400009400234FF400720C4973
:1012900000F0E8F804F1380000944FF40072094BB4
:1012A000094900F061F9094B0C215220E365084B14
:1012B000236602B0BDE8104000F05EB84026002072
:1012C000AC2600203D110008AC280020007800402A
:1012D00000E1F505254B002908BF1946037C012BC9
:1012E000816630B511D1224B98420ED1214BD3F8F3
:1012F000E82042F08042C3F8E820D3F8102142F001
:101300008042C3F81021D3F810310A68036EC46D0F
:1013100003EB5203B3FBF2F34A68150442BF23F018
:10132000070503F0070343EA4503E3608B6843F0D6
:1013300040036360CB68510543F00103A36042F4AE
:10134000967343F0010323604FF0FF33236205D50A
:1013500012F0102205D0B2F1805F04D080F8643022
:1013600030BD7F23FAE73F23F8E700BFC440000801
:10137000402600200044025800F1604300F01F02A4
:101380000901400903F56143C9B2800083F80013E5
:10139000012300F16040934000F56140C0F88031C6
:1013A00003607047F8B51546826804460B46AA42AA
:1013B00000D28568A1692669761AB54207D2184617
:1013C0002A46FFF7C7FDA3692B44A3610DE011D99D
:1013D000AF1B32461846FFF7BDFD3A46E168304480
:1013E000FFF7B8FDE2683A44A261A36828465B1B98
:1013F000A360F8BD18462A46FFF7ACFDE368E4E7B2
:10140000836893422DE9F04104460F46154600D209
:10141000856860692669361AB54207D22A46394678
:10142000FFF798FD63692B4463610EE013D9A5EBC8
:10143000060832463946FFF78DFD4246B919E06885
:10144000FFF788FDE26842446261A36828465B1B9F
:10145000A360BDE8F0812A463946FFF77BFDE368CB
:10146000E2E7000010B50A440024C361029B00605B
:1014700040608460C160816141610261036210BDAE
:1014800008B582694369934201D1826882B9826852
:10149000013282605A1C42611970426903699A42A2
:1014A00001D3C3684361002100F0AAFE002008BDFB
:1014B0004FF0FF3008BD000070B5202304460E46F3
:1014C00083F31188A568A5B1A368A269013BA36055
:1014D000531CA36115782269934224BFE368A3617A
:1014E000E3690BB120469847002383F3118828460F
:1014F00070BD3146204600F073FE0028E2DA85F325
:10150000118870BD2DE9F74F05460F4690469A4663
:10151000D0F81C90202686F311884FF0000B14465B
:1015200064B1224639462846FFF73CFF034668B9B6
:101530005146284600F054FE0028F1D0002383F3E2
:101540001188A8EB040003B0BDE8F08FB9F1000FDB
:1015500003D001902846C847019B8BF31188E41AF9
:101560001F4486F31188DBE7C1608161416111444A
:10157000C361009B0060406082600161036270474C
:10158000F8B504460E461746202383F31188A56854
:10159000A5B1A368013BA36063695A1C62611E7018
:1015A000236962699A4224BFE3686361E3690BB10E
:1015B00020469847002080F31188F8BD3946204620
:1015C00000F00EFE0028E2DA85F31188F8BD000075
:1015D000836942699A4210B501D182687AB98268FA
:1015E000013282605A1C82611C7803699A4201D3DD
:1015F000C3688361002100F003FE204610BD4FF058
:10160000FF3010BD2DE9F74F05460F4690469A462C
:10161000D0F81C90202686F311884FF0000B14465A
:1016200064B1224639462846FFF7EAFE034668B908
:101630005146284600F0D4FD0028F1D0002383F362
:101640001188A8EB040003B0BDE8F08FB9F1000FDA
:1016500003D001902846C847019B8BF31188E41AF8
:101660001F4486F31188DBE7026843681143016079
:1016700003B11847704700001430FFF743BF000064
:101680004FF0FF331430FFF73DBF00003830FFF755
:10169000B9BF00004FF0FF333830FFF7B3BF000091
:1016A0001430FFF709BF00004FF0FF311430FFF78F
:1016B00003BF00003830FFF763BF00004FF0FF3278
:1016C0003830FFF75DBF000000207047FFF7D4BD42
:1016D000044B0360002343608360C36001230374F1
:1016E000704700BFDC40000810B52023044683F398
:1016F0001188FFF7EFFD02232374002383F3118881
:1017000010BD000038B5C36904460D461BB904215D
:101710000844FFF7A9FF294604F11400FFF7B0FEC3
:10172000002806DA201D4FF48061BDE83840FFF73D
:101730009BBF38BD026843681143016003B118477D
:101740007047000013B5446BD4F894341A681178CC
:10175000042915D1217C022912D11979012312897A
:101760008B4013420CD101A904F14C0001F098FF09
:10177000D4F894440246019B2179206800F0EAF9EC
:1017800002B010BD143001F01BBF00004FF0FF335A
:10179000143001F015BF00004C3001F0EDBF000027
:1017A0004FF0FF334C3001F0E7BF0000143001F080
:1017B000E9BE00004FF0FF31143001F0E3BE00003D
:1017C0004C3001F0B9BF00004FF0FF324C3001F057
:1017D000B3BF0000D0F8942438B5136805461978D3
:1017E000042901D0012038BD017C0229FAD11279E7
:1017F00001205C8990400440F4D105F1140001F00F
:101800007BFE02460028EDD0D5F894544FF4807347
:101810002868697900F08CF9204638BD406BFFF7E5
:10182000D9BF000000207047704700007FB5124B01
:1018300001250226044603600023057400F184029A
:10184000436029468360C3600C4B029014300193BF
:101850004FF48073009601F02BFE094B04F52372C0
:101860002946019304F14C004FF4807302940096D2
:1018700001F0F2FE04B070BD044100081D1800081C
:10188000451700080A68202383F311880B790B336E
:1018900042F823004B79133342F823008B7913B1BC
:1018A0000B3342F823000223C0F89414037400237E
:1018B00083F311887047000038B5037F044613B1E5
:1018C00090F85430ABB90125201D0221FFF732FFFB
:1018D00004F1140025776FF0010100F09DFC84F8FD
:1018E000545004F14C006FF00101BDE8384000F0A5
:1018F00093BC38BD10B5012104460430FFF71AFF30
:101900000023237784F8543010BD000038B5044616
:101910000025143001F0E4FD04F14C00257701F0BE
:10192000B3FE201D84F854500121FFF703FF204629
:10193000BDE83840FFF74EBF90F8803003F06003F9
:10194000202B19D190F88120212A0AD0222A4FF089
:1019500000030ED0202A0FD1084A4267072282676F
:1019600004E0064B4367072383670023C367012016
:10197000704743678367F9E7002070471C24002005
:10198000D0F8943437B51A680446117804291AD16E
:10199000017C022917D11979012312898B40134246
:1019A00011D100F14C05284601F02EFF58B101A9D4
:1019B000284601F075FED4F894440246019B217933
:1019C000206800F0C7F803B030BD000001F10B0340
:1019D000F7B550F8234005460E46F4B1202383F3B3
:1019E000118805EB8607201D08214C34FFF7A2FE65
:1019F000FB685B691B6813B1204601F05FFE01A91B
:101A0000204601F04DFE024648B1019B3146284672
:101A100000F0A0F8002383F3118803B0F0BDFB6849
:101A20005A691268002AF5D01B8A013B1340F1D194
:101A300005F18002EAE70000133138B550F8214083
:101A4000DCB1202383F31188D4F8942413685279ED
:101A500003EB8203DB689B695D6845B10421601874
:101A6000FFF768FE294604F1140001F04FFD2046FF
:101A7000FFF7B0FE002383F3118838BD70470000E4
:101A800001F04AB8012300F1300200F15001037067
:101A90000023436042F8043B8A42D361FAD10381B8
:101AA0004381704738B50446202383F3118800250D
:101AB00000F10C0300F13002416043F8045B9342F3
:101AC000FBD1204601F04AF80223237085F31188E8
:101AD00038BD000070B500EB8103054650690E4625
:101AE0001446DA6018B110220021FFF75BFAA069F2
:101AF00018B110220021FFF755FA31462846BDE8FB
:101B0000704001F03DB90000038900F1300200216E
:101B100003F001030381438903F00103438100F1D2
:101B2000100343F8041B9342FBD101F0C1B900003C
:101B3000F0B4012500EB810447898D40E4683D4302
:101B4000A469458123600023A2606360F0BC01F0BA
:101B5000DDB90000F0B4012500EB810407898D4058
:101B6000E4683D436469058123600023A2606360EB
:101B7000F0BC01F055BA0000022300F10C0200F1A4
:101B8000300110B5037004460023A0F8883080F8B7
:101B90008A3080F88B300381438142F8043B8A42CB
:101BA000FBD184F87030204601F07EF863681B6832
:101BB00023B120460021BDE81040184710BD0000A9
:101BC0000278436880F88C2005221B6802700BB1F4
:101BD0000421184770470000436890F88C201B6868
:101BE00002700BB1052118477047000090F8703063
:101BF00070B5044613B1002380F8703004F1800200
:101C0000204601F079F963689B6863BB94F88050C3
:101C100015F0600615D194F8813005F07F0545EA8E
:101C2000032540F202339D4200F00E815BD8022D65
:101C300000F0DC803FD8002D00F08780012D00F0FF
:101C4000CF800021204601F00FFC0021204601F04A
:101C5000FFFB63681B6813B10621204698470623E3
:101C600084F8703070BD204698470028CED094F894
:101C7000872094F8863043EA0223A26F934238BF4C
:101C8000A36794F98030A56F002B4FF0200380F2FA
:101C9000FD80002D00F0EC80092284F8702083F391
:101CA00011880021A36F626F2046FFF753FF0023C6
:101CB00083F3118870BDB5F5817F00F0B180B5F573
:101CC000407F49D0B5F5807FBBD194F88230012B9D
:101CD000B7D1B4F8883023F00203A4F888306667DF
:101CE000A667E667C3E740F201639D421ED8B5F5DB
:101CF000C06F3BD2B5F5A06FA3D1B4F88030B3F577
:101D0000A06F0ED194F88230204684F88A3001F01A
:101D100029F863681B6813B1012120469847032303
:101D2000237000236367A367E367A0E7B5F5106F2F
:101D300032D040F602439D4252D0B5F5006F80D1BB
:101D400004F18B036367012324E004F18803E56752
:101D500063670223A3678AE794F88230012B7FF43C
:101D600070AFB4F8883043F00203B6E794F88520EA
:101D70002046616894F884304D6843EA022394F861
:101D8000831094F88220A84700283FF45AAF436894
:101D900063670368A367A4E72378042B10D120238B
:101DA00083F311882046FFF7AFFE86F3118863683E
:101DB000032184F88B601B6821700BB12046984783
:101DC00094F88230002BACD084F88B30042323703D
:101DD00063681B68002BA4D0022120469847A0E727
:101DE000374B63670223A36700239DE794F88410B1
:101DF000204611F0800F01F00F010ED001F06EF8B7
:101E0000012806D002287FF41CAF2E4BA067636721
:101E100067E72D4BA567636763E701F051F8EFE7CC
:101E200094F88230002B7FF40CAF94F8843013F0D8
:101E30000F013FF476AF1A06204602D501F02CFBC5
:101E40006FE701F01DFB6CE794F88230002B7FF404
:101E5000F8AE94F8843013F00F013FF462AF1B0624
:101E6000204602D501F000FB5BE701F0F1FA58E7EC
:101E7000142284F8702083F311882B462A462946C1
:101E80002046FFF755FE85F3118870BD5DB1152220
:101E900084F8702083F311880021A36F626F2046BD
:101EA000FFF746FE03E70B2284F8702083F31188C6
:101EB0002B462A4629462046FFF74CFEE3E700BFA3
:101EC000344100082C4100083041000838B590F832
:101ED00070300446152B29D8DFE803F03E28282867
:101EE00028283E28280B2939282828282828282867
:101EF0003E3E90F8871090F88620836F42EA0122D8
:101F00009A4214D9C268128AB3FBF2F502FB153566
:101F10006DB9202383F311882B462A462946FFF703
:101F200019FE85F311880A2384F8703038BD142314
:101F300084F87030202383F31188002320461A464A
:101F40001946FFF7F5FD002383F3118838BDC36FF1
:101F500003B198470023E7E7002101F085FA00214B
:101F6000204601F075FA63681B6813B1062120460C
:101F700098470623D8E7000090F87020152A38B556
:101F8000044622D80123934040F6416213421DD1FA
:101F900013F480150FD19B0217D50B2380F87030F6
:101FA000202383F311882B462A462946FFF7D2FDCA
:101FB00085F3118838BDC3689B695B682BB9C36F13
:101FC00003B19847002384F8703038BD002101F038
:101FD0004BFA0021204601F03BFA63681B6813B1FD
:101FE0000621204698470623EDE70000024B002219
:101FF0001B605B609A607047AC2A002000238268F7
:102000000374054B1B6899689142FBD25A680360C0
:102010004260106058607047AC2A002008B5202349
:1020200083F31188037C032B05D0042B0DD02BB92F
:1020300083F3118808BD436900221A604FF0FF3313
:102040004361FFF7DBFF0023F2E790E80C001A6022
:1020500002685360F2E70000002382680374054BB6
:102060001B6899689142FBD85A680360426010600F
:1020700058607047AC2A0020054B1969087418682D
:10208000026853601A60186101230374FEF79CB95B
:10209000AC2A00204B1C30B5054687B00A4C10D046
:1020A000236901A8094A00F0D3F82846FFF7E4FFA6
:1020B000049B13B101A800F007F92369586907B020
:1020C00030BDFFF7D9FFF8E7AC2A00201D2000083B
:1020D00038B50C4D044641612B6981689A6891427C
:1020E00003D8BDE83840FFF789BF1846FFF786FFE1
:1020F00001232C61014623742046BDE83840FEF7D9
:1021000063B900BFAC2A0020044B1A681B699068B1
:102110009B68984294BF002001207047AC2A0020A1
:1021200010B5084C236820691A68546022600122A7
:1021300023611A74FFF790FF01462069BDE8104043
:10214000FEF742B9AC2A002082600222027400220B
:10215000427470478368A3F17C0243F80C2C026937
:1021600043F83C2C426943F8382C074A43F81C2CAE
:10217000C268A3F1180043F8102C022203F8082CBF
:10218000002203F8072C7047E103000810B5202354
:1021900083F31188FFF7DEFF00210446FFF798FF65
:1021A000002383F31188204610BD0000024B1B69F9
:1021B00058610F20FFF760BFAC2A0020202383F373
:1021C0001188FFF7F3BF000008B50146202383F311
:1021D00011880820FFF75EFF002383F3118808BDF4
:1021E00049B1064B42681B6918605A60136043602E
:1021F0000420FFF74FBF4FF0FF307047AC2A00209C
:102200000368984206D01A68026050601846596107
:10221000FFF7F4BE7047000038B504460D4620684D
:10222000844200D138BD036823605C604561FFF7DC
:10223000E5FEF4E7054B03F114025A619A614FF091
:10224000FF32DA6100221A62704700BFAC2A002018
:10225000F8B503614FF08043C26002295C6A06460C
:10226000184B38BF02211A461F4652F8145F954298
:102270000AD1586198611C62056045608160081947
:10228000BDE8F84001F0E2BA186AAB68241A0C19EC
:1022900002D3E41A2D6804E09C4202D2204401F0EB
:1022A000E3FAAB689C42F4D86B68356073601E60DB
:1022B0004FF0FF336E60B460A968091BA960FB6131
:1022C000F8BD00BFAC2A002010B41B4C234653F8C5
:1022D000141F814210D0416802680A600268516090
:1022E0009A424FF00001C16003D0936881680B44AB
:1022F00093605DF8044B70470A6800209A4262615F
:102300005360C86003D15DF8044B01F0A7BA93682D
:1023100088680344206A93604FF08042526A121A20
:102320009342E6D9991A5DF8044B012998BF931C92
:10233000184401F099BA00BFAC2A00200020704771
:10234000FEE70000704700004FF0FF3070470000CC
:10235000022906D0032906D00129064818BF00200B
:10236000704705487047032A9ABF044800EBC20033
:102370000020704704420008B841000824240020CF
:1023800070B59AB006460846144601AD294600F0DD
:1023900095F82846FEF7FEFDC0B2431C5B0086E8B8
:1023A000180023700323023404F8013C002319466B
:1023B000DAB20234904201D81AB070BDEA5C01333F
:1023C00004F8011C04F8022CF2E7000008B52023F1
:1023D00083F311880348FFF7D3FA002383F31188AE
:1023E00008BD00BFEC2A002010B50446052916D808
:1023F000DFE801F016150316161D202383F311885C
:102400000E4A0121FFF766FB20460D4A0221FFF725
:1024100061FB0C48FFF77AFA002383F3118810BDA3
:10242000202383F311880748FFF746FAF4E72023B7
:1024300083F311880348FFF75DFAEDE738410008A0
:102440005C410008EC2A002038B50C4D0C4C2A46A3
:102450000C4904F10800FFF793FF05F1CA0204F1EB
:1024600010000949FFF78CFF05F5CA7204F1180046
:102470000649BDE83840FFF783BF00BFB42F0020F6
:102480002424002088410008924100089D41000852
:1024900070B5044608460D46FEF77CFDC6B22046E0
:1024A000013403780BB9184670BD32462946FEF751
:1024B0005BFD0028F3D1012070BD00002DE9F84F2D
:1024C00005460C46FEF766FD2B49C6B22846FFF7C7
:1024D000DFFF2A492846FFF7DBFF08B11036F6B2C6
:1024E000632E0DD8DFF89080DFF89090244FDFF84E
:1024F00098A0DFF898B02E7846B92670BDE8F88F1E
:1025000029462046BDE8F84F01F0B6BD252E2ED154
:10251000072241462846FEF727FD70B9DBF8003058
:102520000735073444F8073CBBF8043024F8033C73
:102530009BF8063004F8013CDDE7082249462846AE
:10254000FEF712FD98B9A21C0E4B13F8011F0232C0
:1025500009095345C95D02F8041C197801F00F01FF
:10256000C95D02F8031CF0D118340835C3E72670A2
:1025700001350134BFE700BF244200089D41000837
:1025800034420008FFE7F11F0BE8F11F2C4200085E
:10259000BFF34F8F044B1A695107FCD1D3F81021B8
:1025A0005207F8D1704700BF0020005208B50D4B0C
:1025B0001B78ABB9FFF7ECFF0B4BDA68D10704D5FA
:1025C0000A4A5A6002F188325A60D3F80C21D207C5
:1025D00006D5064AC3F8042102F18832C3F8042163
:1025E00008BD00BF123200200020005223016745C1
:1025F00008B5114B1B78F3B9104B1A69510703D575
:10260000DA6842F04002DA60D3F81021520705D5AB
:10261000D3F80C2142F04002C3F80C21FFF7B8FFB9
:10262000064BDA6842F00102DA60D3F80C2142F07E
:102630000102C3F80C2108BD123200200020005214
:102640000F289ABF00F5806040040020704700000A
:102650004FF4003070470000102070470F2808B575
:102660000BD8FFF7EDFF00F500330268013204D10B
:1026700004308342F9D1012008BD002008BD0000CC
:102680000F2810B504463FD8FFF782FFFFF78EFFF3
:102690001E484FF0FF33072C4361C0F814311DD89A
:1026A0000361FFF775FF230243F02403C360C3688F
:1026B00043F08003C36003695A07FCD4FFF768FF47
:1026C0002046FFF7BDFF4FF4003100F0F7F8FFF7A9
:1026D0008FFF2046BDE81040FFF7C0BFC0F81031A3
:1026E000FFF756FFA4F108031B0243F02403C0F8D0
:1026F0000C31D0F80C3143F08003C0F80C31D0F825
:1027000010315B07FBD4D9E7002010BD0020005238
:102710002DE9F84F40EA020305460E461746DB0650
:1027200056D13446DFF8C090DFF8C0A0FFF73EFF77
:102730003B1B33441F2B04D8FFF75AFF0120BDE891
:10274000F88F20222146284601F086FC002837D049
:1027500005F17843214A22489342224B98BF98467C
:1027600003F5827392BFD346C8469B46A3F1080384
:1027700088BF1846FFF70CFF4FF0FF3304F11C0130
:10278000A5EB040ECBF80030036843F002030360AE
:10279000231FD8F8002012F0050FFAD153F8042FA8
:1027A00099424EF80320F4D1BFF34F8FFFF7F0FEAC
:1027B0004FF0FF33CBF80030036823F002030360CF
:1027C00020222146284601F047FC20B1FFF710FFE8
:1027D0000020BDE8F88F20352034A9E7FFFF0F0067
:1027E0000C200052102000521021005214200052E0
:1027F00010B5084C237828B153B9FFF7D7FE012351
:10280000237010BD23B12070BDE81040FFF7F0BE6B
:1028100010BD00BF1232002002440439064BD2B270
:1028200010B5904200D110BD441C00B253F82000F6
:1028300041F8040FE0B2F4E7504000580F4B30B5B8
:102840001C6F240405D41C6F1C671C6F44F40044E7
:102850001C670B4C024404392368D2B243F48073E2
:102860002360084B904200D130BD441C51F8045FF6
:1028700000B243F82050E0B2F4E700BF0044025831
:10288000004802585040005807B5012201A9002015
:10289000FFF7C2FF019803B05DF804FB13B50446CF
:1028A000FFF7F2FFA04206D002A90122002041F862
:1028B000044DFFF7C3FF02B010BD00000144BFF399
:1028C0004F8F064B884204D3BFF34F8FBFF36F8FF8
:1028D0007047C3F85C022030F4E700BF00ED00E071
:1028E000034B1B685B0142BF0122024B1A70704709
:1028F000D044025813320020014B1878704700BFB3
:1029000013320020064A536823F001035360EFF3AB
:102910000983683383F30988002383F311887047A0
:1029200030EF00E010B5202383F31188104B5B6873
:1029300013F4006318D0F1EE103AEFF309844FF06E
:10294000807344F84C3C0B4BDB6844F8083CA4F122
:10295000680383F30988FFF7D7FB18B1064B44F8E7
:10296000503C10BD054BFAE783F3118810BD00BF42
:1029700000ED00E030EF00E0F1030008F403000890
:10298000F0B5BFF34F8FBFF36F8F1D4B0021C3F81E
:102990005012BFF34F8FBFF36F8F5A6942F400326A
:1029A0005A61BFF34F8FBFF36F8FC3F88410BFF32B
:1029B0004F8FD3F8802043F6E076C2F3C904C2F308
:1029C0004E32A507520102EA060E284621464EEA7B
:1029D0000007013900F14040C3F860724F1CF6D186
:1029E000203A12F1200FEED1BFF34F8F5A6942F413
:1029F00080325A61BFF34F8FBFF36F8FF0BD00BFBE
:102A000000ED00E0FEE70000084A094B09498B424F
:102A100004D3094A0021934205D3704752F8040FAA
:102A200043F8040BF3E743F8041BF4E720440008E1
:102A3000603500206035002060350020D0F89430EB
:102A4000002230B51146D0F890409D684FF0FF301D
:102A500004EB421301329542C3F80019C3F8101970
:102A6000C3F80809C3F8001BC3F8101BC3F8080B10
:102A7000EED24FF00113C4F81C3830BD00EB8103D7
:102A80002DE9F04FD3F80CE04F1C4FEA4118DEF867
:102A900014403F03D4F800C06568D0F89020654525
:102AA0000AD30120D2F8343800FA01F123EA0101F7
:102AB000C2F83418BDE8F08FACEB0503BEF8106027
:102AC000B34228BF334602EB0806D6F81869B6B2FF
:102AD000B3EB860F13D8A6683A449946A6F1040AC8
:102AE0005AF804BFB9F1040FC2F800B002D9A9F135
:102AF0000409F5E71E442B44A6606360CCE7002080
:102B0000BDE8F08F890141F02001016103699B0656
:102B1000FCD4122000F034BF10B50A4C2046FEF75A
:102B2000B1FF094BC4F89030084BC4F89430084CFE
:102B30002046FEF7A7FF074BC4F89030064BC4F8B9
:102B4000943010BD14320020000008406C42000890
:102B5000B032002000000440784200080378012BC6
:102B600070B505465DD1494BD0F89040984259D197
:102B7000474B0E216520D3F8D82042F00062C3F8FD
:102B8000D820D3F8002142F00062C3F80021D3F826
:102B90000021D3F8802042F00062C3F88020D3F8EF
:102BA000802022F00062C3F88020D3F88030FEF746
:102BB000E3FB384BE360384BC4F800380023D5F80A
:102BC0009060C4F8003EC02323604FF40413A36355
:102BD0003369002BFCDA01230C20336100F0D0FEB6
:102BE0003369DB07FCD4122000F0CAFE3369002BE6
:102BF000FCDA00262846A660FFF720FF6B68C4F8C1
:102C00001068DB68C4F81468C4F81C68002B3AD15B
:102C1000224BA3614FF0FF336361A36843F00103CC
:102C2000A36070BD1E4B9842C8D1194B0E214D2098
:102C3000D3F8D82042F00072C3F8D820D3F800218E
:102C400042F00072C3F80021D3F80021D3F88020AD
:102C500042F00072C3F88020D3F8802022F0007286
:102C6000C3F88020D3F88020D3F8D82022F08062E7
:102C7000C3F8D820D3F8002122F08062C3F80021E5
:102C8000D3F8003193E7074BC3E700BF14320020AD
:102C9000004402584014004003002002003C30C0B1
:102CA000B0320020083C30C0F8B5D0F8904005465E
:102CB00000214FF000662046FFF724FFD5F894105E
:102CC00000234FF001128F684FF0FF30C4F8343802
:102CD000C4F81C2804EB431201339F42C2F8006978
:102CE000C2F8006BC2F80809C2F8080BF2D20B68F0
:102CF000D5F89020C5F898306362102313611669E7
:102D000016F01006FBD1122000F03AFED4F800387D
:102D100023F4FE63C4F80038A36943F4402343F06E
:102D20001003A3610923C4F81038C4F814380B4BFE
:102D3000EB604FF0C043C4F8103B094BC4F8003BB4
:102D4000C4F81069C4F80039D5F8983003F11002BE
:102D500043F48013C5F89820A362F8BD48420008E8
:102D600040800010D0F8902090F88A10D2F80038F7
:102D700023F4FE6343EA0113C2F8003870470000F1
:102D80002DE9F0410EB20D4600EB8608D8F80C1084
:102D90000F6807F00303022B53D0032B53D03F4A95
:102DA0003F4F012B18BF1746D0F890404FEA451E01
:102DB000002205F1100C04EB0E03C3F8102B8A69F6
:102DC000002A42D04A8A05F158033A435B01E25097
:102DD0000123D4F81C2803FA0CF31343C4F81C385D
:102DE000A64400234A69CEF8103905F13F03002AB2
:102DF0003BD00A8A04EB8303898B9208012988BFA0
:102E00004A43D0F89810561841EA02422946C0F8C1
:102E1000986020465A60FFF775FED8F80C301B8A80
:102E200043EA85531F4305F148035B01E750012343
:102E3000D4F81C2803FA05F51543C4F81C58BDE85E
:102E4000F081184FB0E7184FAEE704EB4613D3F804
:102E5000002B22F40042C3F8002B0123D4F81C28D5
:102E600003FA0CF322EA0303B8E704EB83030F4AE7
:102E700004EB461629465A602046FFF743FED6F873
:102E80000039012223F4004302FA05F5C6F800399F
:102E9000D4F81C3823EA0505CFE700BF00800010F6
:102EA000008004100080081000800C100004000254
:102EB000D0F894201268C0F89820FFF7BFBD00003A
:102EC0005831D0F8903049015B5813F4004004D0D9
:102ED00013F4001F14BF0120022070474831D0F8BE
:102EE000903049015B5813F4004004D013F4001FE4
:102EF00014BF01200220704700EB8101CB68196AE2
:102F00000B6813604B6853607047000000EB81034F
:102F100030B5DD68AA691368D36019B9402B84BF46
:102F2000402313606B8A1468D0F890201C4402EB95
:102F30004110013C09B2B4FBF3F46343033323F0C3
:102F4000030343EAC44343F0C043C0F8103B2B687B
:102F500003F00303012B0ED1D2F8083802EB411025
:102F600013F4807FD0F8003B14BF43F0805343F04C
:102F70000053C0F8003B02EB4112D2F8003B43F093
:102F80000443C2F8003B30BD2DE9F041D0F8906019
:102F900005460C4606EB4113D3F8087B3A07C3F805
:102FA000087B08D5D6F814381B0704D500EB81033D
:102FB000DB685B689847FA072FD5D6F81438DB072B
:102FC0002BD505EB8403D968CCB98B69488A5E6838
:102FD000B6FBF0F200FB12628AB91868DA68904218
:102FE0000DD2121A83E81400202383F3118821469E
:102FF0002846FFF78BFF84F31188BDE8F081012399
:1030000003FA04F26B8923EA02036B81CB6823B1D4
:1030100021462846BDE8F0411847BDE8F081000090
:1030200000EB81034A0170B5DD68D0F890306C691F
:103030002668E66056BB1A444FF40020C2F8100917
:103040002A6802F00302012A0AB20ED1D3F8080856
:1030500003EB421410F4807FD4F8000914BF40F051
:10306000805040F00050C4F8000903EB4212D2F83F
:10307000000940F00440C2F800090122D3F83408E6
:1030800002FA01F10143C3F8341870BD19B9402E9A
:1030900084BF4020206020681A442E8A841940F0A2
:1030A0000050013CB4FBF6F440EAC440C6E700001F
:1030B0002DE9F041D0F8906004460D4606EB41132F
:1030C000D3F80879C3F80879FB071CD5D6F810386F
:1030D000DA0718D500EB8103D3F80CE0DEF81430E2
:1030E000D3F800C0DA6894451BD2A2EB0C024FF073
:1030F00000081A60C3F80480202383F31188FFF7C7
:103100008FFF88F311883B0618D50123D6F83428A1
:10311000AB40134212D029462046BDE8F041FFF7EC
:10312000ADBC012303FA01F2038923EA0203038100
:10313000DEF80830002BE6D09847E4E7BDE8F081E0
:103140002DE9F047D0F8905004466E69AB691E40F7
:10315000F1046E6103D5BDE8F047FEF70DBD002E0A
:1031600012DAD5F8003E9A0705D0D5F8003E23F0D4
:103170000303C5F8003ED5F80438204623F00103C8
:10318000C5F80438FEF728FD330502D52046FEF7C2
:1031900017FDB7040CD5D5F8083813F0060FEB6807
:1031A00023F470530CBF43F4105343F4A053EB606B
:1031B000300704D56368DB680BB120469847F102FD
:1031C00000F1A180B2020BD5D4F8908000274FF017
:1031D0000109D4F89430F9B29B688B4280F0D28018
:1031E000F3061AD5D4F890100A6AC2F30A1702F04F
:1031F0000F0302F4F012B2F5802F00F0EB80B2F56D
:10320000402F0AD104EB830301F58051DB68186A73
:1032100000231A469F4240F0D1803003D5F8185859
:1032200035D5E90303D500212046FFF7ADFEAA03FB
:1032300003D501212046FFF7A7FE6B0303D502212A
:103240002046FFF7A1FE2F0303D503212046FFF7F9
:103250009BFEE80203D504212046FFF795FEA90254
:1032600003D505212046FFF78FFE6A0203D506210C
:103270002046FFF789FE2B0203D507212046FFF7E2
:1032800083FEEF0103D508212046FFF77DFE700382
:1032900040F1C780E90703D500212046FFF708FF6A
:1032A000AA0703D501212046FFF702FF6B0703D5CC
:1032B00002212046FFF7FCFE2F0703D503212046FD
:1032C000FFF7F6FEEE0603D504212046FFF7F0FED9
:1032D000A80603D505212046FFF7EAFE690603D5B7
:1032E00006212046FFF7E4FE2A0603D507212046E3
:1032F000FFF7DEFEEB0540F1948020460821BDE893
:10330000F047FFF7D5BED4F890904FF000084FF08B
:10331000010AD4F894305FFA88F79B68BB42FFF447
:1033200051AF09EB4713D3F8002902F44022B2F55C
:10333000802F24D1D3F80029002A20DAD3F80029DD
:1033400042F09042C3F80029D3F80029002AFBDBA1
:103350003946D4F89000FFF7D5FB22890AFA07F323
:1033600022EA0303238104EB8703DB689B6813B124
:1033700039462046984739462046FFF77FFB08F13B
:103380000108C6E708EB4112D2F8003B03F44023E2
:10339000B3F5802F10D1D2F8003B002B0CDA6289F4
:1033A00009FA01F322EA0303638104EB8103DB687A
:1033B000DB680BB12046984701370AE713F0030F8B
:1033C00000D10A68072B03F101039EBF0270120AA5
:1033D00001301FE704EB830301F58051DA6890693F
:1033E0000268D0F808C04068A2EB000E0022104628
:1033F000974208D1DB689B699A683A449A605A6898
:1034000017445F6009E712F0030F00D10868964582
:1034100002F1010282BF8CF80000000A0CF1010CDD
:10342000E6E7BDE8F087000008B50348FFF788FE2F
:10343000BDE80840FFF776BA1432002008B503480B
:10344000FFF77EFEBDE80840FFF76CBAB0320020FF
:10345000D0F8903003EB4111D1F8003B43F4001356
:10346000C1F8003B70470000D0F8903003EB4111E9
:10347000D1F8003943F40013C1F800397047000057
:10348000D0F8903003EB4111D1F8003B23F4001346
:10349000C1F8003B70470000D0F8903003EB4111B9
:1034A000D1F8003923F40013C1F800397047000047
:1034B00030B50433039C0172002104FB0325C36172
:1034C000049B00600363059B4060C1604261026130
:1034D0008561046242628162C162436330BD000063
:1034E0000022416AC260416101616FF001018262A4
:1034F000C262FEF791BE000003694269934203D1A4
:10350000C2680AB100207047181D7047036919602E
:103510000021C2680132C260C269134482699342C9
:10352000036124BF436A0361FEF76ABE38B50446EF
:103530000D46E3683BB162690020131D1268A36267
:103540001344E36238BD237A33B929462046FEF797
:1035500047FE0028EDDA38BD6FF00100FBE7000000
:10356000C368C269013BC3604369134482699342E3
:10357000436124BF436A436100238362036B03B149
:103580001847704770B52023044683F31188866A74
:103590003EB9FFF7CBFF054618B186F311882846E0
:1035A00070BDA36AE26A13F8015B9342A36202D37F
:1035B0002046FFF7D5FF002383F31188EFE70000D3
:1035C0002DE9F84F04460E4690469946202787F38A
:1035D00011880025AA46D4F828B0BBF1000F09D104
:1035E00049462046FFF7A2FF20B18BF311882846F9
:1035F000BDE8F88FA16AA8EB050BE36A5B1A9B454F
:1036000028BF9B46BBF1400F1BD9334601F1400256
:1036100051F8040B914243F8040BF9D1A36A4036E8
:1036200040354033A362A26AE36A9A4202D320463D
:10363000FFF796FF8AF311884545D8D287F31188A2
:10364000C9E730465A46FDF785FCA36A5E445D44EF
:103650005B44A362E7E7000010B5029C04330172EB
:10366000C36103FB0421002300608362C362039BE8
:1036700040600363049BC460426102618161046233
:103680004262436310BD0000026A6FF00101C26034
:10369000426A4261026100228262C262FEF7BCBDE0
:1036A000436902699A4203D1C2680AB10020704797
:1036B000184650F8043B0B6070470000C3680021B7
:1036C000C2690133C3604369134482699342436111
:1036D00024BF436A4361FEF793BD000038B504463A
:1036E0000D46E3683BB1236900201A1DA262E2691E
:1036F0001344E36238BD237A33B929462046FEF7E6
:103700006FFD0028EDDA38BD6FF00100FBE7000027
:1037100003691960C268013AC260C26913448269D0
:103720009342036124BF436A036100238362036BF6
:1037300003B118477047000070B5202304460E46B9
:1037400083F31188856A35B91146FFF7C7FF10B1B9
:1037500085F3118870BDA36A1E70A36AE26A013303
:103760009342A36204D3E16920460439FFF7D0FFF6
:10377000002080F3118870BD2DE9F84F04460D46F6
:1037800091469A464FF0200888F311880026B346E8
:10379000A76A4FB951462046FFF7A0FF20B187F333
:1037A00011883046BDE8F88FA06AA9EB0603E76AE6
:1037B0003F1A9F4228BF1F46402F1BD905F14003E7
:1037C00055F8042B9D4240F8042BF9D1A36A4036EA
:1037D0004033A362A26AE36A9A4204D3E1692046B5
:1037E0000439FFF795FF8BF311884E45D9D288F342
:1037F0001188CDE729463A46FDF7ACFBA36A3D4464
:103800003E443B44A362E5E7026943699A4203D11F
:10381000C3681BB9184670470023FBE7836A002B77
:10382000F8D0043B9B1AF5D01360C368013BC3601A
:10383000C3691A4483699A42026124BF436A0361DF
:10384000002383620123E5E700F04AB94FF080438B
:10385000002258631A610222DA60704700224FF09A
:103860008043DA60704700004FF080435863704730
:10387000FEE7000010B5194CFEF7B8FBFEF7DAFCC6
:10388000802217492046FEF75FFC012344F8180CFC
:103890000374144B144AD96821F4E0610904090C3B
:1038A0000A431249DA60CA6842F08072CA60104A5C
:1038B0001049C2F8B01F116841F0010111601022D7
:1038C000DA77202283F82220002383F3118862B65E
:1038D0000948BDE81040FEF759BC00BFD42A0020BB
:1038E0008442000800ED00E00003FA05F0ED00E07E
:1038F000001000E055CEACC58C4200082DE9F84F11
:103900001E4C4FF00008656904F11407C1464FF0E2
:103910008043266AAA685B6A9E1B96421CD34FF0BE
:10392000200AAA68236AD5F80CB0B61A1344236299
:103930002B68BB425F606361C5F80C8001D1FFF763
:103940008DFF89F311882869D8478AF31188656942
:10395000AB689E42E5D2DAE76269BA420CD0916860
:1039600023628E1B9660A86802282CBF1818981C2A
:10397000BDE8F84FFFF778BFBDE8F88FAC2A00200C
:10398000034B59685A68521A9042FBD8704700BFDF
:10399000001000E04B6843608B688360CB68C360B5
:1039A0000B6943614B6903628B6943620B68036077
:1039B0007047000008B52C4B40F2FF712B48D3F83C
:1039C00088200A43C3F88820D3F8882022F4FF62B5
:1039D00022F00702C3F88820D3F88820D3F8E0202B
:1039E0000A43C3F8E020D3F808210A43C3F80821AA
:1039F0001F4AD3F808311146FFF7CCFF1D4802F1EA
:103A00001C01FFF7C7FF1C4802F13801FFF7C2FF96
:103A10001A4802F15401FFF7BDFF194802F1700185
:103A2000FFF7B8FF174802F18C01FFF7B3FF164804
:103A300002F1A801FFF7AEFF144802F1C401FFF73D
:103A4000A9FF134802F1E001FFF7A4FF114802F1BA
:103A5000FC01FFF79FFF104802F58C71FFF79AFFFA
:103A6000BDE8084000F016B90044025800000258B2
:103A7000AC4200080004025800080258000C02582A
:103A8000001002580014025800180258001C025876
:103A900000200258002402580028025808B500F0FF
:103AA000C9FAFFF7E7FEFEF71BFFBDE80840FEF787
:103AB000CBBC0000704700004FF080431A699207AA
:103AC00010B508D500241C61202383F31188FFF76B
:103AD00015FF84F31188BDE81040FEF723BF0000F6
:103AE000134B08211C20D3F8E82042F00102C3F850
:103AF000E820D3F8102142F00102C3F810210D4A4A
:103B0000D3F81031D36B43F00103D3634FF08043FC
:103B1000C7229A624FF0FF32DA6200229A615A633A
:103B2000DA605A6001225A611A60FDF725BC00BFB5
:103B3000004402580010005CF8B5514B0024D3F843
:103B400080204FF0FF32C3F88020D3F88010C3F8F4
:103B50008040D3F88010D3F88410C3F88420D3F8C1
:103B60008410C3F88440D3F88410D96F41F0FF412A
:103B700041F4FF0141F4DF4141F07F01D967D96F82
:103B800021F0FF4121F4FF0121F4DF4121F07F0109
:103B9000D967D96FD3F888106FEA41516FEA515154
:103BA000C3F88810D3F88810C1F30A01C3F888104D
:103BB000D3F88810D3F89010C3F89020D3F8901061
:103BC000C3F89040D3F89010D3F89410C3F8942021
:103BD000D3F89410C3F89440D3F89410D3F8981005
:103BE000C3F89820D3F89810C3F89840D3F89810E9
:103BF000D3F88C10C3F88C20D3F88C10C3F88C4009
:103C0000D3F88C10D3F89C10C3F89C20D3F89C20D8
:103C1000C3F89C40D3F89C3000F0ECF9194B072214
:103C20009A60194ADA60194A1A6105225A60184ADC
:103C3000536A43F480335362C2F88440BFF34F8F1A
:103C4000D2F8803043F6E076C3F3C904C3F34E33B1
:103C5000A5075B0103EA060E284621464EEA000747
:103C6000013900F14040C2F874724F1CF6D1203B7C
:103C700013F1200FEED1BFF34F8FBFF36F8FF8BD5D
:103C80000044025890ED00E0000004301B000803DF
:103C900000ED00E001225B4B5B491A605B4B196051
:103CA0009A605B4ADA6000221A614FF440429A61DE
:103CB0009A699204FCD51A6842F480721A60554BD6
:103CC0001A6F12F4407F04D04FF480321A6700223A
:103CD0001A671A6842F001021A604E4A13461168C8
:103CE0004807FCD5002111611A6912F03802FBD196
:103CF000012119604FF0804159605A67464ADA62E3
:103D0000464A1A611A6842F480321A60414A1346E0
:103D100011688903FCD5116841F0800111601A68AF
:103D2000D205FCD53E4A3F499A6200225A63196384
:103D3000A1F58021DA634B3999635A643A4A1A64CF
:103D40003A4ADA621A6842F0A8521A60314B1A688D
:103D500002F02852B2F1285FF9D1482222219A615B
:103D60004FF48862DA6140221A624FF00052DA643E
:103D70001A652F4A5A652F4A9A652F4A11601A69A7
:103D800042F003021A61234B1A6902F03802182A22
:103D9000FAD1D3F8DC2042F00052C3F8DC20D3F88B
:103DA000042142F00052C3F80421D3F80421D3F8CF
:103DB000DC2042F08042C3F8DC20D3F8042142F03A
:103DC0008042C3F80421D3F80421D3F8DC2042F068
:103DD0000042C3F8DC20D3F8042142F00042C3F8CB
:103DE0000421D3F80421D3F8F42042F00202C3F8EE
:103DF000F420D3F81C2142F00202C3F81C21D3F8AE
:103E00001C3170470881005100C000F00048025882
:103E100002000001004402580000FF0100889008E1
:103E2000222040006302070147040508FD0BFF0143
:103E30000010E0000001010000200052084A08B50F
:103E4000936811680B4003F00103936023B1054AA6
:103E500013680BB150689847BDE80840FEF762BD93
:103E600080000058C0250020084A08B593681168F2
:103E70000B4003F00203936023B1054A93680BB132
:103E8000D0689847BDE80840FEF74CBD8000005858
:103E9000C0250020084A08B5936811680B4003F05C
:103EA0000403936023B1054A13690BB15069984725
:103EB000BDE80840FEF736BD80000058C025002050
:103EC000084A08B5936811680B4003F00803936033
:103ED00023B1054A93690BB1D0699847BDE8084002
:103EE000FEF720BD80000058C0250020084A08B514
:103EF000936811680B4003F01003936023B1054AE7
:103F0000136A0BB1506A9847BDE80840FEF70ABD36
:103F100080000058C0250020174B10B59C681A6817
:103F2000144004F478729A60A30604D5134A936A85
:103F30000BB1D06A9847600604D5104A136B0BB1D9
:103F4000506B9847210604D50C4A936B0BB1D06B8C
:103F50009847E20504D5094A136C0BB1506C984799
:103F6000A30504D5054A936C0BB1D06C9847BDE806
:103F70001040FEF7D7BC00BF80000058C0250020CD
:103F80001A4B10B59C681A68144004F47C429A607D
:103F9000620504D5164A136D0BB1506D9847230581
:103FA00004D5134A936D0BB1D06D9847E00404D546
:103FB0000F4A136E0BB1506E9847A10404D50C4AFA
:103FC000936E0BB1D06E9847620404D5084A136F04
:103FD0000BB1506F9847230404D5054A936F0BB17A
:103FE000D06F9847BDE81040FEF79CBC8000005899
:103FF000C0250020062108B50846FDF7BDF90621B9
:104000000720FDF7B9F906210820FDF7B5F90621CB
:104010000920FDF7B1F906210A20FDF7ADF90621C7
:104020001720FDF7A9F906212820BDE80840FDF773
:10403000A3B9000008B5FFF77FFDFDF773F8FDF7A2
:1040400045FBFDF71DFDFDF7EFFBFFF733FDBDE879
:104050000840FFF7F9BB000010B501390244904257
:1040600001D1002010BD10F8013B11F8014FA3420F
:10407000F5D0181B10BD0000034611F8012B03F802
:10408000012B002AF9D170471210121312110000EF
:1040900001105A0003105900012058000320560057
:1040A000EC2A00204026002053544D333248373F3D
:1040B0003F3F0053544D3332483734332F37353375
:1040C000000000000096000000000000000000005A
:1040D00000000000000000000000000000000000E0
:1040E0009516000881160008BD160008A9160008DC
:1040F000B5160008A11600088D16000879160008EC
:10410000C916000800000000A11700088D1700085C
:10411000C9170008B5170008C1170008AD17000837
:1041200099170008851700082518000800000000EE
:10413000010000000000000002000000000000007C
:10414000CD190008391A000840004000842F0020D3
:10415000942F002002000000000000000300000077
:10416000000000007D1A00080000000010000000A0
:10417000A42F00200000000001000000000000004B
:1041800014320020010102004172647550696C6FA5
:10419000740025424F415244252D424C0025534581
:1041A0005249414C25000000E92300085123000832
:1041B00039190008CD23000843000000C041000861
:1041C00009024300020100C032090400000102029A
:1041D000010005240010010524010001042402024D
:1041E0000524060001070582030800FF09040100F9
:1041F000020A0000000705010240000007058102D5
:1042000040000000120000000C42000812011001E2
:1042100002000040091241570002010203010000A0
:104220000403090425424F41524425004355415699
:104230002D58370030313233343536373839414232
:10424000434445460000000000000000ED1B00084C
:10425000CD1E0008791F0008400040004C330020AC
:104260004C330020010000005C330020800000007F
:1042700040010000080000000001000000040000F0
:10428000080000006D61696E00000000A442000893
:1042900068330020603500200100000071380008FC
:1042A0000000000069646C65000000000000802AC6
:1042B00000000000AAAAAAAA00000000FFFF000058
:1042C0000000000000A00A00000000000000000044
:1042D000AAAAAAAA00000000FFFF00000000000038
:1042E000000000000000000000000000AAAAAAAA26
:1042F00000000000FFFF00000000000000000000C0
:104300000000000000000000AAAAAAAA0000000005
:10431000FFFF00000000000000000000000002009D
:1043200000000000AAAAAAAA00000100FFFF0000E6
:1043300000000000070000005025100000000000F1
:10434000AAA2AAAA50151000FFFF00000000000753
:10435000000000000010100000000000AA8AAAAAB5
:1043600000101000FFFF000000000000000000002F
:104370000000000000000000AAAAAAAA0000000095
:10438000FFFF0000000000000000000000551105C4
:10439000E0000000AAAAAAA800011105FFFF000082
:1043A000000000000000000000000000000000000D
:1043B000AAAAAAAA00000000FFFF00000000000057
:1043C000000000000000000000000000AAAAAAAA45
:1043D00000000000FFFF00000000000000000000DF
:1043E000FF00000000000000A84000083F0000009F
:1043F00050040000B34000083F0000000096000099
:104400000000080004000000204200080000000036
:10441000000000000000000000000000000000009C
:1044200000000000FFFFFFFFFFFFFFFFFFFFFFFF98
:10443000FFFFFFFFFFFFFFFFFFFFFFFFFFFFFFFF8C
:10444000FFFFFFFFFFFFFFFFFFFFFFFFFFFFFFFF7C
:10445000FFFFFFFFFFFFFFFFFFFFFFFFFFFFFFFF6C
:10446000FFFFFFFFFFFFFFFFFFFFFFFFFFFFFFFF5C
:020000040801F1
:020000040802F0
:1000000000060030E50D020841A30A08710302084A
:10001000C9A20A08C1A20A08C5A20A08E70D020877
:10002000E70D0208E70D0208E70D020849CA0F08AC
:10003000E70D0208E70D0208E70D0208E70D0208C8
:10004000E70D0208E70D0208E70D0208E70D0208B8
:10005000E70D0208E70D0208254710085147100870
:100060007D471008A9471008D547100851D80F0838
:1000700079D80F08A5D80F08D1D80F08FDD80F08D8
:1000800025D90F0851D90F0825D40F08B5940A08AF
:10009000DD940A08C9940A08F1940A080148100876
:1000A000E70D020865491008E70D020879491008B4
:1000B0007D4910088D491008A14910083DE10F083D
:1000C0006DE10F089DE10F08CDE10F0835ED0F0838
:1000D0004DED0F08ED48100801491008E70D020822
:1000E00065481008E70D0208E70D0208C949100825
:1000F000E70D0208E70D0208E70D02087DD90F0899
:10010000E70D0208D9481008B5491008E70D0208A4
:1001100015491008E70D0208E70D0208E70D02086F
:10012000A9D90F08D1D90F08FDD90F0829DA0F086E
:1001300055DA0F08E70D0208E70D0208E70D02087F
:10014000E70D0208E70D0208E70D0208E70D0208B7
:100150007DDA0F08A9DA0F08D5DA0F082949100847
:10016000FDE10F082DE20F08E70D0208E70D020878
:10017000E70D020885431008E70D0208E70D0208A5
:10018000E70D0208E70D02083D4910085149100823
:1001900065ED0F087DED0F0895ED0F08E70D0208DE
:1001A000E70D0208E70D0208E70D0208E70D020857
:1001B000E70D0208E70D0208E70D02085DE20F08EF
:1001C0008DE20F08E70D0208E70D0208E70D0208AF
:1001D000E70D020871431008E70D0208E70D020859
:1001E000E70D0208E70D0208E70D0208E70D020817
:1001F000E70D0208E70D0208E70D0208E70D020807
:10020000E70D0208E70D0208E70D0208E70D0208F6
:10021000E70D0208E70D0208E70D0208E70D0208E6
:10022000E70D0208E70D0208E70D0208E70D0208D6
:10023000E70D0208E70D0208E70D020845D40F0894
:10024000E70D0208CDD50F08F5D50F0821D60F0808
:100250004DD60F0879D60F08A5D60F08D1D60F08AE
:10026000FDD60F08E70D0208E70D0208E70D0208AA
:10027000E70D0208E70D0208E70D0208E70D020886
:10028000E70D0208E70D0208E70D0208E70D020876
:10029000E70D0208E70D0208E70D0208E70D020866
:1002A000E70D0208E70D0208E70D0208E70D020856
:1002B000E70D0208E70D0208E70D0208E70D020846
:1002C000E70D0208E70D0208E70D0208E70D020836
:1002D000E70D0208E70D0208E70D0208E70D020826
:1002E000DD2D020829C30208FD050308AD860308B9
:1002F00081C40408A5FC06082D25070851920708AB
:10030000C19B0708119F070851250808E12B080821
:10031000AD4B08082554080839720808FD0E090875
:10032000E11B090899970A08E99B0A08A9B70A0876
:10033000752C0C08B16B0C085DBB0C08A9D80C0817
:10034000B1030E08B5680E08F5820E08A19F0E08CD
:1003500029B70E085DDE0E08B1E90E084D1F0F0823
:1003600011250F08FFFFFFFFFFFFFFFFFFFFFFFF4C
:10037000EFF30383EFF30982EFF30881DFF814D082
:100380002DE9FE4F684600F0F7FFBDE8FE4F8D46B1
:1003900070470000642C0030F1EE101AA0EC200A27
:1003A00001607047A0EC108A704700BF81F00041E7
:1003B00002E000BF83F0004330B54FEA41044FEA4A
:1003C000430594EA050F08BF90EA020F1FBF54EAE5
:1003D000000C55EA020C7FEA645C7FEA655C00F081
:1003E000E2804FEA5454D4EB5555B8BF6D420CDD52
:1003F0002C4480EA020281EA030382EA000083EAD5
:10040000010180EA020281EA0303362D88BF30BD74
:1004100011F0004F4FEA01314FF4801C4CEA1131CA
:1004200002D0404261EB410113F0004F4FEA033329
:100430004CEA133302D0524263EB430394EA050FB4
:1004400000F0A780A4F10104D5F1200E0DDB02FA23
:100450000EFC22FA05F2801841F1000103FA0EF2B7
:10046000801843FA05F359410EE0A5F120050EF17D
:10047000200E012A03FA0EFC28BF4CF0020C43FAAE
:1004800005F3C01851EBE37101F0004507D54FF0BB
:10049000000EDCF1000C7EEB00006EEB0101B1F50B
:1004A000801F1BD3B1F5001F0CD349085FEA300051
:1004B0004FEA3C0C04F101044FEA445212F5800F5C
:1004C00080F09A80BCF1004F08BF5FEA500C50F1F9
:1004D000000041EB045141EA050130BD5FEA4C0CDC
:1004E000404141EB0101013C28BFB1F5801FE9D239
:1004F00091F0000F04BF01460020B1FA81F308BF5C
:100500002033A3F10B03B3F120020CDA0C3208DD27
:1005100002F1140CC2F10C0201FA0CF021FA02F102
:100520000CE002F11402D8BFC2F1200C01FA02F172
:1005300020FA0CFCDCBF41EA0C019040E41AA2BF97
:1005400001EB0451294330BD6FEA04041F3C1CDA5F
:100550000C340EDC04F11404C4F1200220FA04F07F
:1005600001FA02F340EA030021FA04F345EA030129
:1005700030BDC4F10C04C4F1200220FA02F001FAEB
:1005800004F340EA0300294630BD21FA04F029466D
:1005900030BD94F0000F83F4801306BF81F4801106
:1005A0000134013D4EE77FEA645C18BF7FEA655C79
:1005B00029D094EA050F08BF90EA020F05D054EA4B
:1005C000000C04BF1946104630BD91EA030F1EBF50
:1005D0000021002030BD5FEA545C05D14000494154
:1005E00028BF41F0004130BD14F580043CBF01F547
:1005F000801130BD01F0004545F0FE4141F470012D
:100600004FF0000030BD7FEA645C1ABF1946104607
:100610007FEA655C1CBF0B46024650EA013406BF08
:1006200052EA033591EA030F41F4002130BD00BFC7
:1006300090F0000F04BF0021704730B54FF4806484
:1006400004F132044FF000054FF0000150E700BF05
:1006500090F0000F04BF0021704730B54FF4806464
:1006600004F1320410F0004548BF40424FF0000151
:100670003EE700BF42004FEAE2014FEA31014FEA94
:1006800002701FBF12F07F4393F07F4F81F06051E3
:10069000704732F07F4208BF704793F07F4F04BF2E
:1006A00041F40021704730B54FF4607401F000450B
:1006B00021F000411CE700BF50EA010208BF70476B
:1006C00030B54FF000050AE050EA010208BF70475C
:1006D00030B511F0004502D5404261EB41014FF4C5
:1006E000806404F132045FEA915C3FF4D8AE4FF0CD
:1006F00003025FEADC0C18BF03325FEADC0C18BFB0
:10070000033202EBDC02C2F1200300FA03FC20FA00
:1007100002F001FA03FE40EA0E0021FA02F114444D
:10072000BDE600BF80F0004002E000BF81F0004164
:1007300042001FBF5FEA410392EA030F7FEA226C87
:100740007FEA236C6AD04FEA1262D2EB1363C1BF17
:10075000D218414048404140B8BF5B42192B88BF86
:10076000704710F0004F40F4000020F07F4018BFA9
:10077000404211F0004F41F4000121F07F4118BFC9
:10078000494292EA030F3FD0A2F1010241FA03FC71
:1007900010EB0C00C3F1200301FA03F100F0004359
:1007A00002D5494260EB4000B0F5000F13D3B0F121
:1007B000807F06D340084FEA310102F10102FE2A90
:1007C00051D2B1F1004F40EBC25008BF20F0010000
:1007D00040EA03007047490040EB0000013A28BF9F
:1007E000B0F5000FEDD2B0FA80FCACF1080CB2EB22
:1007F0000C0200FA0CF0AABF00EBC25052421843A0
:10080000BCBFD0401843704792F0000F81F4000144
:1008100006BF80F400000132013BB5E74FEA410317
:100820007FEA226C18BF7FEA236C21D092EA030F83
:1008300004D092F0000F08BF0846704790EA010FFD
:100840001CBF0020704712F07F4F04D1400028BF2A
:1008500040F00040704712F100723CBF00F500000C
:10086000704700F0004343F0FE4040F40000704742
:100870007FEA226216BF08467FEA236301464202EE
:1008800006BF5FEA412390EA010F40F48000704701
:100890004FF0000304E000BF10F0004348BF4042A7
:1008A0005FEA000C08BF704743F0964301464FF0E3
:1008B00000001CE050EA010208BF70474FF000033F
:1008C0000AE000BF50EA010208BF704711F0004380
:1008D00002D5404261EB41015FEA010C02BF844650
:1008E0000146002043F0B64308BFA3F18053A3F5AF
:1008F0000003BCFA8CF2083AA3EBC25310DB01FAF6
:1009000002FC634400FA02FCC2F12002BCF1004F79
:1009100020FA02F243EB020008BF20F0010070470A
:1009200002F1200201FA02FCC2F1200250EA4C005E
:1009300021FA02F243EB020008BF20EADC707047A4
:100940007BB972B90029BEBF00204FF0004106E01C
:1009500008BF00281CBF6FF000414FF0FF3000F0CF
:100960003FBAADF1080C6DE904CE002909DB002B7C
:100970001ADB00F0CDF8DDF804E0DDE9022304B075
:100980007047404261EB4101002B1BDB00F0C0F8D7
:10099000DDF804E0DDE9022304B0404261EB4101EF
:1009A000524263EB43037047524263EB430300F050
:1009B000AFF8DDF804E0DDE9022304B0404261EB6A
:1009C00041017047524263EB430300F0A1F8DDF8A8
:1009D00004E0DDE9022304B0524263EB43037047B5
:1009E00053B94AB9002908BF00281CBF4FF0FF3196
:1009F0004FF0FF3000F0F4B9ADF1080C6DE904CE12
:100A000000F086F8DDF804E0DDE9022304B0704769
:100A1000430803F05533C01A830803F0333300F062
:100A20003330184400EB101000F00F3000EB0020C2
:100A300000EB0040000E704707EE900AF5EEC07A1A
:100A4000F1EE10FA01D400F023B8F1EE677A08B5A0
:100A500017EE900A00F01CF8404261EB410108BD1E
:100A600008B502460B4643EC172BB5EEC07BF1EE02
:100A700010FA03D4BDE8084000F02AB8B1EE477B75
:100A800051EC170B00F024F8404261EB410108BD26
:100A90009FED0B6B07EE900A9FED0B5BB7EEE77ACD
:100AA00027EE066BBCEEC66BB8EE464BA4EE457B5C
:100AB000FCEEC77B16EE101A17EE900A704700BFC7
:100AC000000000000000F03D000000000000F041C8
:100AD0009FED0B6B41EC170B9FED0B5B27EE066B4D
:100AE000BCEEC66BB8EE464BA4EE457BFCEEC77B76
:100AF00016EE101A17EE900A704700BFAFF3008091
:100B0000000000000000F03D000000000000F04187
:100B10002DE9F047089D04468E46002B4DD18A42B0
:100B2000944669D9B2FA82F252B101FA02F3C2F1E3
:100B3000200120FA01F10CFA02FC41EA030E944074
:100B40004FEA1C48210CBEFBF8F61FFA8CF708FB95
:100B500016E341EA034306FB07F199420AD91CEB6D
:100B6000030306F1FF3080F01F81994240F21C819F
:100B7000023E63445B1AA4B2B3FBF8F008FB1033E7
:100B800044EA034400FB07F7A7420AD91CEB04041C
:100B900000F1FF3380F00A81A74240F207816444EC
:100BA000023840EA0640E41B00261DB1D440002371
:100BB000C5E900433146BDE8F0878B4209D9002DD5
:100BC00000F0EF800026C5E9000130463146BDE85F
:100BD000F087B3FA83F6002E4AD18B4202D38242C9
:100BE00000F2F980841A61EB030301209E46002D78
:100BF000E0D0C5E9004EDDE702B9FFDEB2FA82F2CD
:100C0000002A40F09280A1EB0C014FEA1C471FFA2A
:100C10008CFE0126200CB1FBF7F307FB131140EA11
:100C200001410EFB03F0884208D91CEB010103F1DE
:100C3000FF3802D2884200F2CB804346091AA4B2A0
:100C4000B1FBF7F007FB101144EA01440EFB00FE74
:100C5000A64508D91CEB040400F1FF3102D2A645D9
:100C600000F2BB800846A4EB0E0440EA03409CE778
:100C7000C6F12007B34022FA07FC4CEA030C20FA25
:100C800007F401FA06F31C43F9404FEA1C4900FA45
:100C900006F3B1FBF9F8200C1FFA8CFE09FB1811C2
:100CA00040EA014108FB0EF0884202FA06F20BD935
:100CB0001CEB010108F1FF3A80F08880884240F285
:100CC0008580A8F102086144091AA4B2B1FBF9F0C9
:100CD00009FB101144EA014100FB0EFE8E4508D9C4
:100CE0001CEB010100F1FF346CD28E456AD9023849
:100CF000614440EA0840A0FB0294A1EB0E01A1422E
:100D0000C846A64656D353D05DB1B3EB080261EB9B
:100D10000E0101FA07F722FA06F3F1401F43C5E975
:100D2000007100263146BDE8F087C2F12003D840AB
:100D30000CFA02FC21FA03F3914001434FEA1C47ED
:100D40001FFA8CFEB3FBF7F007FB10360B0C43EADF
:100D5000064300FB0EF69E4204FA02F408D91CEB8F
:100D6000030300F1FF382FD29E422DD9023863448D
:100D70009B1B89B2B3FBF7F607FB163341EA03412D
:100D800006FB0EF38B4208D91CEB010106F1FF387C
:100D900016D28B4214D9023E6144C91A46EA004673
:100DA00038E72E46284605E70646E3E61846F8E605
:100DB0004B45A9D2B9EB020864EB0C0E0138A3E74E
:100DC0004646EAE7204694E74046D1E7D0467BE72F
:100DD000023B614432E7304609E76444023842E7A7
:100DE000704700BF02E000F000F8FEE772B6374837
:100DF00080F30888364880F3098836483649086009
:100E000040F20000CCF200004EF63471CEF2000148
:100E10000860BFF34F8FBFF36F8F40F20000C0F246
:100E2000F0004EF68851CEF200010860BFF34F8FFC
:100E3000BFF36F8F4FF00000E1EE100A4EF63C71E9
:100E4000CEF200010860062080F31488BFF36F8F94
:100E5000E2F004FDE1F0FCFA4FF055301F491B4A67
:100E600091423CBF41F8040BFAE71D49184A9142F0
:100E70003CBF41F8040BFAE71A491B4A1B4B9A4244
:100E80003EBF51F8040B42F8040BF8E70020184964
:100E9000184A91423CBF41F8040BFAE7E2F01CFD0E
:100EA000E1F05AFB144C154DAC4203DA54F8041B24
:100EB0008847F9E701F0E4FE114C124DAC4203DA29
:100EC00054F8041B8847F9E7E2F004BD000600303F
:100ED000002200300000020808ED00E000000030B1
:100EE00000060030D8791308002200306C2A003048
:100EF000702A0030D4E30130E002020864030208E3
:100F000064030208640302082DE9F04F2DED108AF6
:100F1000C1F80CD0D0F80CD0BDEC108ABDE8F08F31
:100F2000002383F311882846A0470020E1F016F83B
:100F3000FEE7E0F06FFE00DFFEE7000070B54FF067
:100F4000FF0C4CF4E06C1CEA11541DBF1CEA135555
:100F500094EA0C0F95EA0C0F00F0DEF82C4481EABD
:100F6000030621EA4C5123EA4C5350EA013518BFDD
:100F700052EA033541F4801143F4801338D0A0FBCA
:100F800002CE4FF00005E1FB02E506F00042E0FB77
:100F900003E54FF00006E1FB03569CF0000F18BF7D
:100FA0004EF0010EA4F1FF04B6F5007F64F5407425
:100FB00004D25FEA4E0E6D4146EB060642EAC621B8
:100FC00041EA55514FEAC52040EA5E504FEACE2E25
:100FD000B4F1FD0C88BFBCF5E06F1ED8BEF1004F28
:100FE00008BF5FEA500E50F1000041EB045170BDA4
:100FF00006F0004646EA010140EA020081EA0301E8
:10100000B4EB5C04C2BFD4EB0C0541EA045170BDE3
:1010100041F480114FF0000E013C00F3AB8014F15D
:10102000360FDEBF002001F0004170BDC4F10004A6
:10103000203C35DA0C341BDC04F11404C4F1200527
:1010400000FA05F320FA04F001FA05F240EA020082
:1010500001F0004221F0004110EBD37021FA04F6B8
:1010600042EB06015EEA430E08BF20EAD37070BD72
:10107000C4F10C04C4F1200500FA04F320FA05F0D1
:1010800001FA04F240EA020001F0004110EBD370D3
:1010900041F100015EEA430E08BF20EAD37070BD43
:1010A000C4F1200500FA05F24EEA020E20FA04F31C
:1010B00001FA05F243EA020321FA04F001F00041CB
:1010C00021FA04F220EA020000EBD3705EEA430E3C
:1010D00008BF20EAD37070BD94F0000F0FD101F06B
:1010E0000046400041EB010111F4801F08BF013CA4
:1010F000F7D041EA060195F0000F18BF704703F0E2
:101100000046520043EB030313F4801F08BF013D68
:10111000F7D043EA0603704794EA0C0F0CEA135524
:1011200018BF95EA0C0F0CD050EA410618BF52EADE
:101130004306D1D181EA030101F000414FF00000E4
:1011400070BD50EA410606BF1046194652EA4306F2
:1011500019D094EA0C0F02D150EA013613D195EA66
:101160000C0F05D152EA03361CBF104619460AD1AE
:1011700081EA030101F0004141F0FE4141F47001B8
:101180004FF0000070BD41F0FE4141F4780170BDA8
:101190004FEA410212F5001215D211D56FF478739F
:1011A000B3EB625212D94FEAC12343F0004343EA42
:1011B000505311F0004F23FA02F018BF404270471D
:1011C0004FF00000704750EA013005D111F00040A7
:1011D00008BF6FF0004070474FF00000704700BF3D
:1011E0004FEA4102B2F1E04324BFB3F5001CDCF149
:1011F000FE5C0DD901F0004C4FEAC0024CEA507081
:10120000B2F1004F40EB830008BF20F001007047AF
:1012100011F0804F21D113F13872BCBF01F00040B2
:10122000704741F480114FEA5252C2F11802C2F1E4
:10123000200C10FA0CF320FA02F018BF40F0010065
:101240004FEAC1234FEAD32303FA0CFC40EA0C0017
:1012500023FA02F34FEA4303CCE77FEA625307D154
:1012600050EA01331EBF4FF0FE4040F4400070478B
:1012700001F0004040F0FE4040F40000704700BF25
:1012800001F0FF01102A2BDB10F0070F08D010F837
:10129000013B013A8B422DD010F0070F42B3F6D13B
:1012A000F0B441EA012141EA014122F007047FF054
:1012B00000070023F0E80256083C85EA010586EAAB
:1012C000010685FA47F5A3FA87F586FA47F6A5FAE7
:1012D00087F68EB9EED1F0BC01F0FF0102F00702F3
:1012E00032B110F8013B013A83EA010313B1F8D19E
:1012F0000020704701387047002D06BF354603387F
:10130000073815F0010F07D1013015F4807F02BFB7
:10131000013015F4C03F0130F0BC0138704700BF08
:1013200010F8012B11F8013B012A28BF9A42F7D08F
:10133000D01A7047034613F8012B002AFBD1181A64
:101340000138704710B5044620461CB154F80C3BD8
:10135000013300D110BD0822012100F071FB54F8C7
:101360000C0C54F8082C14F8041C121AB2FBF1F2FD
:1013700000F066FBE8E70000C26AD0E9003112F035
:10138000040F2DE9F04118BF0B46A6B00021594CBF
:10139000042601270291CDE90003D0064CBF03F1DA
:1013A000200203F168020392DA690399D2099B696A
:1013B00002F004021B880A4303F47F4303924FF0B8
:1013C000E022A3F53E41D2F8882D02F4A002B2F546
:1013D000A00F04BF012202924B424B410493464DA1
:1013E00003A82C6000F02AFA04220121434800F0EF
:1013F00027FB0422012102A800F022FB1022012178
:10140000019800F01DFB0098202201210C3000F013
:1014100017FB019804220121103000F011FB042277
:10142000012103A800F00CFB01980C2201211430CB
:1014300000F006FB0C220121009800F001FB029B4A
:10144000DA071FD5009BDB6ADB064ED415A8FEF732
:10145000A9FFDDF804C00DF1140E0CF120030CF10E
:1014600060081868083353F8041C7246434503C2E9
:101470009646F6D1DCF8603025938422012105A838
:1014800000F0DEFA00F0C0F8FFF75CFF4FF0E02359
:10149000D3F8003D03F47023B3F5402F0ED0184B62
:1014A00005A88DF81C60059314338DF828700693F9
:1014B0004FF0FF33CDE90833FFF744FF2B68A34219
:1014C00006D0104B0422012105A8059300F0B8FABC
:1014D00000F02AFA002882D0049B1BB1019A93697C
:1014E0000233936126B0BDE8F08105A8FEF754FFF2
:1014F000C3E700BFED55CEAC702A0030D0D0100845
:1015000028ED00E0ACCE55ED37B50E4D2A78202AF7
:1015100015D10D4C0D4823680D4918440192E1F096
:10152000BFFA23680021019A2033094829702360FB
:10153000E7F024FC03B0BDE83040E2F0A3B803B00C
:1015400030BD00BF642C00308C2C0030608213084A
:10155000662C003008B54720DEF09AFD144BD3F816
:10156000982042F02002C3F89820D3F8982022F067
:101570002002C3F89820D3F89820D3F8F02042F046
:101580002002C3F8F020D3F8182142F02002C3F85B
:1015900018216D22D3F81831064BDA604FF0FF3274
:1015A0001A620D221A600122034B1A7008BD00BF97
:1015B00000440258001401409C2C0030014B186874
:1015C000704700BFFCFF1F08014B0248C01A70475C
:1015D00060821308000020080048704760821308EA
:1015E00007490022074B5B1A9A4201D3012070473A
:1015F00051F8040B013001D10432F5E700207047A7
:1016000060821308000020085E4B2DE9F74F1A682E
:1016100002255D4B02F56A58DFF894911A7808F1BB
:1016200018085A4F5A4C9044DFF888A1E0F00AFAA3
:10163000A9EB070B06460EB14E2D49D9A9EB0702BF
:10164000B2EB080700F192804E2D00F28F80DFF898
:1016500068C16B1C4F4E0C21DBB2ACEB060069433A
:10166000B84273DD60184FF0010C665090463E445E
:1016700080F808C04660B2EB080213D44F2B11D09B
:10168000454E19464548AB1C351ADBB295424FF022
:101690000C0505FB01F163DD65180126024460506D
:1016A0002E726A600C2201215343E21811724FF02E
:1016B000FF31E15051603A4B1B782BB1394B1B681D
:1016C0002360394B1B686360314803B0BDE8F08F7D
:1016D000336AF06953450ABF344BF31AA3EB0A038C
:1016E00080B10193E1F0D8FB019B58B12A460C214F
:1016F00001354A430121EDB2A0180172F169A150F0
:101700000D3141600C200121984400FB05FCD845B7
:1017100004EB0C0244F80C6006F13C0C1172C2F8A8
:1017200004C005EB010205F10205D2B2EDB200FBE7
:1017300002F204EB02000172316AA15019444160C7
:1017400014D23046E0F08EF9064674E767184FF081
:10175000010E8044665087F808E0C7F804C08AE7A5
:10176000621801256050157256609BE74F2D01D815
:101770002B4697E7012384F8BC334FF0FF33C4E9CD
:10178000ED3398E78C2C0030642C00306082130815
:1017900004220030702A003000000430D8E3013009
:1017A00000220030902C0030882C003000220030C5
:1017B0000000200800060030D4E301300C4B1B78F9
:1017C00010B50BB9FFF7C6FE00230A490A48CA69DB
:1017D0009206FCD54A6A1C5CD2B2944205D1013310
:1017E000DBB20E2BF3D1002010BD0023EFE700BFCA
:1017F0009C2C003000140140D4D0100838B5084BA0
:1018000004461B780BB9FFF7A5FEE4B2054DAC62A8
:10181000EB695B0600D538BDE1F034FFF8E700BFA7
:101820009C2C00300014014010B5441E14F8010F28
:1018300000B910BDFFF7E2FFF8E7000070B50268DD
:101840000446EFF30581D9205369C9B288F03EFD03
:10185000294B1B78A3B1294B94E8030083E80300CC
:101860002748FFF7E1FF6368B3B12648FFF7DCFFC5
:101870002548FFF7D9FFFFF7A1FF2448FFF7D4FF62
:10188000234D2B783BB124681CB12046E1F004FBCA
:1018900020B900232B7070BD1E48E7E720461E4E7E
:1018A000E1F00EFB00F2145084421FD22046E1F01A
:1018B00007FB30602046194EE1F016FB04F5E053BB
:1018C000834217D92046E1F00FFB30600023144A11
:1018D0001360144A1370FFF783FE0028D9D0E1F09B
:1018E000D1FE0120BDE87040E1F062B9A4F21453CA
:1018F0003360DFE73360E9E7652C0030942C00307B
:10190000E4D01008E9D01008FAD0100838A911085E
:1019100000220030F4D01008902C0030882C0030C9
:101920008C2C0030642C0030284B1A7870B542B1F2
:101930002748FFF779FF274B5868003818BF012068
:1019400070BD254A107800283CD0244E244C3368C2
:101950002448254D1A1D21782D1A0A44AA4205D380
:10196000224A4FF0FF31D161202222702278D2B179
:1019700003F120018D4205D81F2A9FBF1B4AD36166
:1019800020222270202219491844E1F089F8326897
:101990002378002115481344202221703360E7F09A
:1019A000EDF9E1F06FFE33689D4207D90F4920221F
:1019B0000F48CB61E1F074F8E1F064FE0020E1F043
:1019C000F7F8B8E701221A70BAE700BF652C0030BB
:1019D00040D11008942C0030002200308C2C0030B4
:1019E000642C00306082130800002008662C003050
:1019F000E0FF1F082DE9F84307460E460024DFF8F4
:101A00003890DFF83880B44201D1BDE8F88324B1C2
:101A1000230702D14846FFF707FF3D5D01342B093C
:101A200005F00F0518F80300FFF7E8FE18F80500A9
:101A3000FFF7E4FEE7E700BF38A9110850D110080E
:101A4000474B1B782DE9F74F07460E4690465BB192
:101A5000022925D0042938D0012902D11146FFF7E7
:101A6000C9FF4048FFF7E0FE3F4B1B78002B4ED0EC
:101A70003E4A00253E4BA2EB030938E037F814300C
:101A8000ADF8043024B1620702D12846FFF7CCFE3E
:101A90000134022101A8FFF7ADFFA045EED1E0E738
:101AA0000024304DF9E757F82430019324B1A307FF
:101AB00002D12846FFF7B8FE042101340DEB0100E6
:101AC000FFF798FFA045EED1CBE70024254DF9E7BD
:101AD000FFF71AFD022E1DD0042E2CD0012E06D1A8
:101AE0002378795D5A1C2270224AD1540135A845C9
:101AF0000DD0214B214C1B682278043313444B45F5
:101B0000E6D31C4B4FF0FF32DA612023237003B081
:101B1000BDE8F08F2378DFF85CA05A1C22703A7879
:101B20000AF80320FFF7F0FC23785A1C22700022E9
:101B30000AF80320DAE74FF0000ADFF838B022781D
:101B40003B78511C23FA0AF30AF1080A21700BF8BA
:101B50000230FFF7D9FCBAF1200FF0D1C6E700BF81
:101B6000652C003038A91108002200300000200840
:101B700060821308662C00308C2C0030642C0030FE
:101B8000036800221B6818470120704737B5019190
:101B90002021044681F0DAFCE0B10F4B93F9921951
:101BA000B1B1B3F9941903F58053019AD3F83433E2
:101BB000B3F90C5001F10A039D4203DD40F28D336D
:101BC000994205DC2046054B202181F0C5FC002010
:101BD00003B030BD0120FBE7A06C003064D11008D9
:101BE00008B506F045F80121BDE8084005F0B4B895
:101BF0002DE9F04300278FB00E46054606F038F871
:101C000080462E22394602A80197E7F0B7F8322322
:101C100001AA3946404605F06DFA044648B901ABC1
:101C2000174A3146284681F017FF20460FB0BDE81D
:101C3000F083DFF85890D9F8600003689B689847F4
:101C40000028F2D0A9F5C04003F05EFE814630B90D
:101C50000C4A314628464C4681F0FEFEE5E76946CF
:101C6000404605F06BF80028DFD09DF801305B0698
:101C7000DBD5054A314628463C4681F0EDFED4E7E7
:101C800078D1100881D1100898D11008A08C0030AC
:101C900008B5064B93F8A9359B0704D5044A81F093
:101CA000DBFE002008BD0120FCE700BFA07C003067
:101CB000A8D1100870B50C4C05460E46206E03687E
:101CC000DB68984710B10124204670BDA4F5C040E0
:101CD00003F038FE04460028F5D1044A3146284670
:101CE00081F0BAFEF0E700BFA08C0030B8D1100838
:101CF000284B2DE97043D3F8AC35814688461D7BCF
:101D00005DB9254B1B68986A03685B6B984738B9C7
:101D1000224A4146484681F09FFE2846BDE870832E
:101D200060F0BEFE202162F053F938B160F0B8FED9
:101D30001F2162F04DF908B1194AEAE7484681F0DF
:101D4000FDFB38B9D9F80030414648469B6BBDE8E9
:101D50007043184741464846FFF718FF064641467C
:101D6000484682F0E7FC064020214846F5B281F063
:101D7000EDFB41464846FFF78BFF0540414648468C
:101D8000FFF798FF05404146484682F05BFF05405B
:101D9000C3E700BFA07C0030088E0030CCD1100813
:101DA000E3D1100808B5FFF7A3FF054A92F898158C
:101DB00060F3410182F89815024A907108BD00BF96
:101DC000A07C00308D8F00302DE9F04106460F4693
:101DD00081F0F2FB044678B30221304681F0B6FB75
:101DE00050B305F045FF4FF48071804604F0B4FF16
:101DF000054608BB4FF40071404604F0ADFFD8B172
:101E00000F4886F0DFFA0F4B03F67C33D3ED007AF0
:101E1000F8EEE77A30EE670ADFED0B7AB0EEC00A33
:101E2000B4EEE70AF1EE10FA06DD2C46074B3A460F
:101E30000221304681F090FB2046BDE8F08100BFD2
:101E400014890030A07C00300000C84200D2100885
:101E5000F8B504460F4681F0C1FF10210546204623
:101E600081F074FB58B12046FFF7BAFE064630B940
:101E70003546044B3A461021204681F06DFB28463A
:101E8000F8BD00BF14D2100870B505460E4681F0AB
:101E90006DFD044678B18021284681F057FB50B192
:101EA000094B93F8793B43B10024084B324680211B
:101EB000284681F051FB204670BD31462846BDE8DA
:101EC000704082F06DB900BFA07C003028D21008AD
:101ED0002DE9F04180460E461A4FFFF789FE044671
:101EE00010B90024FC7109E0174D05F5C043186EC8
:101EF00003689B68984720B90123FB712046BDE821
:101F0000F0810821404681F021FB0028F4D095F8AB
:101F10003436B02202FB035305F58045B3F83E2466
:101F2000B5F990399A4206DD084B32460821404601
:101F300081F012FBD5E73146404681F045FC002890
:101F4000DAD1CEE78D8F0030A02C00303CD21008C3
:101F500082F024BA70B505460E46FFF749FE084BDD
:101F600004463146D8712846FFF7A4FE00283146C2
:101F7000284608BF002482F0C5FD204070BD00BF88
:101F80008D8F00302DE9F843404F81463B78002B80
:101F90007AD13F4C0126D4F8AC553E702D7B1DB153
:101FA0003B702846BDE8F88382F036FF054630B91D
:101FB000384A3870137843F001031370F1E7DFF803
:101FC000F08052F0A1FC314651F05EFC88F80460CC
:101FD0000B26013E49F058F949F074F816F0FF0657
:101FE000F7D12D49484682F0DFFD05F041FED0F8DB
:101FF0000C22C4F8BC2590F89432DA0732D405F0EC
:10200000E7F852F081FC3C2152F00EFA04F2A4539E
:1020100000221A60214B01211B68D86A03681B68E3
:102020009847D4F8AC25137B1BB90123137388F8A8
:10203000043052F069FC94F89D2594F89C1551F0F9
:1020400017FE4EF04DFF4EF07DFA00233B7088F0F6
:10205000ABF9134B586594F8993543F0200384F895
:1020600099359EE79B07D5D431460E4802F0F2FA27
:102070000D4886F0A7F9DFED0D7A04F2A45320EEA7
:10208000270A83ED000AC5E700258AE79D2C00306A
:10209000A07C0030AC8F00304CD21008088E00308D
:1020A000A08C0030A02C0030148900300AD7233CCB
:1020B0008D8F00302DE9F043354D87B006460C4634
:1020C000D5F8AC351B7B002B60D000294BD02146C6
:1020D000304682F067FF0446002852D02D49304632
:1020E00082F062FD05F0C4FD07460BF01BF8804648
:1020F000384604F069FAD8B198F92830022B17D184
:1021000000264FF00009F1B203AA3846CDF80C9032
:102110000191CDF81090CDF8149004F087FE01994C
:1021200018B103AA40460AF009FD0136032EEAD190
:10213000D5F8AC25137B1BB100231373164A13711A
:1021400052F0E2FB002151F09FFB144B00211B6871
:10215000D86A03681B68984795F899356FF345135B
:1021600085F899350EE005F580530192186E0368E5
:10217000DB689847019A0028A9D195F89835DB06C5
:10218000A5D40024204607B0BDE8F0830124F9E778
:10219000A07C00305CD210088D8F0030088E00309B
:1021A00000F5A04008B590F89835C3F380028A4244
:1021B0000BD061F3820380F8983531B152F0A4FB63
:1021C0000F21BDE8084052F02FB908BD00F5A0422C
:1021D00010B592F8A9350C4603F00101A14209D0CF
:1021E00064F3000382F8A935DB0704D402F082FC13
:1021F000024B9C7210BD02F02FFDF9E78D8F00306D
:1022000000F5A04090F8A93561F3410380F8A935A5
:10221000014B1973704700BF8D8F0030002070474D
:102220000020704700207047002070470020704752
:102230000020704700207047002070470020704742
:102240000020704700207047002070477047000052
:102250007047000000207047002070470020704742
:102260000020704700207047002070470020704712
:102270000020704700207047704700000020704722
:1022800000207047002070470020704700207047F2
:1022900000207047002070470020704700207047E2
:1022A00000207047002070470020704700207047D2
:1022B00000207047704700007047000000F5934011
:1022C00020307047004870476C03110800F5A040AB
:1022D00090F89C0570470000034808601C211170AD
:1022E00008221A60704700BF34D610084EF044BD73
:1022F0001FF0C2B951F04ABC5FF0AEBF5DF056BCF2
:1023000002F018BC02F04CBB02F072BA48F0DABE20
:1023100066F008BE60F076BA14F086B902F086B9AD
:1023200002F04CBE02F004BB02F09CBD03F014B9F5
:102330001FF03EBF03F01CBB02F030BC02F0E8BC53
:10234000694B70B5044640F8043B65F011F8002570
:1023500004F1100004F5924609F032FA04F1B000DD
:1023600082F08EFE04F51C704EF094FA04F54A706B
:1023700012F0FEFA04F5EE6007F0E8FD04F618101E
:102380000AF02AF804F546601EF0C8FE04F5BF50B6
:102390002836103064F062FF04F5C6504DF05CFE44
:1023A00004F5DF50083051F0AFF904F5E7501C3068
:1023B0006DF04AF804F5E850183063F031FA04F58E
:1023C000EA50143078F012FC04F50F5024307FF0FE
:1023D00069FE04F510504EF017FE04F51450143049
:1023E00066F0B2F904F5005304F515503F4A83F83E
:1023F000585504F5155328301833136048F04AFC3B
:1024000004F516502946383003F0B2FD04F5325079
:1024100068F0C2FF04F53250303075F06BFE04F501
:102420005A503C3076F086FB04F571507CF094FEF7
:1024300004F5755018307EF08FFF04F576503C306F
:102440007FF0C4FB04F57850143074F01FFA04F5E3
:102450007A503C3007F0AEFB04F58040203076F037
:10246000C5FC04F58140203080F0B8FF04F58740BA
:102470001F4974304CF084FC04F588400C306DF03A
:102480002BFC04F58A40203080F07CFE04F58A4065
:10249000783087F095FF04F58E402C3062F0E2FC36
:1024A00004F5804383F8945704F58F452835284672
:1024B0000C3554F0A9FCAE42F9D104F592400D4D13
:1024C000343080F0DFFE04F59240583054F006FBC3
:1024D0002B6813B1084887F037FF204607494CF0B6
:1024E0004FFC20462C6070BDFCB71108649C003086
:1024F000B83C120890900030B4D21008A4B611086D
:1025000010B503F003F960F0CBFA0368BDE81040A2
:102510005B681847FFF7F4BF38B500F5AB450446D4
:102520004035284609F016F80AF0FCFD90F92530F0
:10253000D3B190F84433BBB12846002108F06EFDBA
:10254000DFED0A7A04F6743304F6181020EE270A39
:10255000DFED077A93ED287AA7EE270A83ED280AA4
:10256000BDE838400AF0ECBC38BD00BFCDCCCC3D56
:102570006666663FFFF7D0BF10B50121044603F041
:1025800019FA10B1204601F0E7F94FF480512046C6
:1025900003F010FA20B12046BDE8104001F09EB9CA
:1025A00010BD0000FFF7E8BF38B50221044603F074
:1025B00001FA38B10121204603F0FCF910B9204698
:1025C00001F0CAF90221204603F0F4F958B320467D
:1025D00001F0D0F94021204603F0ECF968B104F590
:1025E000DF550835284650F057FB04F5805393F922
:1025F000183D13B1284650F01BFD4FF48061204672
:1026000003F0D8F920B104F5DF50083050F0E6FBB4
:102610008021204603F0CEF960B120F027FFBDE80D
:1026200038401EF075BB0121204603F0C3F9002895
:10263000CDD1CFE74FF48021204603F0BBF900282D
:10264000EBD14FF40021204603F0B4F90028E4D187
:1026500038BD0000FFF7A8BF10B50121044603F004
:10266000A9F910B1204601F085F98021204603F038
:10267000A1F928B120F0FAFEBDE810401EF024BBFD
:1026800010BD0000FFF7E8BF38B504464FF6FF71F4
:1026900003F090F904F5A04528B1D5F89825072155
:1026A000204601F06FF962F07BFA61F04FFF95F878
:1026B0009835074A83F01003C3F3001353714EF0AB
:1026C0000FFC4EF061F80348BDE8384073F058BB8A
:1026D0008D8F0030008C0030FFF7D6BF2DE9F04F12
:1026E00000F516540546012138342DED028B2046A5
:1026F000A1B005F02FFA05F5B74120461C3105F0D1
:1027000097F805F5B7412046343104F083F804F515
:102710004B7005F5245105F5A044083104F53C6BD8
:1027200004F69C3604F53A6826F0AEFB05F5B74092
:102730008BED000A1EA932684830D8F8003004F644
:10274000A8371E9204F6AC391F9355F041F805F5F1
:10275000B74105F5B840B0EE608A04F53B6AF0EE8B
:10276000408A24310C3054F0C7FE05F5B74105F519
:10277000B840C7ED008A403189ED008A40308AEDCB
:10278000000A54F0B9FE04F6C43383ED000A1B932B
:1027900052F0BAF8054687F00FFE2F4A1B9B92EDC8
:1027A000007A04F6BC32B7EEC77A8DED187B92ED55
:1027B000007A04F6B832B7EEC77A8DED167B92ED4B
:1027C000007A04F6B43204F6A434B7EEC77A8DED7D
:1027D000147B92ED007A214AB7EEC77A8DED127B19
:1027E00093ED007A1E4BB7EEC77A8DED107B9BED13
:1027F000007AB7EEC77A8DED0E7B9AED007AB7EED0
:10280000C77A8DED0C7B94ED007AB7EEC77A8DED2B
:102810000A7B99ED007AB7EEC77A8DED087B98EDCB
:10282000007AB7EEC77A8DED067B97ED007AB7EEAA
:10283000C77A8DED047B96ED007AB7EEC77ACDE9C5
:102840000001084928468DED027B51F07DFC21B046
:10285000BDEC028BBDE8F08F70540030D6D210086A
:10286000C8D2100803D31008FFF738BF10B50446CC
:1028700002F0D2FF1021204603F09CF850B120F066
:10288000F5FD1EF01DFB04F5EA50BDE810401430C4
:1028900077F0E0BB10BD0000FFF7E8BF00F5165071
:1028A000D1ED017A91ED006AD0EDA85AD0EDAB6A76
:1028B00026EEE77A67EEA57AA6EE257AE6EE267A88
:1028C00081ED007AC1ED017A7047000000F51650E5
:1028D000D1ED017A91ED006AD0EDA85AD0EDAB6A46
:1028E00027EEA67A67EEA57AA6EE257AE6EE667A58
:1028F00081ED007AC1ED017A704700002DE9F041C9
:1029000004464FF001082DED028B86B004F5A0457A
:10291000FFF716FDC04B04F5934004F5A64623606F
:1029200004AF5430483601F04FFD04F59343304670
:102930001833C5F83C33062385F8403380F06AFD30
:10294000B64B301D04F5A7463946C5F84833443622
:102950008DF810804DF030FAB14B06F10C00C5F83F
:10296000C43386F05BFE1E234FF4E16085F82885B2
:10297000C5F830350023A5F8343509F0E1FCC5F879
:102980002C0504F5AA40383086F048FE04F5AA402C
:102990007C3086F043FEA34B1A6802B91E60A24940
:1029A00030464CF0EDF9A14B04F5AB40F7EE008A50
:1029B000C5F8C43301231E309FED9D8AA5F89C35D0
:1029C000142682F043FB9B4B04F5AB404FF400719F
:1029D0000593994B40300494009397E80C0008F05D
:1029E00059F903A904F5B740CDED038A54F0C6FAAE
:1029F00004F5B7400C3009F03FF805F69C33B0EE13
:102A0000083A9FED8E2A83ED008A04F5B94083EDE4
:102A1000018AF0EE420A83ED028A05F6A833F0EE51
:102A2000432A103083ED008AB0EE430A83ED018A19
:102A3000F0EE481A83ED028A05F6B433B0EE481A78
:102A400083ED008A83ED018A83ED028A05F6EC337B
:102A500083ED008A83ED018A05F6F43383ED008A65
:102A600083ED018A05F6FC3383ED008A83ED018A4C
:102A700005F6044383ED008A83ED018A05F674436D
:102A800083ED008A83ED018A83ED028A04F5B94360
:102A900083ED008A83ED018A83ED028A04F51653E3
:102AA0003833C5F88C3C73F0A3FBB0EE083A04F55C
:102AB000BA40B0EE682AF0EE481A614DF0EE432AB3
:102AC0004430B0EE481AF7EE080AB1EE0C0A73F083
:102AD0003DFDB0EE083A04F5BB40F0EE481AB0EE0A
:102AE000481A9FED562AF0EE432ADFED560AB0EE63
:102AF000430A3C3073F02AFDB0EE083A04F5BC40BE
:102B0000F0EE481AB0EE481A9FED4F2AF0EE432A35
:102B1000DFED4E0AB0EE680A343073F069FBB0EEB8
:102B2000083A04F5BD40B0EE482AF0EE481A9FED91
:102B3000480AF0EE432A6830B0EE481AF0EE480A30
:102B400073F004FDF0EE083A04F5BE40B0EE485ACA
:102B5000F0EE684A9FED3F0AB0EE484A6030B0EEB2
:102B6000633AF0EE632AB0EE002AF0EE481AB0EEB7
:102B7000481AF6EE000A73F0B3F8374B04F5C0427A
:102B80001D6000235C3298B2013306FB0051097CC2
:102B90000029F8D1314B1880314B1880314B19681E
:102BA00011B1314887F0D0FB04F5C04004F5C045B1
:102BB0001A606430286602F0B9F92C4B04F5C14064
:102BC0006B66143002F0B2F9294B04F5C140C5F828
:102BD0009430443002F0AAF9264B04F5C140C5F800
:102BE000C430743002F0A2F9234B04F5C24085EDE5
:102BF000498AC5F8F43085ED4A8A343085ED4B8A30
:102C000002F094F91D4B2046C5F8343106B0BDECF6
:102C1000028BBDE8F08100BF70D8100878D2100890
:102C2000A0DD11080C9500302CD9110898D9100896
:102C3000000000003D23020864D81008CDCC4C3EB3
:102C400078161108CDCCCC3ECDCCCC3DCDCC4C3D76
:102C50003333333F9A99993F54900030509000306D
:102C600020900030EC8F003008D31008C41F1108EA
:102C70000C1F110878201108641F11081420110876
:102C800038B5054B0A4601461C68236820461D6876
:102C9000024BA847002038BD088E0030A02C003021
:102CA00038B5037904463BB905682DB128461DF0B7
:102CB0009DF9284609F046FB204638BD384B70B5D3
:102CC0000360044600F58740143008F0B7FE04F5B1
:102CD000405393F8B02D42B9D3F8AC5D2DB12846DE
:102CE0001DF084F9284609F02DFB04F50F5004F57A
:102CF000C35504F5C056243014357FF0E7F904F5C8
:102D0000FB5014360830FFF7CBFF04F5FB50FFF7FC
:102D1000C7FF04F5FA501830FFF7C2FF04F5E8507A
:102D2000183062F095FDB54204D0183D28461CF0DD
:102D30004FFDF8E704F5945504F59256194B0C3500
:102D40000436C4F8603CB54204D0083D2846FFF77D
:102D5000A7FFF8E704F6B47504F6A846B5420ED00E
:102D6000A5F5827505F1780055F038F805F14C00AD
:102D700055F034F805F1200055F030F8EEE70A4B35
:102D8000C4F8FC3094F80C3243B9D4F808522DB191
:102D900028461DF02BF9284609F0D4FA204670BDCC
:102DA000FCB71108CC8111081C6B1208094B0A4AA8
:102DB00010B5036000F5A0430446D3F82C05C3F812
:102DC000C42308B109F0C2FA2046FFF777FF204676
:102DD00010BD00BF70D81008A0DD110810B586F036
:102DE000FBFE064C064B18602046FFF787FD204689
:102DF000044A0549BDE81040E2F03CB9A02C00307F
:102E0000088E0030B43C0130AD2D020810B50446E8
:102E1000018002494BF0B4FF204610BD60D9100874
:102E200000234FF07C524FF07E5110B5264C0365C5
:102E3000C0F88030C0F89030C0F8A030C0F8C03082
:102E40004365C0F88430C0F89430C0F8A430C0F8AE
:102E5000C43083668367C0F89830C0F8A830C0F8E3
:102E6000B830C366C367C0F89C30C0F8AC30C0F857
:102E7000BC304FF03F430267C0F8B0204267C0F853
:102E8000B420C0F88820C0F8C820C0F88C200166A3
:102E900044668465C1654FF47A71C0F8CC30212056
:102EA00061F0C6FA4FF47A71222061F0C1FA4FF452
:102EB0007A71232061F0BCFA4FF47A712420BDE8C6
:102EC000104061F0B5BA00BF000080BF70B52DEDB5
:102ED000068B037B82B004469FED8A8A3BB980ED66
:102EE000358A80ED368A80ED388A80ED378AD4EDD8
:102EF000371A04F1100594ED381AB7EE009AD4EDA4
:102F0000360A212694ED350A7F4800F07BFCB7EEA7
:102F1000001AFFEE000A582094ED350A21F0B6FFA2
:102F2000B7EE001AFFEE000A592084ED350A94ED41
:102F3000360A21F0ABFFB7EE001AFFEE000A5A2066
:102F400084ED360A94ED380A21F0A0FFB7EE001A9E
:102F5000FFEE000A5B2084ED380A94ED370A21F079
:102F600095FF84ED370A87F015FA07EE900A9FED7A
:102F7000677A2946F8EE677ADFED659A67EE877A19
:102F8000C4ED027AD4ED353A94ED384AD4ED367A70
:102F900095ED105AD5ED145A95ED186A23EE855A21
:102FA00067EEA55AD4ED374A24EE066AD5ED1C6AC1
:102FB00088FE055AB5EEC05AC8FE255A64EEA66AC8
:102FC000B0EEC66A35EE257AF0EEE66AF1EE10FA5A
:102FD00037EE067AF5EEC05ACCBF0123002337EE58
:102FE000267AF1EE10FAB5EEC06AA5EC017A95EDFD
:102FF000233A85ED079A67EE837A95ED1F3AE3EE63
:10300000837AD5ED273AE4EE237A95ED2B4AE4EE68
:10301000847AC5ED037A84F8D030C2BF94F8D030FA
:10302000013384F8D030F1EE10FAF5EEC06AC2BF79
:1030300094F8D030013384F8D030F1EE10FAC2BFEA
:1030400094F8D030013384F8D03094F9D030002B8C
:10305000C1BF06EE903AF8EEE66A87EEA66A85ED05
:10306000036AD5ED038AF0EEE87A37EE277AB4EEFC
:10307000C97AF1EE10FAC4BF39EE677A05ED017A2C
:1030800094F9E83015ED01AA73B1B4EEE9AAF1EEB6
:1030900010FA09D89FED1F7AF4EEC77AF1EE10FA14
:1030A000A4BF4FF08043EB6194ED390AD5ED077A68
:1030B000019120EE270AD4ED027A20EE270ADFEDF7
:1030C000167A30EE000A20EE270AE1F0D9FFEAEE88
:1030D000008A30B201369FED110AB6B228EE800A9E
:1030E000C5ED0B8A61F080F9252E01997FF44AAF76
:1030F00004F12002044802B0BDEC068BBDE870402C
:1031000000F0B2BB00000000A02C0030BD378635B7
:103110009A99193FCDCCCC3EDB0F494000007A4450
:103120000022C0F8D420C0F8D820C0F8E020C0F8B1
:10313000DC20FFF7CBBE0000002070470020704766
:103140000120704790F830308B4286BF00EB810041
:10315000406B00207047000090F830308B4286BFF3
:1031600000EB8100406B002070470000FA207047A0
:10317000D0E9093242F4E05243F4F8438262C26A71
:10318000436242F4E052C26270470000014802F01C
:103190002BBC00BFA02C003013B54FF45E70019122
:1031A00009F0C8F8044620B101995DF0FDFF024B1B
:1031B0002360204602B010BDE0D91008704700001F
:1031C00070470000002070477047000000207047E3
:1031D0000020704700207047002070470020704793
:1031E00070470000704700000320704708207047B8
:1031F000064BD3F8AC353BB11B7B002B0CBF5020EA
:10320000D02040F0010070475020FAE7A07C003049
:103210007047000070470000114BD3F8AC05F0B1C7
:10322000D0ED387A90ED367AF0EEE77AD0ED376A65
:10323000B0EEC77AF0EEE66AC7FE877A90ED357A8F
:10324000B0EEC77A87FE267AC7FE877A9FED057AA9
:1032500067EE877AFDEEE77A17EE903A18B270477C
:10326000A07C00300000C84257F04ABC10B50446AC
:1032700059F062F8054802F0B7FB054A03460621FB
:103280002046BDE8104059F03FB800BFA02C0030E8
:10329000CCD9100857F032BF084608B508F00EFD2B
:1032A00000280CBF0420002008BD0000162A01D011
:1032B00057F05CBC032201200A7070475DF06CBCC3
:1032C00008B557F0B5FE40F41C6040F00D0008BD95
:1032D00010B5044609F036F8204610BD08B5094B74
:1032E00093F89825D2060AD403F58053186E036824
:1032F000DB6A984700280CBF0220042008BD01208B
:10330000FCE700BFA07C0030044B187820B9044BC8
:1033100093F89905C0F38010704700BF608E0030AD
:10332000A07C003000B5002389B00293039304937E
:1033300004F09EFC02A904F057FAA0B104F098FC36
:1033400000F5607005AB07C883E80700184626F053
:103350003DF9F1EE047A20EE270AFCEEC07ACDEDBD
:10336000017A9DF8040009B05DF804FB7FB50023E5
:1033700003930493059304F07BFC03A904F034FA4F
:10338000D8B104F075FCD0EDE00A90EDE10AF1EE61
:10339000600AB1EE400AE2F04BFEDFED097A20EE62
:1033A000270A21F0CFFCF6EE007A20EE270AFCEE89
:1033B000C07ACDED017A9DF8040007B05DF804FBFA
:1033C000E02E65421FB5002301930293039304F09E
:1033D0004FFC01A904F008FA28B101A826F0F6F87C
:1033E00005B05DF804FB13F05DF9B02290F80C33E2
:1033F00002FB030090ED410AF2E700000B4B93F84B
:10340000792B7AB993F8A92551070BD193F8982510
:10341000D20609D493F8993513F0020F14BF042093
:10342000012070470520704703207047A07C0030C2
:103430002DE9F04F394D8FB0044695F89C25012AAF
:103440005BD9A5F5805705F54D68354E4FF0080955
:1034500005F5805516F901BBB7F9AC390BF1FF3A08
:1034600043FA0AF3D90743D594F8280055F036FDFE
:10347000039094F8280056F029FD039A00F12103E7
:103480009A4206D294F828000FB0BDE8F04F57F0EA
:10349000E7B9BAF1070F2BD8DFE80AF03E0432345F
:1034A00036383A3C1F4B5A69D8681969D3F804E09A
:1034B000D3F818C0D3F800A00A925A6A1B6ACDF854
:1034C0002D206222CDF83130212308900991C221AC
:1034D00094F82800CDF814A0CDF818E0CDF81CC061
:1034E0008DF82CB0CDE90032192305AA55F074FDF2
:1034F00009F1FF3313F0FF09ACD10FB0BDE8F08F35
:10350000094BD0E7094BCEE7094BCCE7094BCAE79B
:10351000094BC8E72B46C6E74346C4E7A07C00300A
:10352000C0DA10089C890030148A00308C8A003080
:10353000148B0030408B0030B88B0030094BD3F82F
:10354000D829920701D457F005BB03F58053DFED6E
:10355000067A03F5396393ED000AB8EEC00A20EE4F
:10356000270A7047A06C00300AD7233C10B594B0EE
:10357000044603A808F080FA1A4B03A9186E0368E2
:103580005B6B984758B394F8284086F00DFF059B75
:103590009622DDED047A57210893069BF8EEE77A30
:1035A0009FED117A0993002367EE877A07900B93BA
:1035B00020460C930D930E930F9310931193129337
:1035C0004FF6F853CDED0A7AADF84C3000238DF864
:1035D0004E303323CDE9003207AA55F0FDFC14B07C
:1035E00010BD00BFA08C00300AD7233CF0B5254D9C
:1035F00095B00E46074603AC0FCD0FC42B68236071
:10360000731EDBB2042B2AD814AA02EB830353F8EF
:10361000445C2B6828461B6A98472B68044628465A
:103620009B6A98470023052297F828500890099331
:103630008DF828208DF829608DF82A3094B923223E
:1036400021460DF12B00E5F099FB86222E2340F256
:10365000B3112846CDE9003208AA55F0BDFC05207B
:1036600015B0F0BD20460DF12B0304F1200250F8F7
:10367000041B904243F8041BF9D102881A80827817
:103680009A70E2E7ECCE1008014802F0ABB900BF37
:10369000A02C0030014B93F89C057047A07C0030B3
:1036A000024B93F89905C0F340007047A07C0030AE
:1036B000154B30B505460C462DED028B186E85B0C6
:1036C00091ED018A0368DB69984728B9BDEEC88A85
:1036D00018EE103ADB0712D5D4E9040121F0BAFE46
:1036E00068B1684608F0C8F96A46214628465CF089
:1036F00055FB20B10549684608F0ECFA00B10220FC
:1037000005B0BDEC028B30BDA08C00302C880030A1
:103710008B8B162B05D0C02B01D1FFF7C9BF5EF0F4
:1037200029BA00207047000030B5002305462DED72
:10373000028B8DB003930493059304F099FA03A9C7
:1037400004F052F860B304F093FA00F5607306AC2D
:1037500095F8285093E8070084E80700DDED060A95
:103760009DED070AF1EE600AB1EE400AE2F060FC5E
:103770002046B0EE408A25F029FF089B0122DFEDAC
:103780000A7AA8210B930C2328EE278A28468DED70
:103790000A0ACDE9003209AA8DED098A55F01CFC10
:1037A0000DB0BDEC028B30BDE02E6542242938B54A
:1037B000054605D040290DD0BDE838405CF068BE14
:1037C0000C2157F05FF8044610B12846FFF7ACFF14
:1037D000204638BD0124FBE7F6EE007A08B591EDEE
:1037E000007AB4EEE77AF1EE10FA06DD0122052147
:1037F0000348FEF75FFC002008BD0420FCE700BF83
:10380000E87F00302DE9F04188B080461B2200217E
:1038100001A810EE107A10EE906A11EE105A11EE17
:10382000904AE5F0ABFAA3238DF8043095238DF888
:1038300005300B238DF8063086F0BEFDCDF807006D
:1038400008F5DF50CDF80B101B2201A90830CDF888
:103850000F70CDF81360CDF81750CDF81B4050F025
:103860002FF808B0BDE8F08170B58CB00D46144655
:1038700006462B22002101A8E5F080FAA3238DF84B
:10388000043095238DF805300C238DF8063086F032
:1038900093FD2B682B22CDF8070006F5DF50CDF8FD
:1038A0000F3023680830CDF80B1001A9CDF8133084
:1038B0006B68CDF817306368CDF81B30AB68CDF876
:1038C0001F30A368CDF82330EB68CDF82730E368CC
:1038D000CDF82B304FF0F4FF0CB070BD70B500F593
:1038E000DF5400F5B94605460E21083406F15002B2
:1038F00020464FF099FE06F17C0220460F214FF042
:1039000093FE05F5BA4220461021743205F5BC46F7
:103910004FF08AFE05F5BB42204611216C324FF074
:1039200083FE06F1740220466C214FF07DFE06F105
:10393000A00220466D214FF077FE05F5BE422046DD
:103940000D2118324FF070FE05F5C0422046692166
:10395000BDE870404FF068BE1FB500F5165000235B
:1039600001A9383001930293039302F0FFF905B0E7
:103970005DF804FB08B504F07BF9BDE8084003F0EE
:1039800005BE00007FB50E464FF6FF710446154692
:1039900002F010F8E8B1102200216846E5F0EEF9D7
:1039A000A3238DF8003095238DF8013004238DF882
:1039B000023086F001FDCDF8030004F5DF50CDF8AC
:1039C00007101022694608308DF80B6003954FF000
:1039D000F7FF04B070BD0000B220704738B500F5A5
:1039E000DF55044602F000F80C4908350246284627
:1039F00050F002F904F5A043284693F89D2593F86A
:103A00009C1550F035F904F51650383004F0E8FAFA
:103A100004F54A70BDE8384011F05EBDCCD91008FD
:103A200037B5069D044600B92C7801B9697802B90A
:103A3000AA7803B9EB78002064F3070061F30F2044
:103A400062F3174063F31F6003B030BD2DE9F04F00
:103A5000DC4CF7EE006ADFEDDC5A924605460E4676
:103A6000DFF894832DED0C8B9DB00D93D4EDB99AB6
:103A700004F5A04490ED006AD4F8AC35D3ED367A65
:103A800093ED387AF0EEE77AB0EEC77A77EE877A80
:103A9000F4EEE67AF1EE10FAC8BF86EEA78ADFED03
:103AA000CB7AD8BFB0EE668A28EE277AA6EE257AC2
:103AB00080ED007AD4F8AC3593ED357A93ED376A22
:103AC000B0EEC77AB0EEC66A37EE067AB4EEE67AA2
:103AD000F1EE10FAC8BFC6EE878A90ED017AD8BF22
:103AE000F7EE008A68EEA77AE7EE257AC0ED017A54
:103AF00050F00AFF074686F05FFCB7EEE87AB7EEB3
:103B0000C88AB34BB34A8DED087B95ED017AB7EEC9
:103B1000C77ACDE900018DED047B95ED007A38463A
:103B2000AD49B7EEC77AAD4F8DED068B8DED027BBB
:103B300050F00AFBAA49304697ED00AA25F012F989
:103B40008DED160A9AED000ACDED170A30EE4A0AFD
:103B50008DED181A21F06EF99DED167A08F6CC134A
:103B6000B0EEC77AD3ED007AA7F5FA63B4EEE77A40
:103B70000B93F1EE10FA00F12982D4F8AC351B7BDF
:103B8000002B00F02382B8F8CA99C9F340099DEDD3
:103B9000177AB0EEC77AF4EEC77AF1EE10FA00F3B6
:103BA0001882D4F8AC351B7B002B00F01282B8F8D9
:103BB000CA3903F001039DED187A0A93B0EEC77A73
:103BC000F4EEC77AF1EE10FA00F30582D4F8AC35C2
:103BD0001B7B002B00F0FF81B8F8CA39C3F38007C4
:103BE000B0EEC00AF4EEC07AF1EE10FA00F3F581FF
:103BF000D4F8AC351B7B002B00F0EF81B8F8CA3944
:103C0000C3F3C00B0DAB3A460A99484600935B4696
:103C1000FFF706FF9FED738AC3B20F900BEE103AC9
:103C2000C0F307230AEE903AC0F307430CEE903A34
:103C3000030E0DEE103A9DF83430002B40F0D08189
:103C40009DF83530002B40F0CB81F8EE4B7A644A7A
:103C5000B0EE690A19AB314602F52070CDED197A44
:103C6000F8EE6A7ACDED1A7AF8EE6C7ACDED1B7A21
:103C700072F04AFCB0EE409A8DED140AF0EE608AC4
:103C8000CDED150A9DF83630574C002B40F0AD8134
:103C900004F6BC33B0EE691A1CEE901A96ED020AD7
:103CA000D3ED000A04F6E86072F04CFDB0EE40CAB5
:103CB0009DF83730002B40F09B819AED000A30EEE2
:103CC0004A0A21F0B7F8F0EE690A1DEE101A4748CB
:103CD00072F04EFAF0EE40BADAF80020444B1A6067
:103CE00083ED01AA08F51B63B0EE490A472093ED66
:103CF000001A0C93F1EE410A21F0C8F80C9BB0EECB
:103D000040AA482093ED001AB0EE680AF1EE410A8D
:103D100021F0BCF808F6B41308F6B818B0EE409AD3
:103D200093ED001A4920B0EE4C0AF1EE410A21F061
:103D3000ADF898ED001AF0EE408A4A20B0EE6B0A1A
:103D4000F1EE410A21F0A2F895ED007AD5ED017A65
:103D500004F6A8336AEE076A8DED148AF0EE40BAD5
:103D60008DED158ACDED106A69EE276ACDED116AE9
:103D7000D3ED006A04F6AC3327EE267AD3ED006A61
:103D80009DF8343067EEA67A8DED127ACDED137A78
:103D9000A3BB9DF835308BBBB0EE690A19ABB8EE0A
:103DA0004BBA12AAF8EE6AAA10A912488DED19BAF8
:103DB000CDED1AAA72F094FA8DED140ACDED150A24
:103DC0001CE000BFA02C0030A4707D3F00D7233C36
:103DD00090E110086C13110885131108705400301D
:103DE0005488003000000000A07C0030008C0030BF
:103DF000A08C003030890030A06C00309DF8363047
:103E0000002B40F0F88004F53B6395ED000AB0EE1E
:103E1000691A1CEE901AD3ED000A8F4860EE200A52
:103E200028EE800A72F08EFCF0EE40AA14A98B48AE
:103E3000FEF74CFD9DF83730002B40F0DF8004F694
:103E4000C43395ED010AB0EE691A1DEE101AD3EDD8
:103E5000000A834860EE200A20EE2B0A72F072FC02
:103E6000F0EE409AD4F8AC351B7B7BBB19A97D489A
:103E70008DED198A8DED1A8A72F05CFB9FED7A0A3E
:103E80007A4872F07BFC9FED780A794872F09CF9D1
:103E900019A978488DED198A8DED1A8A72F04AFBBE
:103EA0009FED710A6C4872F069FC6D489FED6E0AD7
:103EB00072F064FC04F6B43393E807000B9B03F53F
:103EC000FA6386E807001B68CAF80030B9F1000FF2
:103ED00000F09780D4F8AC3583ED368A0A9B002B2E
:103EE00000F09A80D4F8AC3583ED358A002F00F0CD
:103EF0009E80D4F8AC3583ED388ABBF1000F00F01A
:103F0000A080D4F8AC3583ED378A04F6A8339FED52
:103F10005A8A9FED554AD3ED002A04F6B433D6ED04
:103F2000000AF0EE443A93ED001AB0EE443A62EE25
:103F3000882A2AEE082AF0EE441A21EE081A60EECA
:103F4000880AB0EE440A84F0F9FA04F6AC339FED27
:103F5000464A29EE082AD3ED002A04F6B833D6EDF6
:103F6000010AF0EE443A93ED001AB0EE443A62EEE4
:103F7000882AF0EE441A21EE081A60EE880AB0EEA4
:103F8000440A84F0DFFA04F53B6304F6BC349FED89
:103F9000364AD3ED002A28EEC82A94ED001AF0EE36
:103FA000443AD6ED020AB0EE443A62EEC82AF0EE88
:103FB000441A21EE481A60EEC80AB0EE440A84F0B2
:103FC000C5FA1DB0BDEC0C8BBDE8F08F4FF00109B8
:103FD000DDE50123EFE5012702E64FF0010B11E6D5
:103FE000F0EE488AB0EE489A4CE69FED1FCA5FE6B5
:103FF000DFED1DBA76E6DFED1CAA17E7DFED1A9AB2
:1040000030E79DF83430002B7FF468AFD4F8AC353E
:10401000149AC3F8D82061E79DF83530002B7FF45F
:1040200065AFD4F8AC35159AC3F8D4205EE79DF897
:104030003630002B7FF461AFD4F8AC35C3ED38AA2D
:104040005BE79DF83730002B7FF45FAFD4F8AC35D9
:10405000C3ED379A59E700BFE4890030A02C003047
:104060005C8A0030D48A003000000000888B003069
:10407000008C0030308900300000C8422DE9F04F3C
:104080002DED068B91B0064688460593C74B0392EB
:1040900003F5A044D3EDB9AAD4F8AC25127B002ACD
:1040A00000F0508103F58043B3F8CA59C5F3400BC3
:1040B00005F0010AC5F3800715F0080500D00125B9
:1040C00005ABDFF800933A465146009358462B461D
:1040D000FFF7A6FC99ED001A98ED000AF1EE410AEF
:1040E00007909A2020F0D2FE4B46F0EE409A9B209B
:1040F000B3EC011A98ED010AF1EE410A049320F0A5
:10410000C5FE049BB0EE409A9C2093ED001A98EDFA
:10411000020A4FF00008F1EE410A20F0B7FE039BBF
:1041200099ED021AF0EE408A9D2093ED000AF1EE1F
:10413000410A20F0ABFE96ED007AD6ED017A04F646
:10414000A83369EE876ACDF83080B0EE408ACDF8AA
:104150003480CDED086A69EE276ACDED096AD3EDAA
:10416000006A04F6AC3327EE267AD3ED006A9DF898
:10417000143067EEA67A8DED0A7ACDED0B7AFBB995
:104180009DF81530E3B99DF81C30B0EE6A0A0AAA12
:1041900008A907EE103A9DF81D3009F5975007EE73
:1041A000903AB8EE477A0EABF8EE677A8DED0E7A5C
:1041B000CDED0F7A72F094F88DED0C0ACDED0D0A6D
:1041C0009DF81630002B40F0C18004F53B6396ED5E
:1041D000000AB0EE6A1A9DF81E10D3ED000A74486A
:1041E00060EE200A28EE800A72F0ACFAB0EE40AA27
:1041F0000CA96E48FEF76AFB9DF81730002B40F0C3
:10420000A88004F6C43396ED010AB0EE6A1A9DF850
:104210001F10D3ED000A674860EE200A20EE080A5E
:1042200072F090FAB0EE408AD4F8AC351B7B8BB9B3
:104230000EA96148CDF83880CDF83C8072F07AF94B
:104240009FED5E0A5A4872F099FA9FED5C0A594850
:1042500072F094FABBF1000F7ED0D4F8AC35C3F8FD
:10426000D880BAF1000F00F08180D4F8AC35C3F8E3
:10427000D480002F00F08580D4F8AC35C3F8E080FE
:10428000002D00F08880D4F8AC35C3F8DC8004F64B
:10429000A8339FED4B8A9FED494AD3ED002A04F6DF
:1042A000B433F0EE443A93ED001AB0EE443A62EEC5
:1042B000882A29EE882AF0EE441A21EE081AF0EE38
:1042C000440AB0EE440A84F039F904F6AC339FEDA9
:1042D0003B4A29EE082AD3ED002A04F6B833F0EE63
:1042E000443A93ED001AB0EE443A62EE882AF0EEBA
:1042F000441A21EE081AF0EE440AB0EE440A84F0A3
:1043000021F904F53B6304F6BC349FED2C4AD3ED50
:10431000002A28EEC82A94ED001AF0EE443AB0EED6
:10432000443A62EEC82AF0EE441A21EE481AF0EE42
:10433000440AB0EE440A84F009F911B0BDEC068BD2
:10434000BDE8F08F0127BA46BB46B8E69FED1BAA31
:104350004EE79FED1A8A67E79DF81430002B80D155
:10436000D4F8AC350C9AC3F8D8207AE79DF815300C
:10437000002B7FF47EAFD4F8AC350D9AC3F8D4206F
:1043800077E79DF81630002B7FF47AAFD4F8AC3580
:1043900083ED38AA74E79DF81730002B7FF477AFD0
:1043A000D4F8AC3583ED378A71E700BFA02C00301C
:1043B000E48900305C8A0030308900300000000061
:1043C0000000C8425076003070B5044610305EF0F0
:1043D00063F9A0250A4B0B4E236160195EF036FC91
:1043E00066513035B5F5687FF7D104F5687060F037
:1043F000FDF9204604494AF0C3FC204670BD00BFC9
:10440000DC1C1108C81C1108E815110837B500F5A7
:1044100093410122044604314DF024FC1E4A1368E6
:10442000D9070AD404F580431C4920330B6004F5F6
:104430008A437833CB600123136004F59340022252
:104440001649012554304AF06FF8002304F5DF5176
:10445000134AFD200831CDE9005349F0F7FF114B15
:10446000012111481A68D2075FBF0F4A04F51054A2
:104470001D6014604AF074F84AF074FE0B4A04217F
:104480000B48138843F040031380002203B0BDE8BB
:10449000304049F0D7BF00BF0C8E0030C42500303B
:1044A00088BF1108108E0030DC2500302C900030C1
:1044B000EC1A11080069C0F3401070470F299DBF26
:1044C000302303FB0100903000207047014B93F92B
:1044D0009E097047A06C0030024B93F8A90500F0CC
:1044E00001007047A07C0030014BD3F838037047BF
:1044F000A07C0030002910B517DB104CCBB294F82B
:1045000040239A4211D3D4F83C330122A4F5A040B1
:10451000595C00F077FD94F8993538B99A0704D5BD
:10452000074A137843F00403137010BD9B07FCD5B2
:10453000034A137843F00203F6E700BFA07C003083
:10454000AC8F0030022A10B50F4C12D13522A4F5E1
:10455000A04000F057FD94F899359B0705D50B4B0B
:104560001A7818B142F002021A7010BD42F004022B
:10457000FAE794F89C258A42F7D15EF091FABDE8FB
:1045800010405EF07BB900BFA07C0030AC8F0030E3
:10459000064A92F8A93592F8A82503F001031343BF
:1045A00001D15EF065B80020704700BFA07C0030EC
:1045B000332901D05FF006BB7047000008B50A68D8
:1045C000332A07D0382A08D10A790321FFF7BAFF26
:1045D000012008BD0A790121F8E7BDE808405EF036
:1045E00069BF000030B5044689B004F51655684629
:1045F00007F042FA04A8383507F03EFA6946284623
:1046000003F068F878B104A9284603F005F950B121
:1046100004A9684607F05EFA236800226946D3F8C9
:10462000B8302046984709B030BD000000F5005270
:1046300092F84C28D2070BD400F5A042D2F8AC2552
:10464000117B09B1FFF7CEBF0368D3F8B430184728
:104650007047000010B586B0044602A8019107F02B
:104660000BFA04F5165002A9383003F033F830B1D4
:10467000236802A9019A2046D3F8B830984706B0BB
:1046800010BD0000F0B5044685B00F46154604F590
:104690001656684607F0F0F969463836304603F09A
:1046A000BBF810B9002005B0F0BD3946304602F025
:1046B00043FE0028F6D0002DF5D004F5005428461E
:1046C00094F84C3843F0020384F84C38EBE70000D0
:1046D00010B500F593448AB00023D4ED0A7A28344B
:1046E000F5EEC07AF1EE10FA44D9079300F51650B2
:1046F000089303AA099306AB04A93830019307ABCA
:10470000009305AB02F0B6FEDDED087A9DED077A69
:1047100087FE277ADDED097A87FE277AD4ED007AC5
:10472000B4EEE77A9DED047A77EEA76AF1EE10FA1F
:10473000F4EEC76AACBF01200020F1EE10FA0CD8ED
:1047400002309DED037AF4EEC77AF1EE10FA0CD840
:10475000003818BF01200AB010BDF4EEC77AF1EEA0
:1047600010FA9CBF0130C0B2EBE7012894BF0020D3
:104770000120F0E70020EEE700F5A04210B592F826
:10478000A935044659071BD443F0040382F8A93520
:1047900050F0BAF8012211214FF066FE094B186E55
:1047A00003689B68984728B904F5804393F9A539B5
:1047B000032B05D120460621BDE8104000F01EBDA8
:1047C00010BD00BFA08C003000F5A04008B590F8E7
:1047D000A9355A070BD56FF3820380F8A93550F03D
:1047E00093F800221121BDE808404FF03DBE08BDFE
:1047F0002DE9F043054685B005F51658684607F0E3
:104800003BF9694608F13808404603F005F8D8B18D
:1048100005F5A043434C444FD3F8AC351B7B43B163
:1048200005F59343D3ED0A7AF5EEC07AF1EE10FA6E
:104830000DD82388284623F4FF7323F00103238037
:104840000023FB73FFF7C0FF05B0BDE8F0832846E7
:1048500001F070F8064618B9284601F02FF8064610
:104860002846FFF735FF814640B93EB12378002B3B
:1048700041D1637803F00103FB73E5E76378DB075D
:10488000F7D423780133DBB2082B237006D12846F6
:10489000FFF71EFF10B1404602F06CFE2378092B93
:1048A00002D1404602F05EFE2378092BE1D923882D
:1048B00023F4FF7323F0010343F48573238050F046
:1048C00023F8022210214FF0CFFD85F06DFD6368C3
:1048D000C01A47F23053984209D905F5A740134A48
:1048E0000221443055F06CFD85F05EFD6060284685
:1048F000FFF742FFBDE7013B23702388C3F30803A2
:10490000B3F5807FB5D1637860F3000363704FF037
:10491000FBFF4A4610214FF0A7FD2846FFF754FF42
:10492000A7E700BF148E00308D8F0030F81C1108EF
:1049300037B5044600F5165001A904F5A0453830F6
:1049400002F03EFCD5F8B033834206D0C5F8B00380
:104950004FF0DAFF3E214FF067FD04F5005395F963
:10496000B41393F8E02893F9E038994213D0FF2A62
:1049700011D085F8B4334FF0C7FF95F8B423182150
:104980004FF072FD04F5A74095F9B4330421034AB2
:10499000443055F015FD03B030BD00BF081D1108AF
:1049A0002DE9F043064695B085F0FEFC002403ABEC
:1049B00006F5165805460BAA019308F1380802AB14
:1049C00008A94046089400930EAB09940A940B94EE
:1049D0000C940D940E940F94109402F039FDDFEDB9
:1049E000427A07469DED0A7AB4EEE77AF1EE10FAC4
:1049F00037DB9DED0D7AB4EEE77AF1EE10FAACBF3D
:104A00004FF001094FF0000907AB1194129404AA6A
:104A1000019311AB139406F5A044009305A906ABCE
:104A2000404602F027FD94F92033002808BF0027F4
:104A300083B17FB1D4F8AC351B7B5BB1B9F1000F0A
:104A400008D0F7EE007A9DED057AB4EEE77AF1EE44
:104A500010FA09D594F8B83363B90023C4F8BC330D
:104A60000DE04FF00009CFE7D4F8BC0310BBC4E958
:104A7000EF5004E0D4F8C00320B9C4F8C05315B017
:104A8000BDE8F083281A43F698239842E5D900251B
:104A900084F8B853C4F8C0534FF036FF2A461D219E
:104AA0004FF0E2FC06F5A740104A0221443055F0D1
:104AB00087FCD2E72D1AB5F57A7FE0D994F8B833A0
:104AC000002BDCD1012584F8B8534FF01DFF2A4696
:104AD0001D214FF0C9FC06F5A740054A02214430CC
:104AE00055F06EFCCBE700BF00000034201D11081C
:104AF0003B1D110810B504464FF006FF00220521AA
:104B00004FF0B2FC04F5A740034A04214430BDE84D
:104B1000104055F055BC00BF581D110800F5A040CD
:104B200090F899359B065ABF90F89805C0F300108D
:104B30000120704738B5044603F09AF84FF48041DD
:104B400002F00AF904F5A042054692F89935C3F33C
:104B5000001181421CD060F3041304F5A74482F8CD
:104B60009935443460B14FF0CFFE02220B214FF053
:104B70007BFC084A20460221BDE8384055F020BCA5
:104B80004FF0C2FE2A460B214FF06EFC024AF1E7BD
:104B900038BD00BF701D11087B1D110800F5804352
:104BA00070B593F98E390446B3B300F5A045D5F836
:104BB00024658EB385F0F8FB95EDCA0ADFED177A10
:104BC000861B9FED171A692020EE270ADFED150AD4
:104BD00020F05CF9BCEEC00A10EE103A9E4209D2F9
:104BE00095F8A9359A0717D520460021BDE87040F1
:104BF000FDF706BB10D995F8A9359B070CD42046C4
:104C00000121FDF7FDFA04F5A640012212214830EA
:104C1000BDE87040FDF74EBA70BD00BF00007A4499
:104C20000000804F000000000B461146012B10B41D
:104C300004D0052B06D05DF8044B70475DF8044B9B
:104C400000F0DCBA00F5A640012214215DF8044B07
:104C50004830FDF72FBA0000F8B504464FF054FE77
:104C6000012205214FF000FC04F5804304F5A7461E
:104C7000204693F992594436003D18BF0125FFF7AD
:104C80004DFF98B11E4A04213046002555F098FB8F
:104C900004F5A640012210214830FDF70BFA294601
:104CA00020460322BDE8F840FFF7BEBF04F5C04729
:104CB000386E0368DB6A984778B104F5A04393F82F
:104CC000792B52B193F9783B012B06DC0D4A042174
:104CD0003046012555F074FBE1E7386E0368DB6A66
:104CE000984728B104F5A043D3F824331B0705D413
:104CF000054A0421304655F063FBD0E7034AE6E756
:104D0000901D1108AB1D1108D91D1108E81D1108CF
:104D100070B5044615464FF0F7FD0122062104F553
:104D2000A7464FF0A1FB20464436FFF7F7FE98B1A7
:104D300004F5A6400122072100254830FDF7BAF905
:104D4000134A0421304655F03BFB294620460422F5
:104D5000BDE87040FFF768BF04F5C043EDB2186EC0
:104D60000368DB6A984768B104F5A043D3F824339D
:104D70001B0707D535B1074A04213046012555F0F8
:104D80001FFBE2E7044A0421304655F019FBDCE73B
:104D90000C1E1108B31D1108291E1108F8B5044690
:104DA00085F0F8FA284B0546B4F8C6221988274E34
:104DB00091420ED01A80264B18603378A3B100249C
:104DC00034704FF0A1FD22461321BDE8F8404FF0AA
:104DD0004BBB33781F4FC3B93B782BB11C4B1E4ADA
:104DE0001B68C31A934200D8F8BD0123337004F541
:104DF000A043D3F8AC05037B0BB1FEF791F94FF05C
:104E000083FD012213214FF02FFB3B78002BEBD0C9
:104E10003378002BE8D00E4A10491368EB1A8B4206
:104E2000E2D904F5A0441560D4F8AC25137B002B1F
:104E3000DAD0002313730A4AD4F8AC051371BDE825
:104E4000F840FEF743B800BF1E8E00301C8E0030C5
:104E5000208E00301D8E003080841E0040420F00E6
:104E60008D8F0030F0B5044600F5B84500F5A04739
:104E700085B0743504F5165697F8B81328463836B9
:104E800083F04EFA684606F0F7FD6946304602F0B8
:104E900021FC029B20213046C7F8943B039BC7F8B6
:104EA000983B01F059FFD0B1284604F5B74583F08F
:104EB00089FAFDEEC07A0C3504F50054022217EE93
:104EC000901A284617EE906A06F0DAFD94F84C38EE
:104ED000DB0706D401223146284606F0D1FD05B095
:104EE000F0BD0121284606F0A5FE0028F2D0F6E725
:104EF0000120704700207047002070470020704755
:104F00000020704700207047002070470020704745
:104F10009FED010A704700BF000000009FED010AED
:104F2000704700BF0000000070470000104A026098
:104F3000104A02F150014260816001F59551C16053
:104F40000D49016102F62841416102F62C4181615F
:104F500002F6A811C16102F6AC11016202F51B61F3
:104F600002F6B41241628262044AC262704700BF14
:104F7000B41E11082476003058520030C02F003083
:104F8000042918D8DFE801F003070B0F130000F520
:104F9000C1401430704700F5C0406430704700F5E0
:104FA000C1404430704700F5C1407430704700F58F
:104FB000C2403430704700207047000000F5C04008
:104FC000006E03685B68184738B500F5C0450446B5
:104FD000286E03685B699847094B04F5A042187472
:104FE00092F89C25286EDA7003685B6A9847014640
:104FF00004F51550BDE83840283046F0F9B800BF38
:105000008D8F00302DE9F84F00F5A04A06460F4677
:1050100091469AF89C358B4205D101258AF89D2549
:105020002846BDE8F88FFFF7ABFF044620B93046AD
:1050300025464CF0D3FFF3E7DAF8AC3506F5A74880
:105040001B7B08F1440883F0010BE3B92368594640
:1050500020461B689847054678B306F5C04306F519
:10506000DF504A4639461C6608308AF89C758AF833
:105070009D954EF0FDFD404600215CF02BFD304635
:10508000FFF7A2FFCCE703689B689847E0B11C4894
:1050900000F03AFC0546B8B9236820461B6A9847D9
:1050A000184A03460421404655F08AF94FF02CFC7B
:1050B0003A460A214FF0D8F9B2E7236820461B6A26
:1050C0009847114A0346EDE70D4800F03BFC0028E5
:1050D000BCD106F5C043186E0368DB68984700280A
:1050E000B4D023682046DB68984705460028ADD138
:1050F000236820461B6A9847044A0346D2E700BF4C
:10510000A02C00303C1E11088E1E1108651E1108CF
:105110000148FFF777BF00BFA02C0030234B70B5CC
:1051200093F8A93505460C461646DB0705D500233E
:1051300063602360A360336070BD5DF0B1FC037FEA
:10514000002BF4D0EB699FED1A7A1B68B3F90A3093
:1051500007EE903AF8EEE77AC7EE876AC4ED016A87
:105160002B6A1B68B3F90A3007EE903AF8EEE77A3B
:10517000C7EE876AC4ED006A6B6A1B68B3F90A3030
:105180005B4207EE903AF8EEE77AC7EE876AC4ED25
:10519000026AAB6A1B68B3F90A3007EE903AF8EE80
:1051A000E77AC7EE876AC6ED006AC5E7A07C0030E3
:1051B00000007A44002070470120704700207047AB
:1051C0000020704700487047D88D1108004870478C
:1051D000FC1E11080020704743691A680023C2F8BA
:1051E000D43042691268C2F8D83042691268C2F8F5
:1051F000DC3042691268C2F8E03070470A4600218C
:1052000008B5FFF7FFFE034A137843F00803137055
:1052100008BD00BFAC8F00300120704700207047F0
:105220000120704700207047004870479CE4110837
:1052300000487047541F110803207047084B03F5BE
:10524000B74203F51F533432103330B5044600F132
:10525000300507CA85E807001B680120E36330BDFD
:10526000A02C003030B52DED028B87B00023044612
:10527000584D01AA03A995EDB98A039304930593A8
:10528000FFF74CFF63689DED037AD3ED0E7A68EE6D
:10529000277A27EE277A8DED037A9DED047A67EE63
:1052A000277ACDED047AD3ED0F7A28EE277ADDED5B
:1052B000057A67EE877ACDED057AD3ED107A93F90A
:1052C000443028EE278ADDED017A27EE888A8DEDBD
:1052D000018A1BB903A92846FDF7E0FA3E4D94ED7B
:1052E0000C7AD5ED007AA5F6B435636877EE677A67
:1052F00005F6B832D3ED0E6A94ED0F0AF0EEE77AB8
:10530000F4EEE67AF1EE10FA44BFDDED037A77EEC3
:10531000877A94ED0D7A48BFC4ED0C7AD2ED007A0D
:1053200005F6BC32D3ED0E6A77EE677AF0EEE77AD7
:10533000F4EEE67AF1EE10FA44BFDDED047A77EE92
:10534000877A94ED0E7A48BFC4ED0D7AD2ED007ADB
:10535000D3ED0F6A77EE677A2369F0EEE77AF4EE21
:10536000E67AF1EE10FA42BFDDED057A77EE877A44
:10537000C4ED0E7AD3ED867A30EE670A1FF05AFD3F
:105380006368B0EEC00AD3ED107AB4EEE70AF1EE2E
:1053900010FA09D594ED0F0ADDED017A30EE270AF7
:1053A0001FF048FD84ED0F0A002304F13C0204F1D4
:1053B0003001D5F8B0058DF808308DF809308DF83A
:1053C0000A308DF80B30029BFEF740FB07B0BDECB6
:1053D000028B30BDA02C0030548800300020704774
:1053E0000120704701207047002070470048704737
:1053F000AC1F110800487047B41F11080120704706
:105400001FB5044600236A4601A901930293039342
:10541000FFF784FE6369029A1B68C3F8D4206369AE
:10542000019A1B68C3F8D8206369009A1B68C3F807
:10543000DC206369039A1B68C3F8E02004B010BD48
:1054400001207047002070470120704700207047FE
:10545000004870479EE71008004870479EE7100814
:1054600004207047012070477FB500230B4801AA34
:1054700003A903930493059301930023D0F8B00587
:105480008DF808308DF809308DF80A308DF80B3022
:10549000029BFEF7DBFA07B05DF804FBA07C00304E
:1054A000012070470020704701207047002070479E
:1054B000004870475C2011080048704768201108B8
:1054C0000220704710B586B00023044601AA03A944
:1054D000039304930593FFF721FE63689DED037A20
:1054E000D3ED0B6ADDED047A27EE267A93F944308A
:1054F00067EEA67A8DED037ACDED047A1BB903A988
:105500001348FDF7CBF9636801AADDED057A03A91D
:1055100093ED0C7A0F4867EE877A93ED0D7A0023AE
:10552000D0F8B005CDED057ADDED017A8DF80830C3
:1055300067EE877A8DF809308DF80A308DF80B30D8
:10554000029BCDED017AFEF799FD06B010BD00BFBC
:10555000A02C0030A07C003038B504465FF0B2F9D2
:105560005FF01EFB054604F5A0445FF08DFA5EF087
:1055700031FED4F8AC05FDF7A9FC2846BDE838405B
:105580005FF08ABA10B500F5A0441421D4F82C03BA
:105590005DF070FBD4F8300314215DF06BFBD4F8A0
:1055A00034031E215DF066FBD4F838031421BDE8F6
:1055B00010405DF05FBB000038B505465DF070FA45
:1055C0005DF0BCF905F5A044C4F82C035DF068FA61
:1055D0005DF0BEF9C4F830035DF062FA5DF0C2F927
:1055E000C4F834035DF05CFA5DF0C6F94FF47A71EB
:1055F000C4F83803D4F82C035DF038FB4FF47A710B
:10560000D4F830035DF032FB4FF47A71D4F83803EC
:105610005DF02CFB4FF47A71D4F834035DF026FB77
:105620002846FFF7AFFF94F8993543F0080384F854
:10563000993538BD08B55FF0B3FA5EF087FFBDE875
:1056400008405EF039BF000000F5A040D0F8AC057E
:10565000FDF766BD38B500F58043054693F99229FC
:105660002AB900212846BDE83840FCF7AFBDB3F8A1
:10567000943900F5A0448B4219D994F8A935DA077A
:105680000FD45DF00DFA037F1BB9D4F8AC351B7B4A
:105690003BB194F8A83501335BB2022B02DC84F8ED
:1056A000A83538BD0323012184F8A835DAE794F83A
:1056B000A835013B5BB2002BF1DC002384F8A83550
:1056C00094F8A935DB07CCD4EBE7000038B50D46DC
:1056D000044684F069FE0C4B002D09DD04F5A0445E
:1056E000186094F899356FF3C30384F8993538BD81
:1056F0001B68C01AB0F5C87FF9D904F5A04494F826
:10570000993543F00803F0E7248E0030F7B50446DE
:1057100084F04AFE06465DF0C3F904F5A0455DF04D
:1057200091F998B395F89835204604F5C04743F0B1
:10573000200385F89835D5F834331989FFF78AFFA7
:10574000D5F834332046B3F90A10FFF7BFFFBB6D1D
:105750009FED2E7A6A46F31A01A904F5B74007EEC9
:10576000903AD5F83433F8EE677AB3F90A3067EE39
:10577000877ACDED007A07EE903AF8EEE77ACDED34
:10578000017A51F00DFCBE6503B0F0BD95F8A93566
:10579000DB07F9D404F5C043986D361A5DF020F8A4
:1057A00088BB5DF07DF99FED1A7AD0ED067A67EE41
:1057B000877A9FED187AF4EEC77AF1EE10FA77FE49
:1057C000877AFCEEE77A17EE903AB342DCD804F51C
:1057D000804393F99239002BD6D05DF061F9037FB5
:1057E00023B9D5F8AC351B7B002BCDD04FF08CF80E
:1057F000022211464EF038FE0121204603B0BDE8DA
:10580000F040FCF7E3BC4FF47A73DEE76F12833AA3
:1058100000007A440000C84238B500F5EE65044641
:10582000284604F07DFE94F8810750229FED087A07
:1058300004F5A04302FB0055D5ED0B7A67EE877A9D
:10584000FDEEE77A17EE902AC3F87C2B38BD00BF37
:105850000000C842FEF7C2B80148FFF79FBA00BF78
:10586000A02C003010B5838F044643B94DF0F2F8F8
:1058700092224FF480114DF0A5F8638FA387A08F7B
:1058800010BD000038B500F51655044638352846D9
:1058900000F0FAFC04F50053022204F51C7083F8B2
:1058A000D827FFF7DFFF014604F546601DF014FF1F
:1058B0002846BDE8384000F0EDBD000038B500F5E1
:1058C000165405463834204600F034FF08B900204D
:1058D00038BD05F5A045D5F8AC351B7B63B9102163
:1058E000204601F039FA0028F2D14FF40071204629
:1058F000BDE8384001F030BA8021204601F02CFA92
:105900000028E4D11021F2E738B500F5A0430546A0
:1059100093F8A9355B070AD4FFF7D0FF044620B9F6
:1059200005F51650383000F005FF204638BD00243C
:10593000FBE7000000F5165008B5383000F0FAFE1D
:10594000002008BD10B500F516543834204600F08C
:10595000F1FE50B10421204601F0FEF928B12046A5
:105960002021BDE8104001F0F7B9002010BD000073
:1059700038B500F5A045044695F89835590718D56F
:10598000D5F8AC351B7B2BB920460021BDE838404B
:10599000FCF706BC00F5C043186E0368DB68984747
:1059A00038B195F899351A0703D595F8A935DB076D
:1059B000EAD538BD37B500F5DF5504460191083505
:1059C00004F5A04428464EF09BF894F898350199C8
:1059D00060F3C303284684F8983503B0BDE830402F
:1059E0004EF0B0BD0720704700487047C020110836
:1059F00037B505461148FFF735FF0190EC2006F05A
:105A000099FC044610B10199FDF700FA05F5A04391
:105A1000C3F8AC4534B905F58045094895F9E01956
:105A200005F0BAFF0749204649F0A4FB012049F0E0
:105A300041F803B0BDE8304049F094BB102F00306E
:105A4000C820110860D9100873B5044600F5155038
:105A5000283004F5EE6645F033FB2046FFF7B4FA34
:105A600004F5AB40403005F04BF904F5E850183030
:105A70005FF0F6FE304604F0C9FB04F5A740443061
:105A800057F08CFC2046FFF797FD2046FFF7B0FF4C
:105A90006148FFF7E7FE082006F04CFC18B14FF014
:105AA0007E530360436004F5A045C5F8B0055CF083
:105AB000F7FF992229215EF0CDFA5CF0F1FF5CF04E
:105AC000FBFE2046FFF7B6FD95F8993504F5145016
:105AD00043F04003143085F8993563F055F94F4B86
:105AE0004FF47A724E491B68986A0368DB6A9847DC
:105AF000042304F54A70C4F8C4330EF0DBFF07F04A
:105B000011FB4FF40053436307F00CFB08F026F938
:105B1000802301213046C4F8843704F021FE414B34
:105B200004F5DF500093404B0830019302AB13E9BA
:105B300006004DF08DFE2046FFF7A4FE04F58053CD
:105B40004FF40022C3F86C25D5F8AC05FDF768F9D1
:105B500004F5A64001214830FCF716F810B12046A4
:105B6000FFF772FD04F51C763046FFF77BFED5F893
:105B7000AC3507EE900A04F5B740D3ED390AF2EEE2
:105B80000E1AB8EE670A4830B6EE001A51F008FF58
:105B90003046FFF767FED5F8AC3507EE900A04F5FE
:105BA000B840D3ED390AF2EE0E1AB8EE670A0C309F
:105BB000B7EE001A51F01EFD3046FFF753FED5F840
:105BC000AC3507EE900A04F5B840D3ED390AF2EE91
:105BD0000E1A4030B1EE041AB8EE670A51F00AFD11
:105BE00004F580431A22204693F89F19FFF70AFA1A
:105BF00060B9212201212046FFF704FA95F8993572
:105C000043F0020385F8993502B070BD074A137856
:105C100043F008031370F1E7102F0030088E0030B6
:105C200059580208A02C003055580208AC8F00309B
:105C3000836833B9C36823B94068003818BF0120AE
:105C400070470120704700002DE9F0412DED048BD5
:105C500092B0044602AD284605F00EFF94F8D43306
:105C6000002B70D004F58063D4EDF28A94EDF38AB2
:105C700094EDF49A0FCB85E80F0094F81034002BC4
:105C800061D094F8E833002B5DD02846D4F8D8834F
:105C9000D4F8DC73D4F8E063D4F8E443FFF7C8FF2A
:105CA000002855D12E4B01932D22002106A8E3F0A8
:105CB00065F8A3238DF8183095238DF81930462305
:105CC0008DF81A3084F078FB9FED260ADFED267AF6
:105CD00068EE808ACDF81F1028EE008ACDF81B00F0
:105CE00029EE000A68EEA78A28EE278A20EE270A06
:105CF000FDEEE88ABDEEC88A18EE903AADF8233082
:105D000018EE103AADF825301FF050F8BCEEC00A7E
:105D1000CDF83580CDF83970CDF83D6010EE103AF1
:105D2000CDF84140ADF82730019BCDF82930049BD8
:105D3000CDF82D30059BCDF831304EF0E5FD2D220C
:105D400006A94DF0BDFD12B0BDEC048BBDE8F0819D
:105D500001AA0021284605F07DFF0028A2D0A3E774
:105D60005241C07FE02E65420000C84230B52DEDA3
:105D7000028B8BB0044624220D4601A80021E2F0DC
:105D8000FDFFA3239FED228A8DF8043095238DF823
:105D9000053048238DF8063084F00EFBD4ED847A6C
:105DA0002B6867EE887A95ED020ACDF80F30CDF8B2
:105DB0000B1017EE903AD4ED857ACDF8070067EE18
:105DC000887ACDF813306B68CDF8173017EE903A1B
:105DD000CDF81B301EF0B6FF10EE103A94ED860A97
:105DE00020EE080ACDF81F301EF0ACFF10EE103A7E
:105DF000CDF8233094F824338DF827304EF084FD0D
:105E0000242201A94DF05CFD0BB0BDEC028B30BD2E
:105E1000E02E654230B5104689B00D461446FFF7B6
:105E200007FF28BB002301931822002102A8E2F0FB
:105E3000A5FFA3238DF8083095238DF80930492359
:105E40008DF80A3084F0B8FAA368CDF80F100593E6
:105E5000E368CDF80B000693019B8DF81350079370
:105E60004EF052FD182202A94DF02AFD09B030BDB6
:105E700001AA0021204605F04FFE0028D2D0D3E72A
:105E800010B590B0044604A805F0F6FD04A920461C
:105E900001F020FC002846D001F0EAFE01A901F043
:105EA000EFF902A9204600F00FFD00283DD0DDEDFE
:105EB000027AF1EE677A03AA002104A8CDED027AF6
:105EC00005F0C8FE08B91A4B03931F22002108A849
:105ED000E2F054FFA3238DF8203095238DF8213074
:105EE0004A238DF8223084F067FA069BDDED017AB3
:105EF000CDF82B30079BF1EE677ACDF82710CDF85F
:105F00002F30039BCDF82300CDF8333017EE903AB5
:105F1000CDF83730029BCDF83B304EF0F5FC1F2218
:105F200008A94DF0CDFC10B010BDDFED027AC2E73C
:105F30005241C07F5241C07F0023036043608360B1
:105F4000C360036143618361C36103627047000002
:105F5000B02290F80C3302FB030390F8A12393F8CE
:105F6000E93012B1012B28BF012318467047000009
:105F70002DE9F04F05464FF0000A8BB00C4627F094
:105F8000D3FB05F5097085F820A24FF07E5783F00A
:105F900045FB4FF47A7305F5217085F88042A5F82A
:105FA0007A320024C5F8607205F53179C5F864725B
:105FB00005F53A76C5F8687205F54E7B05F05CFD8F
:105FC00003234846C5F8AC42C5F8983205F27C4830
:105FD000C5F8B042C5F8B442C5F8B842C5F8BC42ED
:105FE000C5F8C042FFF7A8FF3046FFF7A5FF5846A7
:105FF000C5F82C43C5F83043C5F83443FFF79CFF80
:1060000005F57B70C5F85C43C5F86043C5F864438B
:10601000C5F86843C5F86C43C5F87043C5F87443C8
:10602000C5F87843C5F87C43C5F88043C5F8844378
:10603000C5F88843C5F8A443C5F8A843C5F8AC43E0
:10604000C5F8C043C5F8BC43C5F8B843C5F8C84354
:10605000C5F8CC43C5F8D043C5F8E443C5F8E043E0
:10606000C5F8DC43C5F8B473C5F8D87305F004FD72
:1060700005F5806005F000FD05F2144305F5866026
:106080001C605C6005F584631C605C609C6005F0CE
:10609000F3FC05F24443404605F254421C605C6048
:1060A0009C60764BC5F8543405F51073C5F8583428
:1060B00005F51173C5F85C3405F51273C5F8603445
:1060C00005F51373C5F8643405F25123C5F8683437
:1060D00005F51473C5F86C3405F58E631C605C60BF
:1060E0009C60FFF729FF05F59460FFF725FF05F594
:1060F0009A6305F2EC501C605C609C6005F2DC4326
:106100001C605C609C6005F59D631C605C609C602D
:1061100005F2F4431C605C609C6005F204531C6053
:106120005C609C6005F214531C605C609C6005F52B
:10613000A4631C605C609C6005F22C531C605C6076
:106140009C6005F5AA63C2F8EC70C2F8F0701C60A0
:106150005C609C6005F25C531C605C609C6005F5B3
:10616000AD631C605C609C6005F274531C605C60F5
:106170009C6005F5B2631F605C6005F2B4531C605F
:106180005C609C6005F5B8631C605C609C6005F514
:10619000BB631C605C609C6005F06EFC05F2FC5308
:1061A000242251461C6040465C6005F204631C607A
:1061B0005C6005F20C631C605C60E2F0DFFD05F5DD
:1061C000C660C8F82070C8F81070C8F80070FFF7F3
:1061D000B3FE05F2546305F2AC601F609C605C6026
:1061E000DC6005F264631C605C609C6005F5CE6356
:1061F0001C605C609C6005F27C631C605C609C6061
:1062000005F5D1631C605C609C6005F294631C60C2
:106210005C609C60344605F02FFC194B28461949F8
:106220001D6048F0ADFD5146242258466E46E2F00E
:10623000A5FD05F52B7205F52E73C5F85873C5F845
:106240004873C5F8387307CA83E80700484695EDD8
:10625000B01AD5EDAF0A95EDAE0A1FF0E5FA494642
:1062600068461FF009FA0FCE0FC40FCE0FC42846A0
:10627000336823600BB0BDE8F08F00BFA82311087E
:10628000288E00304422110810B5044688B001F071
:106290005BFD94F93E32012B02D1274805F09AFBB1
:1062A000022B0AD1032304A904F1110084F83E3221
:1062B00001238DF8103049F06FFD94F83E3204F25E
:1062C000544084F8A83201F0FBFC94F93D32642B71
:1062D00030D1652304A904F23D208DF8103049F037
:1062E00099FD04A9204647F035FE18B304238DF824
:1062F00018300023CDE9013303930F23059369463A
:1063000004A847F0A9FF059B28B108AA009902EB51
:10631000830242F8581C0133112B0593EFD97DF00D
:106320004DF89DED031ADDED020A65219DED010A90
:106330007DF002F808B010BDD820110870B500F546
:106340002B7600F52E758CB004463146284622F097
:10635000A9FCE0B996E8070085E8070004F531716B
:1063600094EDB01AD4EDAF0A02AD94EDAE0A084632
:1063700001911FF059FA019902A81FF07DF904F567
:106380003A740FCD0FC40FCD0FC42B6823600CB02F
:1063900070BD000084B000F54E7004B01FF080B8EE
:1063A00084B000F54E7004B01FF0A8B813B50446D1
:1063B00000F5097140F2751201A819F067FB04F2AB
:1063C000544001F071FE204627F0E8FB01A819F0C7
:1063D0007FFB02B010BD0000F8B54B6801F110065C
:1063E00007460C46C0F8103200F54E758B68C0F8B1
:1063F0001432CB68C0F818320FCE0FC50FCE0FC5C0
:1064000004F1440233682B6007F54B7307CA83E835
:10641000070004F1500207F5577307CA83E8070025
:1064200004F15C0207F55A73683407CA83E8070071
:1064300007F55D7394E8070083E80700384601F02C
:1064400097FD3846BDE8F84001F07ABD13B5044623
:1064500000F25440019003F0B3FA04F5C4610198CE
:10646000009102F059FE0099204602B0BDE81040AC
:10647000FFF7B2BF4A78064BC2F340121A754A784A
:10648000C2F380125A750A78C2F300129A757047E7
:106490008D8F003013B5044600F5097140F24D327E
:1064A00001A819F0F3FA002104F2544002F02AF88E
:1064B00094F8783223B1204628F016FA84F878024E
:1064C00001A819F005FB02B010BD000038B590F826
:1064D000243305460C462BB1032B0BD095F88032A4
:1064E000DB070CD405F2AC630FCB84E80F0095F802
:1064F000BC0603E027F0D4FB0028EFD038BD002015
:10650000FCE7000000F2544090ED3B0A70470000A9
:1065100000F2544090ED3C0A7047000010B490F82F
:1065200024230C462AB1032A0AD000205DF8044B2C
:10653000704700F5BB6007C884E807000120F5E755
:106540005DF8044B27F068BB90F89C03431E58424B
:106550005841704738B590F824330D468BB900F296
:10656000544001F009FE044610B90024204638BD0D
:1065700001F056FDD5ED007A27EE800A85ED000A80
:10658000F4E7D0EDE67AC1ED007A90F89443002C60
:10659000EBD090EDE47ADFED076AB4EEE67AF7EE41
:1065A000006AF1EE10FA27FE267A67EE877AC1EDCF
:1065B000007ADBE70000003490F82433032B01D18C
:1065C00027F0A6BA0020704790F82423032A01D1AF
:1065D00027F070BC00F2544002F0E6B930B5054631
:1065E00085B00C469AB1032A1BD005F52B7022F01A
:1065F00093FB01A920468DED010ACDED020A8DED38
:10660000031A21F031FC0123184605B030BD90F883
:106610002036002BF8D000F254630FCB84E80F0033
:10662000E3E790F87832002BEED027F00DFCDCE7A2
:1066300090F82423FFF7D2BF7FB590F8242332B11E
:10664000032A4FF0000309D0039304930CE000F2F7
:10665000544007B05DF804EB01F0D8BD03A90393E3
:106660000493059327F04AFA9DED030ADDED040A31
:1066700007B05DF804FB000037B504460D4640F254
:10668000C75200F5097101A819F000FA2046294601
:1066900027F030FB94F82433032B0CBF044600246E
:1066A00001A819F015FA204603B030BD10B52DED44
:1066B000028BB0F8C03682B004461B0730D5D0F844
:1066C000383401A99FED188A00F5157007EE903A4D
:1066D000B8EEE77A27EE087A8DED017A49F048FBAB
:1066E000D4F83C3401A904F5167007EE903AF8EEA0
:1066F000E77A67EE887ACDED017A49F039FBD4F874
:10670000343401A99FED097A04F5177007EE903A29
:10671000F8EEE77A67EE877ACDED017A49F028FB4B
:1067200002B0BDEC028B10BD95BFD6330AD7233C17
:1067300027F014BB90F82403003818BF01207047DD
:1067400038B590F824230C46032A04D1012527F0FC
:10675000D5F9284638BD90F8A056002DF9D000F2A2
:10676000946393E8070084E80700F2E710B590F817
:10677000242303460C461AB1032A0BD0002010BD77
:1067800090F8A8060028FAD003F5C463D3F8843043
:106790000B60F4E727F0C8F9012084ED000AEEE76A
:1067A00090F82433032B01D127F00EBB0020704753
:1067B00030B590F8243387B005460C4623B1032B3F
:1067C00009D0002007B030BD00F2544007B0BDE84A
:1067D000304002F095BB0022002302A9CDE902233C
:1067E000CDE9042327F072F90028EAD0694628464B
:1067F00027F078F90028E4D0DDE90223C4E900237A
:10680000DDE90423C4E90223DDE90023C4E904230C
:10681000D8E7000010B586B0002200230C46694678
:10682000CDE90023CDE90223CDE90423FFF7C0FF22
:1068300088B19DED027B9DED005BF7EEC76BB7EE77
:10684000C55B9DED047B84ED005AC4ED016AB7EE93
:10685000C77B84ED027A06B010BD000090F82423B7
:106860001AB1032A05D00020704700F2544002F00C
:1068700083BB27F02BB900001FB5002200230C4674
:106880006946CDE90023CDE90223FFF7E7FF58B1C0
:106890009DED027B9DED006BB7EEC77BB7EEC66B3F
:1068A00084ED017A84ED006A04B010BD90F82423D1
:1068B0001AB1032A05D00020704700F2544002F0BC
:1068C00045BB27F00FB9000013B50C466946FFF72A
:1068D000EDFF28B19DED007BB7EEC77B84ED007A1C
:1068E00002B010BD90F93E323BB990F8803213F0FF
:1068F000010F14BF032000207047032070470000E1
:10690000F7B50446FFF7EEFF0546002862D00328DE
:1069100039D194F878326BB394F88032D8072BD5FC
:1069200001A9204627F0CEFBBDF80430002B18BF8C
:10693000002594F8206206F0FD06012E4AD10023BE
:10694000032D019307D101A9204627F0C7FB20465C
:1069500027F0E0FA064604F2544002F023FC08B99E
:1069600094F821039DF80430D90703D55A0701D5BF
:106970009F0632D400252DE0204627F009F8002894
:1069800008BF0025D5E70025D3E713F0020F2EE05E
:1069900094F9503223B99DF80430DB092FD0E9E790
:1069A000002EF8D00FF07EFEFFF7D2FA022807D9AA
:1069B0009DF805309806DDD59DF80430D906D9D567
:1069C000FB6A93F89C30002BE5D118E0DA0601D47D
:1069D0001B0718D5284603B0F0BD0028FAD094F85C
:1069E0002123B4F9C036002ACFD013F0010FF1D122
:1069F000154B1F68FB6A93F89C30002BC8D19DF89B
:106A000004309C07E2D406F08DFB06F087FA0028DC
:106A1000B0D10FF047FEFFF79BFA0228AAD90FF07A
:106A200041FEB02290F80C33F0EE007A02FB030036
:106A300090ED417AB4EEE77AF1EE10FA9AD59DF82E
:106A40000530DB09C6D195E7088E00302DE9F04707
:106A500090F8783292B00446002B00F093802046E4
:106A600027F0B2FC2046FFF74BFF03287AD104F54C
:106A70004E78002720464FF00C0A414600970197B8
:106A8000029727F0B7F96946204627F0A9F9009B3D
:106A90002046C4F81032019BC4F81432029BC4F89B
:106AA000183201F065FA204601F04AFA1CF0DEFCCB
:106AB0000546204626F0FCFF002803AA4FF0FF31D0
:106AC000AEBFC6B295F8049995F805692046A8BFEF
:106AD000B14603970497059727F034F803A804F507
:106AE0005D7722F019F90AFB09500AFB065504F5F7
:106AF000577184EDD70A00F5DC60C4EDD80A05F5BE
:106B00005F7584EDD91A06AE22F016F93A4684ED87
:106B1000CB0A4FF0FF31C4EDCC0A204684EDCD1AEC
:106B200027F024F895E8070086E807003946304644
:106B300022F068F904F53172414609A81EF02EFDD5
:106B4000314609A81EF0ACFC09A9204684EDDA0AFA
:106B5000C4EDDB0A84EDDC1A27F0C0FA09A920464F
:106B6000FFF788FC94F8C236002B3AD109A804F04C
:106B700083FF09A9204627F09FF890B3012384F8EA
:106B8000C2362EE0D0F87C321BB983F00DFCC4F87D
:106B90007C02154B1B68D86A03685B68984788B10C
:106BA00083F002FCD4F87C32C01AB4F87A329842EE
:106BB00004D9204627F098FE84F8780294F87832B9
:106BC0007BB14CE783F0F0FBD4F87C32C01A41F281
:106BD00087339842E4D84DF097FE4DF0CFFC002863
:106BE000DED112B0BDE8F087088E003090F8243373
:106BF00023B1032B4FF0000007D0704790F93E22DD
:106C0000032A04D10A70012070470870FBE7184678
:106C10007047000073B50D460DF107010446FFF7FC
:106C2000E5FF064628B19DF807302BB1032B09D0AC
:106C30000026304602B070BD04F2AC630FCB85E88D
:106C40000F00F6E72946204627F02AF894F87862E4
:106C5000EFE7000037B50D460DF107010446FFF7D9
:106C6000C5FF28B19DF8072029462046FFF7B6FC4E
:106C700003B030BD37B50D460DF107010446FFF7EF
:106C8000B5FF28B19DF8073023B1032B11D00020A8
:106C900003B030BD04F224631B682B6004F5C563A8
:106CA0001B686B6004F22C631B68AB6094F82006D1
:106CB000EEE72046294627F093F894F87802E7E7B4
:106CC00010B50446FFF70EFE18B1032807D00020C8
:106CD00010BD04F25440BDE8104001F021BA94F810
:106CE0007832002BF3D0204626F052FE0028EED05A
:106CF00094F8203203F0FD03012BE9D194F824032A
:106D0000C31E58425841E3E710B50446FFF7EAFDB9
:106D100080B1032810D194F8780250B183F044FB7D
:106D2000D4F87C32C01A44F62063984294BF002005
:106D3000012010BD0120FCE70020FAE708B502465B
:106D4000FFF7D0FD032804D1104627F0C7F9012032
:106D500008BD0020FCE7000013B50C4601A9FFF7B1
:106D6000EDFF20B1019B1C4214BF0120002002B0A6
:106D700010BD000030B585B00446019102F032FF2D
:106D80000199054610B9002005B030BD019102F00F
:106D9000F9FE01990028F6D0284602F0F7FE0028F7
:106DA000F1D0B4F8C0365907EED494F82133002B53
:106DB000EAD00B4A1268D26A92F89C506DB103A9CE
:106DC0002046FFF7BBFF30B19DF80E309A07DBD5A8
:106DD000C3F38000D8E72846D6E71846D4E700BFBB
:106DE000088E003010B4BDF8044001945DF8044BE7
:106DF00027F008B910B4BDF8044001945DF8044BC5
:106E000027F09CB827F0D4B890F840245AB100F28B
:106E100034439FED057AD3ED007AF8EEE77AA7EEDA
:106E2000C70A27F029B970470AD7233C10B5044692
:106E3000FFF758FD032804D12046BDE8104026F096
:106E400003BF002010BD00002DE9F04190F824336D
:106E50008CB000270646032B0C4615460097019779
:106E6000029719D126F024FE6A4680464FF0FF3182
:106E7000304626F07BFEB8F1FF3FA76067602760D1
:106E80000DD11CF0F3FA2B46224690F805191BF0A1
:106E900065F80CB0BDE8F0814FF0FF38EBE71CF06F
:106EA000E5FA2B4622465FFA88F11BF057F895ED7C
:106EB000000A684621F06CFF03A920468DED051AF3
:106EC0008DED030ACDED040A21F09CFF06F5317229
:106ED00006F54E7103A81EF061FB214603A81EF0C3
:106EE000DFFADFED077A84ED021A84ED000AC4EDC3
:106EF000010A95ED007AA7EE271A84ED021AC8E779
:106F00000AE81C41DFED0B7A20EE270A1FB50C467C
:106F10001946094BBDEEC00A1868084B8DED020AF0
:106F2000CDE900429DF81820C06A18F0B1FF04B006
:106F300010BD00BFE02E6542088E0030EC20110825
:106F40002DE9F0472DED028B92B000254FF07E5ACF
:106F500004460F4600F54E7106A89046CDF818A0DD
:106F600009950895079520F03FFA06F0DBF805F043
:106F7000D5FF81462046FFF7B5FC032803D094F8DF
:106F80002433032B4FD100269FED548ADFED548A22
:106F90002379F2B2934247D90AAA71B22046CDF8BA
:106FA00028A00D950C950B9526F02EFF0AA906A892
:106FB00020F08AFFB4EEC80AF1EE10FA0DDD3B4670
:106FC000484ACDF8008048492046FFF79BFF002043
:106FD00012B0BDEC028BBDE8F0870AA906A80395A4
:106FE0000495059520F05AFF03A90EA88DED0E0A11
:106FF000CDED0F0A8DED101ACDED111A20F0C2FC67
:10700000B9F1000F0DD09DED050AB0EEC00AB4EE47
:10701000E80AF1EE10FA04DD3B46344ACDF8008070
:10702000D1E70136B4E7002394F8806216F001003E
:1070300001D0012BCCD104F5C6610AA8CDF828A057
:107040000D950C950B9520F0CFF90AA906A820F014
:107050003BFFDFED227AB4EEE70AF1EE10FA05DD30
:107060003B46204ACDF800802149ADE72046FFF796
:1070700039FC03282DD1204626F028FF94F88032D1
:10708000DB0728D438BB0AA906A803950495059503
:1070900020F004FF03A90EA88DED0E0ACDED0F0A16
:1070A0008DED101ACDED111A20F06CFCB9F1000F26
:1070B00011D09DED050ADFED0A7AB0EEC00AB4EEFC
:1070C000E70AF1EE10FA06DD3B46084ACDF80080EB
:1070D000CAE70020D2E701207AE700BFC2B8323EFB
:1070E000C2B8B23E1821110823211108FFD210089E
:1070F000282111082DE9F7431546044688460193D7
:10710000FFF7DEFD019A074638B928482946284B83
:107110000068C06A18F0BCFE019A29462046019218
:10712000FFF70EFF064668B32046FFF7DBFB94F936
:107130003E1243B2019A994207D01E4B1B48294682
:107140000068C06A18F0A4FE1CE094F8243383425F
:1071500007D0019205F0E6FF05F0E0FE019A002855
:10716000EBD12046FFF7BEFB18B103280FD0124B1E
:10717000E4E7134641462A4604F2544000F0E4FF97
:1071800000B107B90026304603B0BDE8F08394F89B
:107190007892B9F1000F01D1084BCFE71346414671
:1071A0002A46204626F004FCEAE700BF088E00309D
:1071B0002C211108382111086821110857211108C4
:1071C00090F82433032B01D126F09EBF0020704796
:1071D00013B5044600F5097140F6783201A818F09D
:1071E00055FC204626F0F4FC01A818F071FC02B012
:1071F00010BD000008B50246FFF774FB10B103286C
:1072000006D008BD02F25440BDE8084000F05CBF63
:107210001046BDE8084026F06DBF00000B46114641
:1072200010B42BB1032B09D000205DF8044B70473C
:1072300000F254405DF8044B00F052BF5DF8044B7F
:1072400026F03ABD13B504460A46FFF74BFB01464C
:1072500020460192FFF7E2FF70B9084B019A1B68C4
:10726000DB6A93F89C0038B194F82413204602B0EE
:10727000BDE81040FFF7D2BF02B010BD088E00304D
:1072800070B590F8943286B004460D46DB070CD4F6
:1072900003F0BCFB5022437C02FB0300D0ED0B7AD1
:1072A000F1EE677AC5ED007A41E002A804F0E4FB54
:1072B00069462046FFF7FAFAE8B90FF0F3F994F9B6
:1072C00050320646022BE3D1FEF742FE0228DFD9F8
:1072D000B02396F80C039FED177A03FB0066D4F8F1
:1072E0008832D6F8F8209B1A07EE903AF8EEE77A43
:1072F00067EE877AD6E702A92046FFF7A3FF0028AA
:10730000DBD0D4F88822039BDFED0A7A9B1A07EEC4
:10731000103AB8EEC77A9DED006B27EE277AB7EEEC
:10732000C77A36EE477BB7EEC77B85ED007A06B0AD
:1073300070BD00BF0AD7233CF0B587B00C460646A7
:1073400000F5097140F6DD3201A818F09FFBA36833
:1073500053B9E36843B9636833B9002701A818F04B
:10736000B7FB384607B0F0BD204604F0A7FC002864
:10737000F3D002AD94E80F0085E80F000021284605
:1073800004F058FC07460028E7D096F89432DB0753
:1073900004D44DF0B9FA19214DF046F806F5217CD8
:1073A00095E80F008CE80F0096F89432304643F0D1
:1073B000010386F8943200F013FE58F027FF4621AF
:1073C0005AF088FB58F022FF45215AF083FB084B06
:1073D000A2681B68DB6A1A61E2685A6162689A6196
:1073E00025F048F80028B9D022F06CFCB6E700BFC1
:1073F000088E003038B5144B04461B68DD6A2B68D4
:1074000028465B689847F0B12B690BB96A69D2B11D
:10741000C4F88C3200226B6904F52170C4F89032F4
:10742000A96904F02DFB94F8943223F0030343F090
:10743000030384F8943258F0E9FE044A0621BDE8BB
:10744000384052F0BDBF38BD088E00307C21110895
:1074500013B504460193FFF745FA0328019B05D1B4
:10746000204602B0BDE8104026F0F8BC002002B073
:1074700010BD000010B588B004460593FFF732FA3E
:107480000328059B4FF000000AD10690079006A83C
:1074900002900B9801900A980090204626F0ECFC90
:1074A00008B010BD13B504460193FFF71BFA03287B
:1074B000019B05D1204602B0BDE8104026F0EABC91
:1074C000002002B010BD000038B5044602F08AFB6F
:1074D0000546D0B194F82433032B03D095F84E41E0
:1074E000204638BD204626F0A3FBFF280446F5D0F1
:1074F0000146284602F04AFB0028EFD021462846E4
:1075000002F040FB0028E9D0EAE70446E8E7000083
:1075100008B590F82433032B05D01BF0A7FF90F992
:107520000409C0B208BD26F0C3FA431CF9D1F4E740
:1075300008B590F8243383B1032B03D1BDE808408C
:1075400026F0AEBA4BF086FA40F64C524FF480115A
:107550004BF038FA4FF0FF3008BD1846FCE700004A
:10756000FFF7D6BF90F82433032B01D127F096B84C
:107570007047000090F82433032B01D126F088B91E
:107580007047000026F0ECB926F004BB10B50446A5
:1075900029F09EFD2046FEF757FB2046BDE810402F
:1075A000FEF76EBC90F824330BB1032B01D126F00B
:1075B00099BC00207047000090F824231AB1032AD8
:1075C00007D00120704790F95002003818BF012001
:1075D000704726F093BC000010B590F840348AB094
:1075E0000446002B62D1B0F8C036DB065ED590EDC4
:1075F000957ADFED2F7AB0EEC77AB4EEE77AF1EE46
:1076000010FA11D590ED967AB0EEC77AB4EEE77A1B
:10761000F1EE10FA08D590ED977AB0EEC77AB4EE95
:10762000E77AF1EE10FA41D42046FFF7C5FF0028B3
:107630003CD1D4ED976ADFED1F7A9FED1F6A66EEAD
:10764000A76A94ED967AD4ED957A27EE067A0090A3
:1076500067EE867A06A8FDEEE66ABDEEC77AFDEE15
:10766000E77A16EE903A17EE102A17EE901A04F009
:1076700021FA06A92046FEF7FFFFB8B158F0C6FD73
:1076800094ED977A0D4A0621B7EEC77A8DED047B0B
:1076900094ED967AB7EEC77A8DED027B94ED957AEC
:1076A000B7EEC77A8DED007B52F08AFE0AB010BDAE
:1076B000000000340000C8428096184B9421110845
:1076C00090F824330BB1032B01D127F04FB80020E1
:1076D0007047000000F57B7330B504460D460FCBB4
:1076E00085E80F0094F8FC0330BD00007FB5064626
:1076F00068460D4604F0C0F996F89432DB0703D4CF
:107700000024204604B070BD69463046FFF7E2FF12
:1077100004460028F4D0694606F5217004F0BAFB4F
:1077200085ED000AC5ED010A85ED021AE9E70000C2
:1077300000F56072034610B50C4607CA84E80700DE
:1077400093F88C0310BD000000B52DED028B85B0C1
:10775000B0EE408A9FED120A01A98DED010A8DED70
:10776000020A8DED030AFFF7E3FFA0B1DDED010A88
:107770009DED020AF1EE600AB1EE400ADEF058FC1F
:10778000DFED087AA8EE670A05B0BDEC028B5DF864
:1077900004EBDDF075BC05B0BDEC028B5DF804FBBD
:1077A0000000000035FA8E3C10B52DED028B90EDF7
:1077B000800A0446FFF7C8FFB0EE408A04F5607007
:1077C00021F066F920EE080ABDEC028B10BD000026
:1077D000D0F898330B6090F894037047D0F8A0333A
:1077E0000B6090F89D03704700F56972034610B571
:1077F0000C4607CA84E8070093F8B00310BD0000E8
:1078000000F56D7330B504460D460FCB85E80F00CB
:1078100094F8C40330BD000000F5866330B504461B
:107820000D460FCB85E80F0094F8400430BD0000F2
:1078300000F24442034610B50C4607CA84E807002C
:1078400093F8500410BD00002DE9F04305460E46A4
:1078500017462DED028B8BB0FFF736FE01468046B2
:107860002846FFF787FA0446002846D002F0BAF906
:10787000414602F08DF986ED000A95F93C32002B65
:1078800038DD0EF00FFFFEF763FB012832D90EF052
:1078900009FFB02290F80C33B7EE008AD5EDE47AF8
:1078A000DFED598A02FB030095F93C32F4EEE87AE9
:1078B000D0ED410A07EE103A96ED000A40F20E4074
:1078C000F1EE10FAB8EEC77A67FE887A20EE270A42
:1078D00037EE201A70EEC70A1DF0D8FAD5EDE47A1B
:1078E000F4EEE87AF1EE10FA67FE887A80EE277AF5
:1078F00086ED007A01233B7003E095F8203333B91D
:10790000387020460BB0BDEC028BBDE8F0834FF021
:10791000000995F82433CDF80490CDF80890CDF8FF
:107920000C9043B1032B10D0CDF81090CDF81490EB
:10793000CDF818907CB902233246414605F25440F6
:107940003B7001F073FB0446DBE701A9284626F0F3
:1079500063F90446E8E795F82433002BEBD004A93B
:107960002846FFF765FF04460028E4D001A904A8D3
:1079700021F0F8F907A8CDED080A8DED091A8DED73
:10798000070A21F023FE04A8B0EE408A21F01EFE73
:1079900095F93C32002B2EDD07EE903A40F2544030
:1079A000F8EEE77A70EE670A37EE801AB0EE480A12
:1079B000F5EEC00AF1EE10FA48BFDFED140AF4EE5E
:1079C000410AF1EE10FA30FE811A1DF05FFAB0EEB6
:1079D000408AD5EDE47A03239FED0B7AF4EEC77A63
:1079E000B7EE007AF1EE10FA67FE877A88EE277A12
:1079F00086ED007A7FE7B5EEC08AF1EE10FA48BF57
:107A00009FED028AE5E700BF00000034000000009F
:107A100038B50446FFF77CFD054694F826338342CB
:107A200004D01BF023FD29461AF052F92046FFF737
:107A30006FFD84F8265384F825032046FFF768FD80
:107A400084F827032046FFF773FD04F5607184F87E
:107A500028032046FEF762FD84F88C0300F0E0FA6C
:107A600004F5677284EDE40A04F566712046FFF7B9
:107A7000EBFE04F5687184F894032046FEF76AFD76
:107A800004F5697184F89D032046FEF795FD04F521
:107A90006D7184F8B0032046FEF7CAFD04F57271DB
:107AA00084F8C4032046FFF7E5F804F5767184F8FE
:107AB000D4032046FFF7CEF804F57B7184F8E80381
:107AC0002046FEF703FD04F5806184F8FC032046A0
:107AD000FFF7A0F884F810042046FEF7ADFD04F28D
:107AE000144004F5836380ED000AC3ED000A20F022
:107AF000CFFF04F21C4304F58461204604F22C42BB
:107B000083ED000AFFF7A0F904F586612046FFF730
:107B100099FB80B194F840349BB90123204684F846
:107B2000403400F05DFA58F071FB452159F0D2FF66
:107B30002046FEF7BBFD94F8403413B92046FFF70A
:107B40004BFD04F244412046FEF7FAFD84F8500450
:107B500038BD000037B50D46044600F0F5F81DB9F4
:107B60001BF084FC1AF024FB4FF4EA7204F509714F
:107B700001A817F08BFF94F881322BB92046FFF74C
:107B800039FC012384F88132224B1D68A86A0368FE
:107B90009B6998472046FEF7D1FB2046FEF756FC2E
:107BA000204600F059FA2046FEF750FF286B30B10E
:107BB0000368D4EDD80ADB6894EDD70A9847D4F867
:107BC0001C0208B1A3F0C0FD204600F079F8204661
:107BD000FEF796FE94F8A83284F8240383420ED070
:107BE00084F8A80298B10C4D0C4B032808BF1D4621
:107BF00058F00CFB2B460A4A062152F0E1FB2046C6
:107C0000FFF706FF01A817F063FF03B030BD054D75
:107C1000EEE700BF088E003059ED1008232111084F
:107C2000C021110828211108D0EDE47AB7EE000A2E
:107C30009FED047AF4EEC77AF1EE10FA27FE800A7F
:107C4000704700BF00000034D0EDE47AB7EE000AC0
:107C50009FED067AF4EEC77AF1EE10FA67FE807AAD
:107C600067EEA77A80EE270A704700BF0000003455
:107C7000014B1868704700BF288E00307047000025
:107C800070470000704700000020704700207047D8
:107C90000120704703681B6E1847000000207047E2
:107CA0000020704700207047002070477047000098
:107CB0000020704700207047002070477047000088
:107CC0007047000008B51BF0D1FB90F8040908BD0F
:107CD00030B59FED1B1A0C46DFED1A0A05462D2024
:107CE0002DED028B87B091ED000A8DED011ACDEDDF
:107CF000000A1DF0CBF89DED011AF0EE408ADDED93
:107D0000000A2E2094ED010A1DF0C0F89DED011A25
:107D1000B0EE408ADDED000A2F2094ED020A1DF03E
:107D2000B5F803A905F52B70CDED038A8DED048A16
:107D30008DED050A48F05CF907B0BDEC028B30BD53
:107D4000C2B8323EC2B832BE10B5044682F02CFB37
:107D5000D4F80C331BB1C21AB2F57A7F12D30A4A97
:107D60001268D26A92F89C2002B15BB9C4F80C0385
:107D700094F83D421BF07AFB80F8F74805F0D2F901
:107D800080F8294010BD00BF088E00302DE9F04377
:107D90002DED028B87B091ED007AD1ED037A0C4680
:107DA0008DED047AB0EEC77A15461E46DDF84C908C
:107DB000B5EEC07ACDED057ADDE91087F1EE10FA67
:107DC00006DCF0EEE77AF5EEC07AF1EE10FA02DDAD
:107DD00004A820F0D1FEB7EE001A6B20FFEE000AD7
:107DE0009DED050A1DF052F8B7EE001AFFEE000AED
:107DF0006C2089ED000AB7EE008A9DED040A1DF0A3
:107E000045F804A888ED000A20F026FE002852D08C
:107E10000023C9F8003088ED008AD4ED067A67EEB9
:107E2000A77AF4EEC87AF1EE10FA4ADB0023336049
:107E300085ED008AB7EE001A7C20DFED3E0A96ED54
:107E4000000A1DF023F8B7EE001A86ED000AFFEED7
:107E5000000A7D2095ED000A1DF018F885ED000A56
:107E6000D4ED067A129BF1EE677ADFED336AC3ED4B
:107E7000007A96ED007AF0EEC77AF4EEE67AF1EE4B
:107E800010FA2BD503AB02AA01A920461DF02CFD48
:107E90009DED018AB0EE480ADDF0F2F885ED000AAA
:107EA000B0EE480ADDF0F2FE87ED000A07B0BDEC47
:107EB000028BBDE8F08304A820F0BAFD0028A7D10A
:107EC000ABE738EE670A1CF005FF86ED000A94ED7B
:107ED000087AC7EE007AC5ED007AABE794ED076A41
:107EE000C6EE077AC7ED007A96ED007AB0EEC77A53
:107EF000B4EEE67AF1EE10FAC4D495ED007ADFED37
:107F00000F6AB0EEC76AB4EE666AF1EE10FAB9DC39
:107F1000B4EE477AF1EE10FAB4D6B0EEE77AB4EEEA
:107F2000667AF1EE10FAADDCF4EE677AF1EE10FA53
:107F3000BCD7A7E70000000000000034FFFF7F7FF0
:107F40001FB500F51D7300F5187200F54E7103930F
:107F500000F51C73029300F51B73019300F51A736F
:107F6000009300F51973FFF711FF05B05DF804FBEE
:107F70009FED196AD0ED846ADFED187A66EE866AA5
:107F800090ED860A20EE060A26EEA77AC0ED7E6AFC
:107F900010B5BDEEC77A044680ED817A90ED857A02
:107FA00027EE067A67EE275A80ED7F7A60EE277A11
:107FB000FDEEE55AFDEEE77AC0ED825A17EE903AF3
:107FC000002BBCBF03F50C43A033C0F80C321CF0EF
:107FD000B9FE84ED800A10BDE02E65420000C84263
:107FE0001FB50E4B04461B68B3B1684603F044FD51
:107FF00069462046FFF710FC20B16A460021204662
:10800000FDF708FF94F89432DB0705D504F52172DB
:1080100001212046FDF7FEFE04B010BDB4920030F1
:1080200008B502F0F3FCBDE8084001F017BF0000FE
:108030007FB51BF01BFA90F8051907B05DF804EB4B
:108040001AF060B810B5044680F8101382F0ACF94D
:10805000C4F8140310BD000010B590F810330446A6
:1080600053B182F0A1F9D4F81433C01AB0F57A7F75
:1080700084BF002384F8103394F8183353B182F08E
:1080800093F9D4F81C33C01AB0F57A7F84BF00236B
:1080900084F8183310BD000000F5C2700B4607C805
:1080A00083E80700012070470023C0F89C30C0F827
:1080B0009830C0F89430C0F8A830C0F8A430C0F8A8
:1080C000A030C0F8AC30704770470000024B0B6026
:1080D0004FF07C5313607047000048427047000027
:1080E00000F5CC7010B50C460FC884E80F00204690
:1080F00003F0B6FC30B1FFF7BBFD00F521700FC8EF
:1081000084E80F00204603F0ABFC80F00100C0B211
:1081100010BD000010B5044604F014F9204610BD4F
:1081200010B5D0F8903104465BB182F03DF9D4F837
:108130009031C01A41F28833984294BF0020012048
:1081400010BD0120FCE7000013B500930368019205
:10815000DB6D98470446DDE9002128B90448054B4A
:108160000068C06A17F094FE204602B010BD00BF40
:10817000088E00302C21110813B50446019101F03E
:1081800031FD019A23680146DB6B08B190F84E116E
:10819000204602B0BDE810401847000090ED007A7C
:1081A000DFED0F7AB0EEC77AB4EEE77AF1EE10FAAF
:1081B00014D590ED017AB0EEC77AB4EEE77AF1EE1D
:1081C00010FA0BD590ED027AB0EEC77AB4EEE77AEA
:1081D000F1EE10FA4CBF01200020704700207047DC
:1081E0000000003410B501F0FDFC044658B190F8D1
:1081F0004E1101F0C7FC30B194F84E112046BDE895
:10820000104001F0C3BC002010BD00002DE9F04378
:10821000002504462DED028B8FB0036802A99B6BED
:10822000039504950595069502959847064638B13D
:10823000FFF7F6FEDDED027A27EE800A8DED020AE9
:108240000EF030FAFDF784FE0746002E50D0DDED2B
:10825000027A0BA9D4ED706A204694ED717A2368F6
:1082600027EE877A0B9567EEA67A0C950D9509ADEA
:108270008DED097ACDED0A7A5B6B98470BA92846FC
:1082800020F04EFB012F8DED030ACDED040A40F2E4
:10829000B3800EF007FAB02590F80C33DFED5A7A70
:1082A00005FB030090ED428A28EE278AB0EE480ACB
:1082B000DCF0E6FEF0EE408AB0EE480ADDF0E6FCC7
:1082C0008DED0C0ACDED0B8A0EF0ECF990F80C3325
:1082D00005FB030009AD90ED410A0BA820F040FB1F
:1082E00005A88DED050ACDED060A96BB03C885E00D
:1082F0000128CED89DED020AB5EEC00AF1EE10FAC3
:108300007FDD07AED4F8C421D4F8C03130460792DF
:10831000089320F04FFB23680BA90B9520460C9582
:108320000D955B6B9847DDED077A9DED0B7A09ABF8
:1083300077EE877A9DED0C7ACDED077ADDED087A40
:1083400077EE877ACDED087A96E8030083E803009C
:1083500049E02369B7EE008A04F5D47904F5DC76A8
:1083600093ED000A03AF04F5D87838EE408A20F088
:10837000F7FA8DED090A4846CDED0A0AB0EE480A33
:1083800020F0EEFA0BA92846CDED0C0A8DED0B0A74
:1083900020F0C6FA3146C4ED6B0A384684ED6A0A0D
:1083A00020F0CEFA8DED090AB0EE480A4046CDED38
:1083B0000A0A20F0D5FA0BA928468DED0B0ACDED5F
:1083C0000C0A20F0ADFA84ED6C0AC4ED6D0A97E852
:1083D000030086E803004946404620F0A1FA8DEDEF
:1083E000090ACDED0A0A9DED090ADDED0A0A0FB072
:1083F000BDEC028BBDE8F083DDE9030185E80300F5
:10840000F1E709950A95EEE735FA8E3C10B590F83C
:108410004613044604F096F97C23C0B203FB0044E3
:10842000D4F8A40010BD0000044B026F1B68DB6A87
:108430005A60426F9A60826FDA607047088E00302F
:10844000F0B58FB004461BF011F8002302AA90F893
:10845000041902930546039304F19407049301ABB6
:1084600019F01CFDD8B39DED010AB5EEC00AF1EE7E
:1084700010FA34DD04F1B00602A820F099FC394668
:1084800084ED2C0A3046C4ED2D0A84ED2E1A20F01E
:108490009FFC04F17C01304620F04EFC04F1880181
:1084A00005A88DED050ACDED060A8DED071A20F021
:1084B00043FC08A88DED080A9DED010ACDED090ADF
:1084C0008DED0A1A20F064FC0BA904F128008DED53
:1084D0000B0ACDED0C0A8DED0D1A1DF027FA95F85B
:1084E00004090C23394603FB005000F5DC6020F042
:1084F00023FC84ED2C0AC4ED2D0A84ED2E1A0FB056
:10850000F0BD00007B4B2DE9F04700251F680446B5
:108510000E462DED028BC0F89C508AB0C0F89850E2
:1085200004F12809C0F89450C0F88450C0F8805075
:10853000C567C0F89050C0F88C50C0F88850C0F89B
:10854000B850C0F8B450C0F8B050F86A03685B681F
:10855000984700284CD081F027FF42F20F739842D1
:1085600046D8FB6A484693ED010A84ED1C0AD3ED18
:10857000020AC4ED1D0A93ED031A84ED1E1A1DF0C4
:1085800053F957F043FEDFED5C7A94ED1E6A062145
:1085900094ED1C7A26EE276A584A27EE277AB7EE22
:1085A000C66A8DED046B94ED1D6A26EE276AB7EE60
:1085B000C77AB7EEC66A8DED007B8DED026B51F088
:1085C000FFFE94ED1E8AB0EE480ADCF059FD84ED02
:1085D000710AB0EE480ADDF059FB84ED700A81F0B3
:1085E000E3FEC4F894010AB0BDEC028BBDE8F0874D
:1085F000A6B194ED1C0AB4EE400AF1EE10FA0DD6C5
:10860000D4ED1D0AF4EE600AF1EE10FA06D694EDF0
:108610001E1AB4EE411AF1EE10FA67D71AF026FFCF
:108620004FF00C0A90F80539B2EE028AF2EE068A93
:1086300007460AFB030307AE4FF0150803F55F7307
:1086400093E8070086E80700304620F0BFFFB4EE4D
:10865000C80AF1EE10FA11D508F1FF3818F0FF083A
:1086600015D1304620F0B2FFF1EE047AB4EEE70AFD
:10867000F1EE10FA1CDC2567656731E0304620F02A
:10868000A5FFB4EEE80AF1EE10FAE5DCE9E73846BA
:1086900019F022FB384619F08BFD97F805390AFBD3
:1086A000037303F55F7393E8070086E80700CBE7E1
:1086B000DDED098A9DED088A68EEA80A9DED070A9E
:1086C000E8EE080AF1EEE00ADDF0B2FC84ED1D0AE6
:1086D000F1EE680AB1EE480ADDF0AAFC84ED1C0A4E
:1086E0009FED071AD4ED1D0A94ED1C0A48461DF0B3
:1086F0009BF866E7088E0030E02E654234231108AF
:10870000000000000021FFF7FDBE000037B5044661
:1087100008461546019120F059FFB7EE007AB4F8EB
:10872000E8300198C7EE007A94ED397A0133A4F865
:10873000E83037EE277A84ED397AB0EE007AF4EE3D
:10874000C77AF1EE10FA06D5B6EE007AF4EEC77AE3
:10875000F1EE10FA0DDC9FED0E7AF4EEC77AF1EE31
:1087600010FA13D59FED0B7AF4EEC77AF1EE10FAFA
:108770000CDDB0EE670A20F00BFB0120C5ED010A0D
:1087800085ED000A85ED021A03B030BD0020FBE73D
:1087900000247449BD37863570B500F1280600F114
:1087A00034050446294630462DED028BB6EE008A8C
:1087B0008AB020F069FB284620EE088AB0EE480A0D
:1087C00020F0E6FA07A93046CDED080A8DED091A2A
:1087D0008DED070A20F0C6FA8DED010AB0EE480AC9
:1087E0003046CDED020A8DED031A20F0D1FA07A92B
:1087F00028468DED070ACDED080A8DED091A20F007
:10880000B1FA04A901A88DED040ACDED050A8DED9C
:10881000061A20F04DFB324601A920468DED070ACD
:10882000CDED080A8DED091AFFF770FF58B981F0F8
:10883000BBFD0121C4F890012046FFF763FE0AB09A
:10884000BDEC028B70BD2A4604A92046FFF75EFFEF
:108850000028ECD004F1400207A92046FFF756FF9C
:108860000028E4D0EBE7000030B50D4604462DEDBE
:10887000028B284683B091F8461303F063FFC1B220
:108880007C2000FB015104F1280094311CF064FEAF
:1088900068468DED000ACDED010A20F0F9F8DFED14
:1088A0001C7AB4EEE70AF1EE10FA05D59FED190A2D
:1088B00003B0BDEC028B30BD684620F05DF9684620
:1088C00020F0CAF80028F1D194ED4E8A284604F031
:1088D000B5F9F0EE400AB0EE480A1CF08DF980B907
:1088E000284604F0ABF9B0EE408A84ED4E0ADCF085
:1088F000C7FB84ED4F0AB0EE480ADDF0C7F984EDFE
:10890000500A04F59E71684620F07EF8D0E700BF5B
:1089100000000034000000009FED0C7AB4EEC70A9E
:10892000F1EE10FA0BD4DFED0A7AB4EEE70AF1EEBD
:1089300010FA07DCC0EE077AB0EE670A7047F7EE70
:10894000007AF9E7F2EE047AF6E700BFF3665F3FDC
:1089500058A00B411C3008B520F09AF8F1EE007ACF
:10896000B4EEE70AF1EE10FA97BFF1EE027A9FED4E
:10897000050A37EEC00ADFED047A98BF20EE270A19
:1089800008BD00BFCDCCCC3DCDCC4C3E08B58369F5
:1089900093F9000038B10DF085FEFDF7D9FA0128F2
:1089A00094BF0020012008BDF8B52DED028B0546CF
:1089B00004F0B8FB04F0B2FA0446B8B3FFF758F974
:1089C00090F8213393B32846FFF7E0FF064668B3DB
:1089D0000DF068FEB02790F80C33F0EE087A07FB34
:1089E000030090ED417AB4EEE77AF1EE10FA1DD46F
:1089F00095ED1E8A0DF056FE90F80C33DFED1E7AD1
:108A000007FB030090ED420A98EE270A1CF0B0F92C
:108A1000B0EEC00ADFED197AB4EEE70AF1EE10FA13
:108A200008DC344681F0C0FCC5F880012046BDEC6E
:108A3000028BF8BD05F5C27020F0C8FDB0EE408A8B
:108A40000DF030FE90F80C339FED0D7A07FB030319
:108A5000D3ED417A67EE877AB4EEE78AF1EE10FA49
:108A6000DFD581F0A1FCD5F88041001BB0F5FA6F8D
:108A70008CBF00240124D9E7E02E65420000344277
:108A8000CDCC4C3F0A4B1B6810B5DB6A044693F80B
:108A90009C305BB981F088FCD4F89431C01A44F65C
:108AA0001F6398428CBF0020012010BD0020FCE70E
:108AB000088E0030F8B52DED068B04460DF0F2FD62
:108AC000054604F02FFB064606F07CFD002840F02A
:108AD000AB802046FFF768FF002800F0A8803046F2
:108AE000FFF794FCD4F8F430984200F01A81304635
:108AF000FFF78CFCD4F8F430DFED8F7AC31A3046E0
:108B000008EE903AF8EE688A68EEA78AFFF77EFCD6
:108B100094F8BC30C4F8F400F3B9304604F010FA0D
:108B2000D0B104F1280796F846233046394604F0C0
:108B300089F8D4ED1D0AB0EE401A384694ED1C0AAF
:108B40001CF072FE0023C4F89030C4F88C30C4F8D6
:108B50008830012384F8BC3020463146FFF784FE7C
:108B600095F80C03B0EE408A05EB0015D5F8B83047
:108B7000C4F8F83004F1B000D4ED129A20F026FDCC
:108B80006368DFED6E7A68EE299A93ED007AB0EEB5
:108B900040AAB4EEE77AF1EE10FA01D5C3ED007AFF
:108BA0002046B0EE4A0AFFF7B7FE636820EE299A26
:108BB00093ED000A29EE009AFFF7CCFE204629EE3D
:108BC000009A84ED249AFFF75DFF38B1B2EE007A87
:108BD000D4ED247A67EE877AC4ED247AF0EE007A39
:108BE000F4EEE78AF1EE10FA10D5DFED557AB4EE27
:108BF000E7AAF1EE10FA09D5DFED527A69EEA79AED
:108C0000D4ED2A7AE9EEA87AC4ED2A7AB0EEC88AC1
:108C10009FED4D0A94ED3C7ADFED4C7A28EE008A08
:108C2000A7EE278A84ED3C8ABDEC068BF8BDFFF7E2
:108C30001FF890F82133002B73D02046FFF7A6FED3
:108C400000286ED095F80C2305EB0213D3F8B8106A
:108C5000D4F8F8308B4264D0B026F0EE087A06FBE8
:108C6000025292ED417AB4EEE77AF1EE10FA58DB57
:108C7000CB1AC4F8F8109FED361A08EE903A95F822
:108C80000C3394ED1E0A06FB0353F8EE688ADFED01
:108C9000317AD3ED429A68EEA78A69EE819A39EE6D
:108CA000C00A1CF0C7F8B0EE409ADCF0EFFF94F871
:108CB000BC30B0EE408AF3B1F3EE047AF4EEE78A0A
:108CC000F1EE10FA17DC95F80C03F2EE027A06FBCF
:108CD000005595ED417AB4EEE77AF1EE10FAFFF621
:108CE00049AFB0EEC99ADFED1C7AB4EEE79AF1EE27
:108CF00010FAFFF63FAFB0EE691AD4ED1D0A94EDFD
:108D00001C0A04F128001CF08FFD9FED148A01233A
:108D100084ED248A84ED238A84ED228A84F8BC3091
:108D200028E7BDEC068B04F188009FED0D0ABDE835
:108D3000F84020F081B800BFBD378635CDCC4C3D22
:108D4000C2B8B23E0AD7233CCDCC4C3ECDCC4C3F32
:108D500035FA8E3C6F12833A1904863F00000000FA
:108D6000EC51783F0C2303FB010130B501F1C00346
:108D70008BB0144604AD93E8070085E8070094E83B
:108D8000070083E807002846FFF708FA07AB58B149
:108D900094E8070083E807009DED070ADDED080A67
:108DA0009DED091A0BB030BD95E80700F2E7000011
:108DB00010B52DED028BDFED0E8AB0EE408A044631
:108DC00060EEA88AB0EE680ADCF05AF920EE480A94
:108DD00084ED610AB0EE680ADCF058FF20EE480A24
:108DE0000023BDEC028B84ED620AC4F88C3110BD07
:108DF00035FA8E3CF0B52DED028BD0F848310446A3
:108E000085B00D468B60D0F84C31CB6001F0FEFD93
:108E100006460DF047FCA369074693F90030022B84
:108E200053D1FDF795F802284FD997F80C33B022AB
:108E300002FB0373D3F8F8100022284602F020FE4C
:108E400094ED561A94ED550A2846B7EEC11AB7EEBE
:108E5000C00A03F0F3F994F85C3183B39FED258ADF
:108E600081F0A2FA01AA97F80C13064638468DED58
:108E7000018A0CF04BFBD4F85001F0EE480A9FED4C
:108E80001E0AB6EE001A361A40F23C4007EE906A0F
:108E9000F8EE677A27EE800A1BF0F8FFDDED017A25
:108EA00004F5907030EE270A8DED010A1FF058FD91
:108EB0002846B7EEE01AB7EEC00A03F0BFF994F8FF
:108EC0005C0105B0BDEC028BF0BD707C502303FB50
:108ED000006696ED0B8AFEF7CBFED0EDA27A9FEDF1
:108EE000077AF8EEE77AE8EE077AFDEEE77A17EE12
:108EF000901AA1E7000000006F12833A0000C842F8
:108F000030B589B004460D46684602F0B5FD6946A5
:108F10002046FFF7E5F818B90024204609B030BD17
:108F200004A802F0A9FD204604A9FFF763FF044648
:108F30000028F1D004A9684602F0E6FF85ED000B99
:108F400085ED021B85ED042BE7E7000010B586B028
:108F5000002200230C466946CDE90023CDE9022317
:108F6000CDE90423FFF7CCFF18B1DDE90423C4E900
:108F7000002306B010BD000070B586B000220023AB
:108F80000C466D462946CDE90023CDE90223CDE903
:108F90000423FFF7B5FF064618B195E80F0084E8F3
:108FA0000F00304606B070BDF8B52DED028B0646B9
:108FB0000F46154600F016FE0446A0B1394600F0F3
:108FC000E1FD80B12046394600F0E0FD044650B195
:108FD00000F008FE394600F0DBFD85ED000A204672
:108FE000BDEC028BF8BDFEF743FE90F82033B7EEE0
:108FF000008A7BB13046FFF7C9FC044650B1D6ED7C
:109000005F8AFFF70DF8C8EE007A67EEA87AC5ED23
:10901000007AE4E7D6ED5F8AFFF702F8C8EE007A3F
:10902000002467EEA87AC5ED007AD8E770B52DED7B
:10903000048B1646FFF7B8FF054670B3FEF718FE1F
:1090400090F93C424CB30DF02DFBFCF781FF012859
:1090500023D9E4B207EE904AB8EE678A0DF022FBFE
:10906000B02290F80C3396ED009A02FB0300D0ED8D
:10907000418AFEF7D5FF40F2654029EE000A38EE3E
:10908000281A78EEC80A1BF001FFB0EE408AFEF7FE
:10909000C7FFC8EE007AC6ED007A2846BDEC048B07
:1090A00070BD000038B50D460DF0FCFA0446FCF723
:1090B0004FFF022885BF94F80C03B023002003FB68
:1090C000004081BF00F58E7007C885E807000120C9
:1090D00038BD000030B585B000230D4601A90193CD
:1090E00002930393FFF7DEFF044620B1039B2B603E
:1090F000204605B030BD01F089FC417C01F032F919
:1091000004460028F4D001F081FC00F05BFFB1EED2
:10911000400A85ED000AEBE7F8B5036F00F14C0754
:109120000C4605464B6001F11006436F8B60836F60
:10913000CB600FCF0FC60FCF0FC63B6805F12801DC
:1091400004F1340033601EF04FF92346012203F886
:10915000442B05F1B00207CA83E8070005F1940229
:1091600004F1500307CA83E8070005F11C0204F16B
:109170005C0307CA83E8070004F174012846FFF77F
:1091800091FF04F1840184F880002846FFF7A2FFD4
:1091900004F18C0184F888002846FFF72BFE84F840
:1091A0009C00F8BD08B503F0BDFFBDE8084003F022
:1091B000B5BE000010B504461FF096FE50B904F18C
:1091C0000C001FF091FE28B904F11800BDE8104012
:1091D0001FF08ABE012010BD38B500F128050446F5
:1091E0002846FFF7E7FF28B120460121BDE83840B7
:1091F000FFF788B9B7EE007AD4ED107AF4EEC77AAB
:10920000F1EE10FA06D5BFEE007AF4EEC77AF1EE71
:1092100010FA12DC2046FFF7BFFA2846FFF7CAFF14
:109220000028E1D1D4ED107AB2EE047AF0EEE77ABC
:10923000F4EEC77AF1EE10FAD6DC38BD10B504466C
:1092400020F0C4F92046BDE810401FF009BE000020
:109250002DE9F04F044600274FF0000804F1FC0B05
:1092600004F1280A2DED028BABB0B0EE408A5E46C9
:1092700009970A970B97FFF71DFC1AF0F7F80546B8
:1092800095F86D335FFA88F1032BA8BF03238B4257
:109290003AD92846019118F013FC019980B312AB1A
:1092A00015AA284615971697179718F057FE9DEDA3
:1092B000120AB5EEC00AF1EE10FA21DD15A81FF072
:1092C00077FD21A950468DED210ACDED220A8DEDC5
:1092D000231A1CF0E5F88DED180AB0EE480A18A81C
:1092E000CDED190A8DED1A1A1FF052FD21A9304655
:1092F0008DED210ACDED220A8DED231A1FF068FDB8
:1093000008F101080C36BBE70C2395F80519504607
:1093100003FB015101F55F711CF0C2F884ED070AEF
:1093200094ED4B0AC4ED080A30EE088A84ED091A60
:1093300084ED4B8A0DF0B6F90646FEF799FC90F8DD
:10934000213320460393FFF721FB80B13046FCF721
:10935000FFFD02280BD996F80C23B023616903FBAB
:10936000026391F9001093F81A01884264DA94EDCF
:109370004B7ADFED857AB4EEE77AF1EE10FA65D438
:1093800094ED5F8AFEF72EFF58B100F02BFC90F8A9
:109390004E1100F0FDFBB0EE408AFEF741FE20EEDC
:1093A000088A236CB0EE480A626B21A8A16A239355
:1093B000229221911FF0ECFC04F5C27109A88DEDF9
:1093C000090ACDED0A0A8DED0B1A1FF001FD80F0A0
:1093D000EBFF0023019084F844312046FFF7D6FAD2
:1093E00000286AD096F80C23B02101FB0262D2F863
:1093F000FC30C4F8483196F80C3301FB0363D3F812
:109400000031C4F84C3180F0CFFF0123C4F8500183
:10941000C4F85471C4F8587184F85C31D4F8303110
:10942000002B5DD1019B04F59074236109AB93E897
:10943000070084E8070009E006EB0212D2F8B82022
:1094400001920199D4F830218A4204D12BB0BDECAD
:10945000028BBDE8F08F03F58E730DF1240C93E8B9
:10946000070094F844318CE807001BB904F59073A9
:1094700083E807000123604604F5C27184F8443193
:109480001FF070FC21A904F14C008DED210ACDEDF7
:10949000220A8DED231A1CF031F8B5EEC00A8DEDCD
:1094A000210ACDED220A8DED231AF1EE10FAD8BF74
:1094B0009FED340A84ED5F0A8FE794ED4B7AD4ED8B
:1094C000557ADDED096AE6EE877ADDED0A6AC4EDCC
:1094D000557AD4ED567AE7EE267AC4ED567A9DE7B2
:1094E000D4ED4B7A244BF5EEC07A0C970D970E9382
:1094F000F1EE10FAAAD9214B9FED217A1B6867EE95
:10950000877ADB6AB7EE007A93F89C30C7EE278A39
:109510000293002B4AD094F8443113B9039B002BDB
:1095200042D0E36804F5907109A893ED008A1FF01A
:1095300019FC8DED210A21A828EE888ACDED220A9A
:109540008DED231AB0EE480A1FF022FC18A90CA8D2
:10955000CDED190A8DED180A8DED1A1A1FF038FCA1
:109560000CA8FFF76BFE0CA81FF0D8FCF0B180F040
:109570001BFFC4F8900169E7000080BF088E00302F
:109580000AE81C4100000000CDCC4C3ECDCC4C3F45
:10959000CDCC4C3D920A06BF920A063FC2B8B23EFD
:1095A000728A0E3C5B821839039B029324220021AD
:1095B00018A80DF18408DFF0E1FB2422002121A886
:1095C000DFF0DCFB4FF0000905F62B131FED138ACB
:1095D0004FF0FF37059395F86D335FFA89F1032B50
:1095E0001A46A8BF03228A427AD98B4204916BD9CA
:1095F000059B13F80930002B66D0B0EE680A584678
:109600001FF01AFC029B0499002B64D00C222AAB99
:10961000204602FB0933A3F12402069304925A4622
:10962000FFF7A0FB069B03ED090A049BC3ED010AAB
:1096300083ED021A4046FEF7B1FD002844D14046B2
:10964000FFF7FCFD40461FF069FC00283CD10C23CD
:109650000CA9404603FB09F22AAB13440792A3F17D
:109660004802069304921FF023FC069B0CA9404677
:1096700003ED120A049BC3ED010A83ED021A1FF0E9
:1096800003FC2AAB079A03EB890303ED1B0A18AB13
:1096900098181FF09BFF7A1C04D0B4EEC08AF1EE3C
:1096A00010FA03DDB0EE408A4FFA89F72AAB03EBDC
:1096B000870353ED1B7AF5EE407AF7EE007AF1EE70
:1096C00010FA48BFB0EE678A09F1010908F10C08E9
:1096D0000BF10C0B7FE79BE8070088E80700A9E780
:1096E0007B1C3FF444AF204684F83471FFF75CF9EB
:1096F00060B12046FFF74AF9002840F033812AAADA
:109700000C2303FB0723002243F8402C18AA07EB85
:10971000470895F8043902EB880895F86C239A42BB
:1097200040F23B812B4493F82839002B00F035811F
:1097300095F8053995F86D239A4240F22E812B4415
:1097400093F82B39002B00F028810C232AAA4146DC
:10975000504603FB07271BF0D1FE07ED120A47ED29
:10976000110A07ED101A40461FF0BEFB002840F01A
:10977000208140461FF0D2FB002840F01A815FEDA7
:109780007E7A04F1B00094ED3B7A28EE278A5FEDF3
:10979000817AA7EE278A84ED3B8A1FF017FFA36822
:1097A0005FED857AB0EE408A93ED007AB4EEE77A09
:1097B000F1EE10FA00F101812046B0EE480AFFF701
:1097C000ABF840461FF0E4FAA3688DED150A15A822
:1097D000CDED160A8DED171A93ED000A1FF0D8FA99
:1097E000204684ED1F0AC4ED200A84ED211AFFF7FC
:1097F00049F928B1B2EE000A04F17C001FF01CFB0D
:10980000039BB3B33046FCF7A3FB012831D996F88C
:109810000C03B023F0EE087A03FB006696ED417A64
:10982000B4EEE77AF1EE10FA23D595F805090C238A
:10983000F1EE0C7A03FB005595EDDF7AB4EEE77A92
:10984000F1EE10FA15DBD4ED1D7A1FEDAE7AF4EED1
:10985000C77AF1EE10FA0CDD1FEDB17AF4EEC77A9B
:10986000F1EE10FA05D5B6EE000A04F17C001FF007
:10987000E3FA5FEDB67AB4EEE78AF1EE10FA22D59C
:109880001FEDB90A40461FF083FA12A88DED120AA7
:1098900094ED4B0ACDED130A8DED141A1FF078FAF2
:1098A00015A904F1A0008DED150ACDED160A8DED78
:1098B000171A1FF08DFAD4ED2B7A94ED4B7A77EED0
:1098C000877AC4ED2B7AF1EE047A94ED2B7A002599
:1098D000B4EEE77AF1EE10FA3BDB19F0C7FD5FED6D
:1098E000CF7A94ED2B1A40F2C93094ED280A21EE7C
:1098F000271AF1EE410A8DED031ACDED020A1BF095
:10990000C5FA40F2CA309DED031ADDED020A84ED7E
:10991000280A94ED290A1BF0B9FA40F2CB309DEDEC
:10992000031ADDED020A84ED290A94ED2A0A1BF0E0
:10993000ADFA04F1A00104F1940084ED2A0A1FF0AD
:1099400047FAC4F8A850C4F8A450C4F8A050C4F80A
:10995000AC502422002104F1FC00DFF00FFAC4F81F
:109960002C515FE5E368F7EE000A93ED000A1BF067
:1099700043F900283FF4C3AE94ED1C0AB0EEC00AD0
:10998000DCF084F90C232AAA03FB072353ED107A99
:1099900027EE800A03ED100AB8E60C232AAA03FB7F
:1099A0000727002347F8403C47F8443C47F8483C29
:1099B000D9E62046FFF710FCD9E5C3ED007AFBE6B7
:1099C000F0B52DED108BA1B0044619F04FFD00F657
:1099D000141390EDDE8AD3ED007AF4EE487AF1EEBE
:1099E00010FA48BFB0EE678ADFED5B7AB4EEE78A23
:1099F000F1EE10FA0CDD2422002104F1FC00DFF06E
:109A0000BDF90023C4F82C3121B0BDEC108BF0BDA2
:109A1000204616ADFEF714FD2046FEF7BDFEB0EE63
:109A2000480A204604F14C06FFF712FC2046FFF7D7
:109A3000D3FBFEF71DF904F1280100F53A7216A8D0
:109A40001BF0ACFD0FCD0FC60FCD0FC62B6804F178
:109A5000740204F1700104F14C00336004F17803E6
:109A60001BF042FF94ED1E8AB0EE480ADBF008FBC3
:109A700084ED710AB0EE480ADCF008F9204684ED66
:109A8000700AFEF7D1FCFEF7F3F804F5CC71FDF790
:109A9000C3FE80F089FCD4F8C831C31A632BB3D954
:109AA000C4F8C8014AF030FF054680F085FCDFEDC0
:109AB0002B7A94ED1E0A074694ED1C8A0E4694ED0F
:109AC0001D9A20EE270A28EE278A29EE279A1BF0F6
:109AD00039F9D4ED5FAAB0EE40AA94ED3BBAB7EEE7
:109AE000C88A94ED3CCAB7EEC99A94ED61DAB7EE34
:109AF000CBBA94ED62EAB7EECCCA94ED63FAFEF706
:109B00008FFA8AEE807A164B164A28460193164B36
:109B10001649B7EECDDA0093B7EECEEA144BB7EEA6
:109B2000CFFAB7EECAAA8DED12FB8DED10EB8DEDDD
:109B30000EDB8DED0CCB8DED0ABB8DED08ABB7EEDA
:109B4000C77A8DED069B8DED147B8DED048BCDE9F1
:109B500002764AF00FFB57E7CDCC4C3EE02E654233
:109B60004BF810086B231108A1F8100828211108E0
:109B70006023110870470000002070477047000004
:109B80000020704700207047002070470020704779
:109B90009FED010A704700BF000000009FED010A21
:109BA000704700BF000000007047000000207047B1
:109BB0007047000010B50446143000F019F804F1A5
:109BC0002C0000F015F804F17000A1F0D9FF04F1A9
:109BD000F400A1F0D5FF4FF0FF332046C4F8543114
:109BE00010BD0000014B1868704700BF2C8E00307C
:109BF00070470000094A0123D2ED057AD8B2F4EE8D
:109C0000C07AF1EE10FA02DD0138C0B270470133BC
:109C10001432082BF0D10720704700BF4C241108E4
:109C20000C4B1422DFED0C6AF0EE407A02FB0030A0
:109C300090ED047A90ED010AB0EEC76AB4EEE66AE0
:109C4000F1EE10FA5EBFD0ED006A77EEE67AA7EE8D
:109C5000270A70474C2411080000003410B5044650
:109C60003648F0EE407A012103462DED068B90ED4B
:109C7000077ACAB2F4EEC77AF1EE10FA23DD013AA0
:109C8000D2B2142101FB023393ED027A87EE870AE8
:109C9000DFED2B7AB4EEE70AF1EE10FA19DA48F0AC
:109CA000D9FEA7224FF4801148F08CFE637C50222D
:109CB000D4ED467A02FB034393ED0B0A30EE270AFC
:109CC000BDEC068B10BD013114300829CFD107221D
:109CD000D7E793ED049A93ED008AB0EEC97AD3EDFD
:109CE000019ADFED188A9FED18AAB4EEE77AF1EE3B
:109CF00010FA12D568EEE98ADBF0ECFCF0EE487A57
:109D000088EE8A7AE0EE077A9FED107A67EE876A2E
:109D100077EE677A86EEA70AD2E768EEC98AC8EEC0
:109D20008A0ADBF0F5FD89EE897AF7EE007A30EEEB
:109D3000670AF0EE487AE7EE007AE5E74C2411086E
:109D400000000034CB868F430AE81C413CFEC14A28
:109D5000DFED257A254920EE277A30EE270A08B56F
:109D600087EE005A2DED028BB0EE450AFFF742FF59
:109D7000142303FB001140B2FFF752FFDFED1C7A02
:109D8000D1ED045A91ED038AB0EEE57AB4EEE77AAC
:109D9000DFED187AF1EE10FA12D520EE270A9FEDCA
:109DA000167AC7EE007A91ED000A35EE400A27EEEA
:109DB000800ADBF0EBFB20EE080ABDEC028B08BD4D
:109DC00065EEA75ADFED0D7AC7EEA50AF7EE007A29
:109DD00070EEA70AD1ED017A80EE270AF1EE600A53
:109DE000DBF096FDE7E700BF3CFEC14A4C241108BA
:109DF00000000034CB868F430AE81CC10AE81C41EE
:109E000008B5FFF7A5FFDFED087A9FED087AB4EEFD
:109E1000E70ADFED077AF1EE10FA20FE270AC7EE17
:109E2000007AB1EEE70A08BD00000034CDCC9C3FBB
:109E3000BC77E93610B52DED028BF0EE608A044652
:109E4000FFF70CFFB0EE408A2046B0EE680AFFF73D
:109E500005FF30EE480ABDEC028B10BD427C50215C
:109E6000D0ED467A01FB020292ED0B0A30EE270A92
:109E7000FFF7C6BF38B52DED088BB0EE409A05460A
:109E8000F0EE609A1524B0EE408ADFED1DAA9FED3A
:109E90001DAA9FED1DBA013CA4B25CB3F0EE490AC5
:109EA0002846B0EE480AFFF7C5FF70EE698AF0EE6B
:109EB000490A284638EE2A0AFFF7BCFFB0EEE87AD6
:109EC00070EE697AB4EECA7A77EEE87AF1EE10FABB
:109ED00010D468EEAA8A40F26310B0EE4B1AF0EE8E
:109EE0004A0A88EEA70A38EE400A1AF0CFFFB0EE11
:109EF000408AD0E7B0EE480ABDEC088B38BD00BF01
:109F0000CDCCCC3D0AD7233C0024744900234360C8
:109F10008360C360036143618361C361002380F890
:109F20002030704790F82020531C00EB8202DBB2F7
:109F3000062B80F8203082ED010A84BF002380F8D0
:109F4000203070470022A3F045B900004FF0FF33E6
:109F500010B543610023044600F5967040F8D03CEC
:109F600040F8CC3C40F8C83C40F8803C40F87C3C91
:109F700040F8783C40F8303C40F82C3C40F8283C15
:109F80000C4B0360002380F82030FFF7BFFF0A4B23
:109F900004F5C870C4F82C317FF040FB074B204615
:109FA00007491C6044F0ECFED4F814312046C4F894
:109FB000183110BD3C2611084C261108308E003097
:109FC000F826110800F5967008B54CF067FEDFED35
:109FD000027A20EE270A08BD00007A4490ED5D0A5F
:109FE000DFED057AB0EEC07AB4EEE77AF1EE10FA62
:109FF00048BF90ED5E0A70470000003410B504467B
:10A0000080ED490A80F0D0F9C4F8280110BD0000A5
:10A0100073B5D0F8283104460E4663B180F0C4F918
:10A02000D4F82831C01A42F20F73984203D894ED45
:10A03000490A02B070BD114B1D687DB195F84E11F3
:10A040002846FFF7A3FD48B101AA95F84E1128460E
:10A05000FFF792FD10B19DED010AEAE75021DFED17
:10A06000087A01FB064494ED0A0AB4EEE70AF1EE21
:10A0700010FA58BFB0EE670ADBE700BF2C8E003045
:10A0800000000C4208B561B10378022B02D90648E2
:10A0900080F05AF95A1C027000EB830041600120E5
:10A0A00008BD0846FCE700BFEC2411082DE9F84381
:10A0B00005460E469146002400F13C082B7CA34245
:10A0C00011DD00234A463146012015F03BFB5023A9
:10A0D00007460021634358F8030015F043FB87420D
:10A0E00004D00134EAE70020BDE8F8830120FBE753
:10A0F00070B50B46064614469AB111469847054678
:10A1000028B9236820465B68BDE8704018470146BF
:10A110003046FFF7B7FF20B92B6828465B689847A1
:10A12000EFE770BD38B5084B04460D4611461B6875
:10A13000986803681B689847294602462046BDE890
:10A140003840FFF7D5BF00BF088E0030F0B50D4690
:10A1500085B011461A460446CDE90213FFF7A6FF63
:10A16000034698B90A480427006840680668DDE994
:10A170000212CDE90037074B3668B0470246294640
:10A18000204605B0BDE8F040FFF7B2BF0022F6E779
:10A19000088E0030801A06001A4B1B682DE9F04724
:10A1A0000546D0F8849158684FF0010A164C0368B0
:10A1B00004F1E4089B68984795F921310646002B85
:10A1C000A4BF01269E40236819EA030F07D0002789
:10A1D0000AFA07F3334206D10137202FF8D10C34A5
:10A1E0004445F0D10BE0237AFAB261682846FFF7C4
:10A1F000ADFF2B78032B02D02B7C032BECD1BDE8D9
:10A20000F08700BF088E0030182811087FB5D0ED08
:10A21000457A01239FED477A0446F0EEE77A03760C
:10A22000F4EEC77AF1EE10FA0AD400F58A70002332
:10A2300003A90190039345F083FD019844F064FF66
:10A2400000230325E363C4F88C30C4F8DC302046D7
:10A25000A3F0B8F901462046FFF714FF2378032B3B
:10A2600026D0237C032B23D0013D15F0FF05EED132
:10A27000314A20463149FFF755FF2378032B17D089
:10A28000237C032B14D02E4A20462C49FFF74AFF8B
:10A290002378032B0CD0237C032B09D094F92121A4
:10A2A000002A07DA2046FFF777FF2378032B0ED129
:10A2B00004B070BD7723D2B220492046FFF746FF95
:10A2C0002378032BF4D0237C032BEBD1F0E7237C02
:10A2D000032BEDD0D4F88431DA0403D5637E0BB9B7
:10A2E000012363760025637EEAB2EB40DB070CD4E2
:10A2F0000135082DF7D1237823B1237C13B163688E
:10A30000002BD5D10F4801F065FB3820019202F0F7
:10A3100011F8064618B1019A2146A4F025FC3146F1
:10A320002046FFF7AFFE2378032BC1D0237C032BFD
:10A33000DED1BDE7000000340825110821E80C0833
:10A340001325110820251108054B1B682BB1416905
:10A350004A1C02D018464AF0F5B80020704700BFEA
:10A36000B492003002290BD8502303FB010191F86D
:10A37000390030B191F83A0018B191F83B007047BC
:10A38000002070472DE9F047044680F00DF842F2B6
:10A3900010730027D4F87C614FF0500942F2107A14
:10A3A000861B9E4288BFC4F87C01FDB2237CAB4271
:10A3B0001CD929462046FFF7D5FF70B109FB054897
:10A3C000D4ED460A204698ED0D0AD8ED097A30EE14
:10A3D000270AFFF74FFD88ED0C0A564504D909FB03
:10A3E0000540303044F090FE0137DEE7617C2046C6
:10A3F000FFF70EFE84ED5E0ABDE8F08770B50446F7
:10A400002DED028B86B07FF0CFFFD4F81C310546CE
:10A41000C31AB3F57A7F3FD394ED467A9FED3A8A1B
:10A42000F0EEC76A394BD4ED457A1B68F4EEC86A82
:10A43000DB6AF1EE10FA93F89C6022D5F0EEE76A41
:10A44000F4EEC86AF1EE10FA1BD502A801F014FB75
:10A4500016BBFDF70DFC02A9FDF7DEF9E0B1DDED5D
:10A46000037A9FED2B7AF8EEE77A67EE877AB0EE03
:10A47000E77AB4EEC87AF1EE10FA11D4C4ED467A58
:10A4800011E077EE676AB7EE006AF0EEE66AF4EE86
:10A49000C66AF1EE10FA1CDC06B0BDEC028B70BD92
:10A4A0001C4BC4F81831C4F81C51FDF7E1FBFCF754
:10A4B0008FFE2046FFF766FF55F0A8FE94ED467A22
:10A4C000154A0621B7EEC77A8DED007B4FF078FF75
:10A4D000E2E7F0EEE76AF4EEC86AF1EE10FADBD4D8
:10A4E000002ECBD004F58A7084ED457A44F00CFE42
:10A4F00055F08CFE094A012106B0BDEC028BBDE887
:10A5000070404FF05DBF00BF00000034088E003087
:10A510000AD7233C6F12833A692511084425110894
:10A520002DE9F0412DED048B84B0044640F27232E7
:10A5300000F5C87103A8002515F0A8FAD4ED437AF8
:10A54000D4ED446A50229FED806A37EEE67A637C50
:10A5500002FB0343B0EEC77AB4EEC67AF1EE10FA0E
:10A56000C1BF9FED7A7A67EE877A9FED797AE6EE42
:10A57000877AC4ED447A93F83970E9B223788B4234
:10A5800006D904EB81030135586800F0ADFAF4E711
:10A590004FF000089FED6F9ADFED6F8ADFED6F9A45
:10A5A0005FFA88F5237CAB4271D9502303FB054346
:10A5B00093F83920002A3FD0D3ED0C7AF4EEC97A13
:10A5C000F1EE10FA0BDBF4EE677AF1EE10FA06D634
:10A5D000F0EEE77AF4EE687AF1EE10FA04DD50233B
:10A5E00003FB05435A6A1A63502606FB054696ED9F
:10A5F000098AD6ED0D0A96F8383038EE208AF3B97C
:10A6000029462046A4F082FD78EE400A204696EDC9
:10A610000C0AC6ED1A0AFFF70DFCD4ED467A30EEAF
:10A62000670AB4EE400AF1EE10FA18D75023002260
:10A6300003FB054383F83A2008F10108B0E7012B3A
:10A6400003BFD6ED0C0AD4ED5C7A30EEC88A96EDE5
:10A650000B0A04BF88EE297A87EE270AE1E7F0EEBD
:10A66000C07A502101FB0545F4EE687AF1EE10FA4C
:10A67000D7BF0123002385F83A30D4ED447ACEBF0A
:10A6800085F83A3037EE800A85ED0B0AD4E7627C14
:10A6900020461146FFF766FE48B1502104F596703A
:10A6A00001FB0242D16992ED0B0A4CF0D9FA94F900
:10A6B0002011267C002907DBB14205DACAB2204608
:10A6C0001146FFF74FFE68B900226274D5B2AE4260
:10A6D00009D9294620460132FFF744FE0028F5D06B
:10A6E000657400E062742046FFF788FE2046FFF79D
:10A6F0002BFE10B12046A3F03DFD637C502505FBE9
:10A70000034393F83930BB4216D04AF0FDF84FF6B8
:10A71000FF7149F017FF78B1607C05FB004494F8A5
:10A720003930002B14BF0022042201924AF0ECF8C9
:10A73000019A122149F098FE03A815F0C9F904B056
:10A74000BDEC048BBDE8F0810AD7233C0AD7A33CBB
:10A7500048E17A3F00000034FFFF7F7F0020194668
:10A760002DE9F04F04460F4687B0007C04F13A0310
:10A7700000220121D5B25033A84205D9013203F895
:10A780004F1C03F8501CF5E76F4B1E68F06A036816
:10A790005B68984740B155F039FD6C4A062107B017
:10A7A000BDE8F04F4FF00CBE55F030FD684A062171
:10A7B0000A254FF005FE002303A904F586700393D4
:10A7C00045F0BEFA7FF0F0FD80462046FFF7A8FE78
:10A7D0007FF0EAFDA0EB0800B0F5FA7F02D95D48F2
:10A7E00001F0F8F8B06A0A2103685B689847617C59
:10A7F0002046FFF7B7FD0028E7D0B06A013D64218D
:10A8000003685B68984715F0FF05DBD1524B05954F
:10A810001B888DF80650ADF80430CDE903550525A9
:10A820007FF0C2FD80462046FFF77AFE7FF0BCFD38
:10A83000A0EB0800B0F5FA7FD1D8617C2046FFF785
:10A8400091FD0028EFD094F810B00DF10C08A1464E
:10A8500001AA4FF0000A5FFA8AF18B4516D920460B
:10A86000FFF780FD50B1D8ED007A99ED097A1378A1
:10A8700077EE877A0133C8ED007A13700AF1010A86
:10A8800008F1040809F150090132E4E7B06A013D1A
:10A89000642103685B68984715F0FF05C0D1A9469D
:10A8A0004FF05008237C5FFA89F6B34226D906ABF5
:10A8B000334413F8143C33B908FB064686F83B30A2
:10A8C00009F10109EEE7002FFAD006AA07EE903A47
:10A8D0002046D4ED460A02EB8602F8EEE77A12ED46
:10A8E000030A80EE270AFFF7C5FA08FB064002A913
:10A8F0008DED020A303045F023FAE1E700264FF0F3
:10A900005008DFF85C902046617CFFF781FB84ED06
:10A910005E0A237CF7B2BB420FD908FB074393F8CA
:10A920003B3043B1013555F071FC7B1C4A46EDB21A
:10A9300006214FF045FD0136EBE70DB907484FE71B
:10A9400007B0BDE8F08F00BF088E003084251108E5
:10A95000AF251108C525110800CF100801261108E0
:10A96000DF25110808B5037C022B02D903487FF0CC
:10A97000EBFC5A1C0274184608BD00BF20261108C3
:10A9800038B50246057C0024E1B28D4206D9104656
:10A990000134FFF7E7FC0028F6D138BD281E18BFA8
:10A9A0000120FAE770B50D4609780446072906D854
:10A9B000027E437E22B901228A401343437670BD52
:10A9C000002BFCD000262278F3B29A42F7D904EB90
:10A9D00083032946013658680368DB689847F2E725
:10A9E00037B50D460192FFF7CBFF0199044630B908
:10A9F00004482A46044B0068C06A15F049FA20460C
:10AA000003B030BD088E0030CB5E1208014B1868D1
:10AA1000704700BF308E00307047000073B5436848
:10AA200005460C461B7C8B4242D900F108012122CD
:10AA300001A815F02BF87FF0B7FC6A68502303FBE0
:10AA40000423D969411AB1F5FA7F33D2196A401A41
:10AA5000B0F5FA6F2ED2D3ED097A9FED177AF0EEAA
:10AA6000E77AF4EEC77AF1EE10FA54BF0120002025
:10AA700050269FED127A06FB04F31A4482F839003F
:10AA800069680B44D3ED0A7AF4EEC77AF1EE10FA56
:10AA900006D49FED0B7AF4EEC77AF1EE10FA04DDDE
:10AAA00006FB0411002381F8393001A815F010F8D5
:10AAB00002B070BD0020DBE700000034000048C396
:10AAC00000004843044B10B50446C0E9003108308B
:10AAD0007EF0A4FD204610BD0429110843685020D3
:10AAE00000FB0131CA63704713B503680446019146
:10AAF0009B6898472368019920461B6902B0BDE80E
:10AB000010401847F8B52DED028B4368F0EE408AEF
:10AB1000B0EE608A05461B7C0C468B421FD950273D
:10AB20007FF042FC6B68F0EE680A674306463B44E0
:10AB300093ED090A1AF060F8A0B96B68502202FB85
:10AB400004331E6250216B684C432344C3ED098AD1
:10AB50006B68234483ED0A8A69680C44E661BDECA6
:10AB6000028BF8BD6B68F0EE480A3B4493ED0A0A8D
:10AB70001AF042F80028E0D0E4E70000B0EEC07A16
:10AB8000DFED297AB4EE677AF1EE10FA49DCB4EE23
:10AB9000400AF1EE10FA44D6436893F9803163B16C
:10ABA00090ED087ADFED217AF0EEC76AF4EEE76AFD
:10ABB000F1EE10FA03D580ED080A01232BE077EEC1
:10ABC000407ADBB237EE006AF0EEE77AC7EE866ACB
:10ABD0009FED176A07EE903AF8EE677A26EE866ADE
:10ABE000B4EEE76A9FED136AF1EE10FA15DDF2EEAE
:10ABF000047A436A013366EEA76A43620023C6EE15
:10AC0000267AF7EE006A27EE800A76EEE76AA7EE6C
:10AC1000260A80ED080A18467047F0EE467A0123AE
:10AC2000EFE70023F7E700BFFFFF7F7F000000345E
:10AC300000004843CDCCCC3D002070470020704739
:10AC400000207047704700000020704790F83600E1
:10AC50007047000090F83B007047000001207047EB
:10AC600000207047022070477047000010B504466E
:10AC700001F068FB204610BD90F8A835934207D933
:10AC800002F5B07250F8220010B103689B6A1847B1
:10AC9000002070472DE9F3416E46054604460F46F5
:10ACA00000F5C87886E80C00114B45F8043B2846AF
:10ACB0002C3500F07BFDA845F9D104F2AC53C4F863
:10ACC000A47596E8030083E80300089B2046094921
:10ACD000C4F8B43544F054F8074B1A6812B1074869
:10ACE0007FF032FB20461C6002B0BDE8F08100BF5F
:10ACF000482B1108102A1108348E00301829110829
:10AD00002DE9F04F2DED028B90F8A83583B0044665
:10AD1000002B64D17F2200F5C87500F5B067061DD1
:10AD200099469FEDB18A80F8B8255FFA89FA1C220E
:10AD3000FF212846DEF022F885F864A096F926B0B7
:10AD4000ABF103031C2B2AD8DFE813F01D001D0014
:10AD5000290029004E009800A500B200C100CE00D5
:10AD60005A0068008C007000290029007F0029002B
:10AD7000E8002900F500DB000301290010011E0195
:10AD80002B0129001D00442001F0D4FA804620B197
:10AD900033462A462146A4F0F3FBC7F80080386802
:10ADA00050B1E96EC5F868B031B1904B43F8291045
:10ADB00044F0E0F944F0D6F90AF1010A57F8040B1F
:10ADC0005FFA8AFA20B103689B68984784F8A8A5BF
:10ADD00009F1010970352C36B9F1090FA5D103B07D
:10ADE000BDEC028BBDE8F08F7C2001F0A3FA804619
:10ADF0000028D2D033462A462146A6F0F1FECCE701
:10AE0000482001F097FA80460028C6D0032300931B
:10AE10002A4633462146A7F005F9BEE7482001F04F
:10AE200089FA80460028B8D00623F0E77C2001F09C
:10AE300081FA80460028B0D033462A462146A6F043
:10AE4000CFFE6B4BC8F80030A7E77C2001F072FA08
:10AE500080460028A1D033462A462146A6F0C0FEEF
:10AE6000644BEFE7442001F065FA8046002894D057
:10AE700033462A462146A7F05BF88EE7E82001F02A
:10AE800059FA8046002888D000232A462146009699
:10AE9000A5F048F881E7382001F04CFA80460028F8
:10AEA0003FF47BAF33462A462146A5F01DFE74E7EA
:10AEB000302001F03FFA804600283FF46EAF334661
:10AEC0002A462146CDF800A0A7F082FB65E7542072
:10AED00001F030FA804600283FF45FAF33462A463F
:10AEE0002146A5F0DFFE58E75C2001F023FA8046FA
:10AEF00000283FF452AF33462A462146A6F028F8F0
:10AF00004BE7582001F016FA804600283FF445AF81
:10AF100033462A462146A5F06FFF3EE7782001F030
:10AF200009FA804600283FF438AF33462A462146C6
:10AF3000A6F0ACF831E72C2001F0FCF9804600289F
:10AF40003FF42BAF33462A462146A4F0C1FC2A4BDE
:10AF500078E7482001F0EEF9804600283FF41DAF65
:10AF600033462A462146A7F0A5FB16E7282001F024
:10AF7000E1F9804600283FF410AF33462A462146C7
:10AF8000A4F0A6FC1D4B5DE75C2001F0D3F98046E0
:10AF900000283FF402AF33462A462146A4F0A8F920
:10AFA000FBE6A02001F0C6F9804600283FF4F5AE8C
:10AFB00033462A462146A4F08BFC114B08F1880049
:10AFC00088ED1D8AC8F800304FF6FF7388ED1E8AA1
:10AFD000A8F82E30A8F8703088ED1F8A88ED208AF6
:10AFE0007EF01CFBD9E600BF0000C07F388E003029
:10AFF000BC291108A0E31208B0E51208A4DE12086B
:10B0000058E4120890F8A8358B4283BF702303FBE5
:10B01000010090F8E10100207047000090F8A83589
:10B020008B4283BF702303FB010090ED6B0A9FED01
:10B03000010A70470000000090F8A8358B4206D93D
:10B0400001F5B07150F8210008B1A4F053BC9FED98
:10B05000010A70470000000010B490F8A8450A46A5
:10B060008C4214D901F5B07450F824407CB1E468E6
:10B07000246A640603D55DF8044BFFF7DDBF702139
:10B0800001FB020393ED6B0A5DF8044B70479FEDE3
:10B09000010AF9E70000000090F8A8358B420BD9AF
:10B0A00001F5B07150F8210038B1C3681B6A1A422B
:10B0B00014BF0120002070470020704770B590F841
:10B0C000A83504460E461546934201D8002070BDAF
:10B0D00002F5B07350F823000028F7D003689B698D
:10B0E00098470028F2D0702202FB0544D4F8B03112
:10B0F0003360ECE770B590F8A83504460E46154667
:10B10000934201D8002070BD02F5B07350F82300BF
:10B110000028F7D003689B6998470028F2D0702276
:10B1200002FB0544D4ED6D7AF4EE677AF1EE10FA85
:10B13000E8D6C6ED007AE6E770B590F8A835044683
:10B140000E461546934201D8002070BD02F5B0733B
:10B1500050F823000028F7D003685B69984700285F
:10B16000F2D0702202FB0544D4F8B8313360ECE72A
:10B1700090F8A83593420ED902F5B07350F82330F9
:10B180005BB1702303FB020292F8F00130B1D2F8F8
:10B19000EC310B6070470020704718467047000084
:10B1A00008299DBF2C2303FB010040680020704745
:10B1B000474B1B682DE9F04F2DED028BDB6A87B002
:10B1C000044693F89C30002B7DD04FF00009DFF847
:10B1D00014A1DFF814B19FED3F8A5FFA89F594F866
:10B1E000A835AB426FD905F5B07354F82300002899
:10B1F00053D003685B6B98477023074603FB0543F6
:10B2000093F8E031834248D2032857D8DFE800F0B2
:10B210004502484F304E4FF0000854F0F7FF94F8C5
:10B22000A8256B1C0421AA4289BF7022B0EE487A7F
:10B2300002FB054292ED6B7A702202FB0545B7EEE8
:10B24000C77A524695ED6D6A0096B7EEC66A8DEDE7
:10B25000027B8DED046B4FF0B3F8012384F8B93510
:10B260008BF80B3085F8E071D4F8B4354BB300227D
:10B2700055B25957481C03D0414502F10102F7D19C
:10B2800094F9B835AB4208DBD4F8B03542463146C4
:10B29000D4F8AC05984784F8B85509F101099CE742
:10B2A0002C230E4E03FB054393F92D80B5E72C2389
:10B2B0000B4E03FB054393F92E80AEE70026B04604
:10B2C000ABE71D46DCE707B0BDEC028BBDE8F08FB5
:10B2D000088E00300000000045291108A2DC120889
:10B2E0003C291108542911088D8F00300020704727
:10B2F00090F8A8358B4207D901F5B07150F82100BC
:10B3000010B10368DB6918470020704708299CBF0B
:10B31000702303FB010000F5C8707047F8B50446C0
:10B320000E4615461F46FFF7E3FFD0B10D2D19D885
:10B33000082E9CBF702101FB06444FF6FD7104F5F9
:10B34000C87434F81520531E9BB28B420AD807EEFE
:10B35000902A9FED057AF8EEE77A67EE877AC7EDD7
:10B36000007AF8BD0020FCE76F12833A90F8A83508
:10B37000934207D902F5B07250F8220010B1036869
:10B380005B6A18470020704790F8A8358B420DD9AA
:10B3900001F5B07350F8233043B1702303FB010172
:10B3A000012081ED740A81F8CC01704700207047BC
:10B3B000F8B5002402460E462C272546E1B292F845
:10B3C000A8358B4210D901F5B07352F823304BB138
:10B3D00007FB01239B689E4204D11046FFF7D4FF70
:10B3E0002843C5B20134E9E72846F8BD0B461146AB
:10B3F00090F8A8259A4207D903F5B07350F82300B6
:10B4000010B10368DB6A1847002070472DE9F04F40
:10B41000002493B005460E46174621462F2206A863
:10B42000059405F5B069DDF0A9FC05F12A0A4FF095
:10B430002C0B05F5FC730BFB04F259F8040BE5B279
:10B440001AF9021030B951B90134092CF3D14FF077
:10B45000010813E0702262439A58914212D00135DC
:10B460001448154B4FF000080068EDB201933246C6
:10B4700000953946114BC06A14F00AFD404613B0DE
:10B48000BDE8F08F05A933220393A4F013FB05A9AF
:10B490008046039B0028D7D10135064801913246EA
:10B4A000EDB20068054B39460095C06A14F0F0FC17
:10B4B000E4E700BF088E0030793611087C291108B6
:10B4C0002DE9F04F06468DB00027DFF87C90DFF8BD
:10B4D0007CA0DFF87CB096F8A835FCB2A3422ED948
:10B4E000702505FB046595F8E83133B395F8E9114B
:10B4F00019BB4FF00108202204A8444489F81980A0
:10B50000DDF03CFC4AF2104307EE904A03AA4C21BE
:10B510005046F8EEE77AADF828302423CDED037AD3
:10B520004EF044FD54F072FE9BF80030054A0421B1
:10B5300000944EF045FF85F8E9810137CBE70DB067
:10B54000BDE8F08F8C2911088D8F0030A493003056
:10B5500020270030304B2DE9F04F1E6885B004469F
:10B5600046B1D0F8A415304648F0ECFF10B1304693
:10B5700047F08EFE4FF000084FF02C0A4FF0700B92
:10B580007EF012FF01905FFA88F594F8A835AB427F
:10B5900039D904EB8507D7F8800588B30AFB054342
:10B5A0000BFB054993F92A20D9F8F8118A4227D1D3
:10B5B00032B30268D2689047D7F880050268126BF0
:10B5C000904799F8E12112B1019BC9F8E431BEB16D
:10B5D000D4F8A415304648F0B5FF88B17EF0ECFEF3
:10B5E00002460B46CDE902102946D7F88005A6F0A1
:10B5F00075F82946D7F88005DDE90232A6F0E4F8AF
:10B6000008F10108BFE72046FFF7D2FD204605B04C
:10B61000BDE8F04FFFF754BFB49200302DE9F0477A
:10B620004FF0000804468946012647464FF0700A4D
:10B630002DED028BB0EE408A94F8A8355FFA88F5BC
:10B64000AB421AD929FA05F3DB070AD505F5B07321
:10B6500054F8230078B10368B0EE480A9B6B984712
:10B6600006400AFB054508F1010895F8E0319F42C4
:10B6700038BF1F46E0E70646F3E727B97F23A4F863
:10B68000B835034BDF723046BDEC028BBDE8F08766
:10B690008D8F003090F8A8358B4207D901F5B07135
:10B6A00050F8210010B10368DB6B18470020704789
:10B6B0000B46114690F8A8259A4207D903F5B073B6
:10B6C00050F8230010B103681B6C18477047000046
:10B6D00070B504460E460025E9B294F8A8358B42B1
:10B6E00005D9324620460135FFF7E2FFF4E770BD89
:10B6F0002DE9F843024690F8A855002400F12A06E7
:10B700002C2700F5FC784FF07009E1B28D420FD97B
:10B7100007FB04F309FB04F0F35658F800008342DA
:10B7200009D11BB11046FFF76DFC10B10134ECE7F5
:10B730000120BDE8F8830020FBE7000010B590F879
:10B74000A82504468A4217D9702202FB010393F808
:10B75000E031022B03D004D9032B18BF0023184675
:10B7600010BDFFF797FF48B92046FFF7C1FF00283B
:10B770000CBF06230123F2E70023F0E70623EEE7E0
:10B780000B46114690F8A8259A4207D903F5B073E5
:10B7900050F8230010B103685B6C18470020704715
:10B7A000014B1868704700BF348E003010B5044656
:10B7B000024943F0E5FA204610BD00BFD02B110826
:10B7C00000F120034022002110B504461846DDF0A8
:10B7D000D5FA9FED0C1ADFED0C0A9FED0C0A6AF00A
:10B7E00049FA002304F1600084F8403084F85C30AA
:10B7F00063F0FEFF064B204606491C6043F0C0FA8A
:10B80000204610BD00008C429A99993E00004843A2
:10B810005C8E0030C42D11082DE9F3410546B7EECA
:10B82000000A0022022142F0B5FE2846A7F038F9AE
:10B8300064F0BCF9234B04461E68F06A03685B6A37
:10B8400098470B46022102462046009163F0E6FF2E
:10B85000B5F99270002F13DDD6F82C80BCB2D8F861
:10B86000003040465B68984728B198F84D3013B1D6
:10B87000C92FA8BFC824B06A214603685B689847EF
:10B880002022002195F9910019F068FBC4B265F0FF
:10B8900031FB65F077FA70B9B06A013405210368AD
:10B8A000E4B25B689847072CF1D9074802B0BDE8BD
:10B8B000F0417DF0EBBF072CF7D885F8914002B03E
:10B8C000BDE8F081088E0030D02C110810B5044678
:10B8D000A7F086F82046BDE81040A7F0B1B80000F8
:10B8E0002DE980481446284B012293B005460E46A8
:10B8F0004FF00008DFF89490DFF894A0DFF894B0E0
:10B900001A707EF051FDD9F80030A0EB080207460E
:10B91000039341F287339A421FD903985346342246
:10B9200005A9B846CDE90056C06A14F0B1FA21461F
:10B9300005A804947DF09AFF03985B46342205A97C
:10B94000CDE90056C06A14F0A3FA049454F05EFCEA
:10B95000049B05AA02214EF01BFD54F057FC54F045
:10B9600025F954F053FC56F077FC0A2105A814F091
:10B9700073F8039B0521986A03685B68984705A8DC
:10B9800014F076F8BDE700BF608E0030088E0030FE
:10B99000A1C11108790213080FB400B595B00021B8
:10B9A00016AA05A8049152F8043B03923C22019385
:10B9B000DDF0E4F9054A4021019B04A87DF0FEFE7C
:10B9C000039A04A90248FFF78BFF00BFE82C110877
:10B9D000FE2C11080FB407B504AA034852F8041B43
:10B9E0000192FFF77DFF00BF102D11080A2938B51D
:10B9F00018D10E4BC4881B68B0F90650D86A14F0F1
:10BA0000040302D190F89C2062B90368DB6998476F
:10BA1000012802D105F0010038BD022804D1C4F389
:10BA20004000F9E70020F7E70120F5E7088E003035
:10BA3000014B1868704700BF5C8E003038B5044673
:10BA40000025E289ABB2A0689A4205D950F82300DC
:10BA50000135D7F09FF9F4E7D7F09CF9204638BDBF
:10BA60001022044908B5DDF02FF9B0FA80F0400942
:10BA700008BD00BF648E003010220021DDF07EB9C9
:10BA80000378022A416023F00D03037008D0032AD3
:10BA90000AD0012A03D1DBB243F0010303707047DF
:10BAA000037843F00803F9E7037823F0050343F034
:10BAB0000503F3E773B504460E4615460193FFF7F9
:10BAC000DBFF2046069A0199C4E90265FFF7D8FF1B
:10BAD00002B070BD4B68436003780A7862F30003DC
:10BAE00003700B780278C3F3800363F38202027061
:10BAF000D2B20B78C3F3C00363F3C3020270704782
:10BB00000078420704D4030704D400F00100704712
:10BB10000320704702207047F0B587B004461546F1
:10BB2000FFF7EEFF88420F46064605D163682B609B
:10BB30000126304607B0F0BD00230328019301D051
:10BB4000032913D146F088F808B90026F1E701234C
:10BB500001AA214645F0E8FD0028F6D0DDED017A86
:10BB60009FED337A67EE877ACDED017A032E32D8D6
:10BB7000DFE806F0020916246468032FE5D8DFE841
:10BB800007F02C2E3C49FCF773F890F89432DB0751
:10BB9000DBD56468FCF76CF8D0F888321C44ECE71D
:10BBA00002A8FFF769FFFCF763F802A9FBF734FE70
:10BBB00006460028BDD06468039BEFE7D4ED017A08
:10BBC0009DED017AF8EEE77A77EE877AFDEEE77A77
:10BBD00017EE904AD1E70024CFE72C60A8E7FCF7E6
:10BBE00047F890F8946216F00106AED0FCF740F8E2
:10BBF000D0F88832E41A2C609BE702A8FFF73CFFDC
:10BC0000FCF736F802A9FBF707FE0646002890D09D
:10BC1000039BEFE707EE904A9DED017AF8EEE77A95
:10BC200077EEC77AFDEEE77AC5ED007A80E700BFD0
:10BC30000000C84273B501AA05460E46FFF76CFF27
:10BC4000044620B1324601992846FFF719FF2046E5
:10BC500002B070BD13B5144601AAFFF75DFF48B1ED
:10BC6000DDED017A9FED047AF8EEE77A67EE877AE8
:10BC7000C4ED007A02B010BD0AD7233C07EE900A4B
:10BC80009FED0C0AF8EEE77A08B527EE800AD9F0A6
:10BC9000F7F9DFED097AB4EEE70AF1EE10FA02DD0A
:10BCA000B7EEC00A08BD9FED010BFBE700000040A6
:10BCB000E17A843F50E0EF300AD7233C10B50446C8
:10BCC000806819F09FFB20B1E068BDE8104019F0D2
:10BCD000ADBB10BD73B5856804460E461DBBC36879
:10BCE00023B98B6801258360CB68C360636873B92F
:10BCF0002378DB070BD52046FFF702FF01AA014698
:10BD00003046FFF709FF10B1019B054663602046EE
:10BD1000FFF7D4FF20B9B3680125A360F368E3609F
:10BD2000284602B070BD0025E0E700000D4B8342BD
:10BD30004FF000038B4106DA00F1255000F5311079
:10BD400000F5E0507047084B98424FF0FF3371EB1D
:10BD50000303BEBF00F1564000F5130000F5244078
:10BD6000704700BF00D2496B002EB69490EA010FD5
:10BD700001D4401A7047C317401A63EBE1710D4BB1
:10BD800083424FF000038B4106DA00F1255000F5A5
:10BD9000311000F5E0507047074B98424FF0FF33E9
:10BDA00071EB0303BEBF00F1564000F5130000F530
:10BDB0002440704700D2496B002EB69470B52DED2B
:10BDC000028B84B004460D466846FFF755FEFBF72C
:10BDD0004FFF6946FBF720FD064628B3A368029A89
:10BDE000DFED148A9B1A039907EE903AF8EEE77A92
:10BDF00067EEA87AC5ED007AE068FFF7B7FF08EEB6
:10BE0000100AA068B8EEC88A024428EE288A02EB1D
:10BE1000D2725010B7EEC88AFFF730FF28EE000B41
:10BE2000B7EEC00B85ED010A304604B0BDEC028BC5
:10BE300070BD00BFF67C8E3F002337B50C4601AACB
:10BE4000022105460193FFF767FE10B9002003B0F9
:10BE500030BD21462846FFF7B1FF0028F6D0DDEDC2
:10BE6000017AF8EEE77AC4ED027AF0E708B5FFF759
:10BE7000E3FF08BD38B50D46FFF7DEFF044620B1ED
:10BE80009FED030A28461CF0D7FF204638BD00BFAF
:10BE90000AD7233CF0B50D4606462DED028B8C6883
:10BEA00089B0D0E90271E868FFF760FF08EE100A78
:10BEB000E019E41B00EBD0704010FFF7DFFEB8EE96
:10BEC000C86ADFED0F4A736826EE246A6A689FED40
:10BED0000D1A9B1AB7EEC66A07EE903A26EE006B73
:10BEE000B8EEE75A07EE904AF8EEE75AF7EEC60BBF
:10BEF00025EE011A25EEA40A09B0BDEC028BF0BDB7
:10BF00008262363C0AD7233CF0B50D4606462DED3D
:10BF1000028B8C688DB0D0E90271E868FFF726FFCC
:10BF200008EE100AE01900EBD0704010FFF7A6FEF3
:10BF300073686A68B8EEC87ADFED107AB0EE401B1D
:10BF40009B1A02EE103AE31BB8EEC22A00EE103A3A
:10BF5000B8EEC00A22EE272ADFED097A27EE277A0B
:10BF600020EE270AB7EEC22AB7EEC77AB7EEC00AAC
:10BF700027EE011B0DB0BDEC028BF0BD0AD7233CB0
:10BF80008262363CF0B52DED028B8BB00D46002160
:10BF9000074605AA0691FFF7BFFD002190BB0023CD
:10BFA000CDE90533D7E90261AC68E868FFF7DEFE4A
:10BFB00008EE100AA019A41B00EBD0704010FFF788
:10BFC0005DFEB8EEC86ADFED134A9FED131A26EE48
:10BFD000246ADDE90532B7EEC66A9B1A07EE903A8D
:10BFE00026EE006BB8EEE75A07EE904AF8EEE75AF5
:10BFF000F7EEC60B25EE011A25EEA40A0BB0BDEC38
:10C00000028BF0BD06AA2846FFF786FD0028C6D0A1
:10C01000C8E700BF8262363C0AD7233C38B50C46DD
:10C0200002462DED028BC168E068FFF79FFE956820
:10C03000A46808EE100A6019641B00EBD070401071
:10C04000FFF71CFE07EE904AB8EEC81BB8EEE77B80
:10C0500087EE006BBDEEC60B10EE103A5B4200EEB1
:10C06000103AB8EEC00BD9F04BFF9FED087B30EED5
:10C07000070BB5EEC00BF1EE10FA03D59FED057B73
:10C0800030EE070BBDEC028B38BD00BF0000006036
:10C09000FB21F93F00000060FB2119400B4630B541
:10C0A0002DED028B8C6885B0D0E90251D868FFF77E
:10C0B0005DFE08EE100A6019641B00EBD0704010A2
:10C0C000FFF7DCFDB8EEC86A9FED095A07EE904A0B
:10C0D00026EE056AF8EEE75AB7EEC66A26EE006B62
:10C0E00025EE850AF7EEC60B05B0BDEC028B30BD20
:10C0F0008262363C0B4630B52DED028B8C6889B0E0
:10C10000D0E90251D868FFF731FE08EE100A601935
:10C11000641B00EBD0704010FFF7B0FD07EE904AB3
:10C12000B0EE401BB8EEE76BB8EEC87B9FED050B99
:10C1300027EE007B26EE000B27EE011B09B0BDECBD
:10C14000028B30BD0000004050CC863F84B004B06C
:10C15000FFF7D0BF10B52DED048B84680B468A68BD
:10C16000111B224409EE101AC168D86802EBD27282
:10C17000FFF7FCFD08EE100A5010B8EEC99BB8EEB0
:10C18000C88BFFF77BFD28EE000B20EE000BA9EE1D
:10C19000090BBDEC048BB1EEC06B9FED020B26EEDC
:10C1A000000B10BD0000004050CC863F094B984268
:10C1B00006DDC0F1D64000F5930000F5A4407047BD
:10C1C000054B9842BEBFC0F1144000F5360000F5A3
:10C1D0003850704700E9A43500175BCAF8B52DED5B
:10C1E000048B9FED149BB0EE418B076806460D460D
:10C1F00020EE090B28EE098BFDEEC07B17EE904A6E
:10C2000004EBD47007EB6000FFF738FD88EE007B8D
:10C210003819FFF7CBFF306051EC170BF4F720FC17
:10C220002B68C01841EBE371FFF780FD2860BDEC7F
:10C23000048BF8BD000000404075564000F10C0131
:10C240000830FFF7CBBF000000B52DED068B9FED4A
:10C25000109B83B0B0EE418B20EE099B0190B0EEB5
:10C26000490BD9F03BF8B0EE40ABB0EE490BD9F03A
:10C2700075F820EE081B01982AEE080B03B0BDEC00
:10C28000068B5DF804EBFFF7D9BF00BFAFF300806A
:10C29000000000A046DF913F10B52DED0A8B9FED09
:10C2A0001ECBB0EE409B0446B0EE42AB21EE0CBB81
:10C2B00029EE0C9BB0EE4B0BD9F010F8B0EE408B92
:10C2C000B0EE490BD9F00AF8B0EE40CBB0EE490B16
:10C2D000D9F044F828EE001B204628EE0C8B21EE06
:10C2E0000A1B28EE0A0BFFF7A9FFB0EE4B0BD9F0A3
:10C2F00035F820EE0A0B63689FED092BBDEC0A8B25
:10C3000020EE020BBDEEC00B10EE102A134463604A
:10C3100010BD00BFAFF30080000000A046DF913FDA
:10C3200000000000000059400148FFF7A5BB00BF16
:10C33000648E00300121884238BF0846D6F026BD01
:10C34000FFF7F8BF08B1D6F025BD7047FFF7FABF79
:10C35000F8B506460F46144622B92546D6F01AFD12
:10C360002846F8BD10461EB9BDE8F840D6F0CEBC50
:10C37000D6F0CCFC05460028F2D0BC42224631461D
:10C3800028BF3A46DCF0B0FC3046D6F003FDE7E7C4
:10C3900010B50B680446084611461B689847206094
:10C3A000204610BD37B5089D0446084611461A467A
:10C3B000036801959DF81C5000951D68069BA847D1
:10C3C0002060204603B030BD90F9253013B190F8BD
:10C3D000440370471846704700214FF0FF33002296
:10C3E00010B54363044600F1400301604160816081
:10C3F000C16080F8291000F50C70D9707C3343F8C7
:10C40000742C43F8702C43F86C2C43F8682C43F8D8
:10C41000642C43F8602C43F85C2C43F8582C43F808
:10C42000542C43F8402C43F83C2C43F8382C43F868
:10C43000342C43F8302C43F82C2C43F8282C43F8A8
:10C44000242C43F8202C43F8102C43F80C2C43F8F0
:10C45000082C9842D1D1214604F5177007F0C8FF87
:10C46000044B1A6822B9044920461C6042F088FC3B
:10C47000204610BD748E0030EC30110873B5D0F832
:10C48000403204460191994213D0D0F84432994287
:10C4900018D0D0F848328B4216D102200AE0D4F8E6
:10C4A000383253B3D4F83C324BB34FF0030002B0F0
:10C4B00070BD002094F826308342F8D8431C84F8DD
:10C4C0002630F4E70120F5E7D0F83462002EE6D1FB
:10C4D00094F845233546B6009AB1A319C3F834122F
:10C4E000A319019A2846C3F8402294F82630AB429B
:10C4F0009CBF6B1C84F82630D9E70126E8E70226AA
:10C50000E6E704F50D7001A9304443F031FDE7E79B
:10C5100038B504460D4643F097FC291D201D43F015
:10C5200093FC05F1080104F1080043F071FD05F1E9
:10C53000140104F1140043F06BFD05F1200104F136
:10C54000200043F065FD05F12C0104F12C0043F0BF
:10C550000FFC05F1300104F1300043F021FD05F13D
:10C560003C0104F13C0043F053FDAB6BA3636B6BE8
:10C57000636338BD2DE9F04300F14007A1B000230B
:10C580000025064600F51078B9468DF8075003934C
:10C590000493059306930793089309930A930B93C7
:10C5A0001093119312931393149315931693179357
:10C5B00018931C931D931E9358F8043BF3B1326FEC
:10C5C000934222D0D6F8EC20934220D0D6F86821AE
:10C5D000934213D10221EBB299420FD0C1EB41112A
:10C5E00001A809EB81042146FFF792FF3946204656
:10C5F000FFF78EFF01A93846FFF78AFF01357C3728
:10C60000032DD9D121B0BDE8F0830021E3E701215A
:10C61000E1E700002DE9F04704460E461546804646
:10C6200007464FF0000A31462046FFF727FFBA6F52
:10C630005FFA8AF9B2420ED1C3B2022B0BD87C2228
:10C6400002FB0A44012084F8433084F8420085F854
:10C650000090BDE8F0870AF1010A7C37BAF1030FB8
:10C66000E1D1002731462046FFF708FFD8F87020B7
:10C670005FFA87F912B9C3B2022B19D9013708F151
:10C680007C08032FEED131462046FFF7F7FEC2B2F9
:10C69000C2EB421304EB830393F8427067B9022A9A
:10C6A0000BD8012083F8432083F842002A70D0E79A
:10C6B0007C2000FB0744C5E700274FF07C0904F10C
:10C6C000420A31462046FFF7D9FE034609FB07F030
:10C6D0005FFA87F81AF8002012B9DBB2022B09D9E9
:10C6E0000137032FEDD194F8271004290BD91448F2
:10C6F0007DF02AFE0444012084F8433084F842008F
:10C7000085F80080A5E704F54477002057F8043B3E
:10C71000C2B2B34208D1914202D8531C84F82730E8
:10C7200003322A70002094E733B9481CC43184F8DE
:10C73000270044F82160F3E701300528E6D1F1E74E
:10C74000F42E1108C9B200EB8101D1F8403253B187
:10C75000426F93420AD0D0F8F020934208D0D0F82C
:10C760006C21934206D04FF00300704700207047C1
:10C7700001207047022070472DE9F8430F4691468B
:10C78000044600F5BA7894F8425035B97C344445F3
:10C79000F9D100252846BDE8F88300234A463946EA
:10C7A000012012F0CFFF06460021206F12F0DAFFC1
:10C7B0008642EBD1EEE70000012303FA01F1D0F845
:10C7C0000C3319420AD14AB190F82430032B1FBF11
:10C7D000591C063380F8241040F8232070470000CD
:10C7E00038B505460C4609B9002038BD084612F098
:10C7F000C9FF0328F8D105F5497305F54E7253F8C2
:10C80000041BA142F0D09A42F9D1AB6F9C42EBD00D
:10C81000D5F8F4309C42E7D0D5F87001001B18BF62
:10C820000120E2E738B505460C4679B1084612F01A
:10C83000A9FF03280AD105F54472002352F8041B0E
:10C840008C4204D1C433002245F8232038BD013383
:10C85000052BF3D1FAE700002DE9F04FD0F80C5387
:10C8600089B0044615F4006525D1E8B203F03CFD1B
:10C87000024618B10B212046FFF79EFF94F827309F
:10C88000052B02D00135082DEFD1B4F84E329B07AD
:10C8900011D594F8455375B904F510763068B14652
:10C8A00012F070FF03285FFA85FA06F1040605D03E
:10C8B0000135032DF2D109B0BDE8F08F5146204675
:10C8C000FFF740FF7C23C0B203FB004090F84270AA
:10C8D000002FEDD104F50D73A9F10C090493314B30
:10C8E0000293029B20465FFA87FBD3F80C804146F7
:10C8F000FFF776FF0390F8B153F088FC56F8043C3C
:10C90000294A012100932B464DF05AFD002307A927
:10C910004846079343F02CFB0023584646F8043C56
:10C9200003F0E2FC07A970B102460B212046FFF795
:10C9300043FF4146FFF776FF029B01371033032F79
:10C940000293CED1B4E7A34604F5BA73DBF87020A6
:10C95000904517D19BF843200593524516D90023E3
:10C960000793049B03EB820043F002FB9BF84320F8
:10C970000023039804EB820207A9C2F84032059B0A
:10C980008BF843A00BF17C0B5B45DFD10028D3D0A3
:10C9900007A94846CDF81C8043F0EAFA46F8048C13
:10C9A000CAE700BF948E0030102F11082DE9F04324
:10C9B000044685B000F5107600257C27DFF87080EE
:10C9C000B14656F80C3CE9B20436D9F8002093423F
:10C9D00019D1C3B12046FFF7B5FEC0B207FB004036
:10C9E00090F842307BB903A9A9F10C00039343F0FE
:10C9F000BFFA53F00BFC56F8043C42460121009369
:10CA00002B464DF0DDFC0135032DD9D104F1700525
:10CA100004F5F274296821B9AB6813B1284641F0D6
:10CA2000B5FA7C35A542F5D105B0BDE8F08300BF6D
:10CA30003C2F110838B50546FFF7C6FC28B3134B49
:10CA40001B68DB6A93F89C30FBB9114C7DF0ACFCA1
:10CA50002368C01AB0F57A7F17D37DF0A5FC20605B
:10CA6000D5F80C4314F400640FD1E0B203F03CFCA1
:10CA7000024618B10B212846FFF79EFE95F8273095
:10CA8000052B02D00134032CEFD138BD088E0030C5
:10CA9000788E003038B504461546FFF753FEC0B215
:10CAA000022808D87C23294603FB0040BDE8384013
:10CAB000543043F09DBA38BD38B504461546FFF7EB
:10CAC00041FEC0B2022808D87C23294603FB00405F
:10CAD000BDE83840603043F08BBA38BD37B50D46FD
:10CAE00004468DED010AFFF72DFE022D07D8C0B2D6
:10CAF0007C2301A903FB00406C3043F021F903B013
:10CB000030BD000038B50546FFF71CFEC4B2022C4C
:10CB100013D8C4EB441440350021A40004F10800EC
:10CB2000284441F033FA04F1340104F1300029447F
:10CB30002844BDE8384043F01BBA38BD70B50546FF
:10CB40000E461446FFF7FEFDC3B2022B0DD87C2023
:10CB500000FB035394E80700483383E8070031469D
:10CB60002846BDE87040FFF7CDBF70BD37B504461D
:10CB70001546FFF7E7FDC0B2022809D87C230DF166
:10CB800007018DF8075003FB0040443043F05CF987
:10CB900003B030BD1FB590F93030044623B390F98F
:10CBA00025300BB36846FEF767FFFBF761F869466F
:10CBB000FAF790FDC0B1DDED037A01239FED0B0A7A
:10CBC000F8EEE70ADDED027A84F84133F8EEE77A11
:10CBD000C0EE800A87EE800A07F060FEDFED047A7F
:10CBE00020EE270A84ED0B0A04B010BD8096184B86
:10CBF00035FA8E3C38B505460C46FFF7E5FB40B1EB
:10CC00002C4494F9300220B195F92800033818BF5C
:10CC1000012038BD70B590F8264006465CB100256D
:10CC20002C46E9B23046FFF7E5FF08B10134E4B223
:10CC30000135032DF5D1204670BD000090ED0B0AA3
:10CC40007047000038B50C46D1ED066A114605461E
:10CC5000FFF778FDD4ED087AC3B27C2094ED076A23
:10CC6000B7EE007A00FB0353D3ED270AA6EEE67A6F
:10CC7000D3ED265A26EE600A93ED255A67EEA00AF8
:10CC8000A5EEA70AF0EE607AE5EE867AB1EE400AEC
:10CC900067EEE60AE5EE070AD9F0CAF940F6580051
:10CCA0009FED061ADFED060A18F0F0F8D5ED0B7AC5
:10CCB000BDE8384030EE270A18F0BCB8DB0F494019
:10CCC000DB0F49C02DE9F04190F8263004460D46AF
:10CCD0008B4202D20020BDE8F081FFF733FD04F162
:10CCE0004006C0B2C0EB401006EB800008301CF0DC
:10CCF0006DFCB0EEC00ADFED147AB4EEE70AF1EE97
:10CD000010FAE7D429462046FFF71CFDC5B27C2067
:10CD100000FB05477B6F002BDCD0032DDAD000FB36
:10CD20000560D7F87080303042F0F6F8D7E91C3251
:10CD3000934201D1984505D07C2000FB0544C4F8FE
:10CD40007080C7E70120C6E7000000342DE9F74FE7
:10CD500004460E46174600F5107A4FF0000B5AF8BD
:10CD6000049B5FFA8BF8B9F1000F26D041462046AC
:10CD7000FFF740FF08B341462046FFF7E3FC7C2362
:10CD8000C0B203FB004090F842505DB908F10103C6
:10CD90001B4A39463046DBB27CF010FD284603B012
:10CDA000BDE8F08F5AF8102C914506D0154A394647
:10CDB000304600257CF002FDF0E70BF1010BBBF1E2
:10CDC000030FCCD14FF000085FFA88F194F82630B9
:10CDD0008B420DD920460191FFF774FF054620B91B
:10CDE00001992046FFF706FF20B908F10108EBE79B
:10CDF0000125D3E7044A394630467CF0DFFCCDE715
:10CE0000642F1108792F11089E2F11082DE9F04188
:10CE100006464FF000082DED048B82B090F84613C3
:10CE2000FFF790FC06F14007C5B27C209FED2F8AEA
:10CE300000FB0575DFED2E8A9FED2E9A54355FFAC3
:10CE400088F496F82630A3424DD921463046FFF7A4
:10CE5000D1FE10B908F10108F1E721463046FFF78D
:10CE600071FCC4B27C2000FB0474D4ED157A5434F8
:10CE7000F0EEE77AF4EEC87AF1EE10FA0ED5D4EDC2
:10CE8000017AF0EEE77AF4EEC87AF1EE10FA05D501
:10CE9000002002B0BDEC048BBDE8F081294620469D
:10CEA0001CF0A4FBB4EEE80AF1EE10FAF0DC29461F
:10CEB00020461BF0F9FDB4EEC90AF1EE10FAE7DCEA
:10CEC000214628461BF03CFD68468DED000ACDED5D
:10CED000010A1BF0DDFDDFED087AB4EEE70AF1EEA2
:10CEE00010FAB7DDD4E70120D3E700BF000000341B
:10CEF000DB0FC93F920A863F00004843022910B564
:10CF0000044608D8FFF71EFC7C23C0B203FB004494
:10CF100094F8410010BD0020FCE7000013B590F824
:10CF2000461304460191FFF7E9FF30B1019920460D
:10CF300002B0BDE81040FFF75DBE02B010BD0000BA
:10CF4000F7B50446FFF740FA0546002873D094F879
:10CF500046132046FFF7D2FF94F84133064613B933
:10CF60002046FFF717FE00252046FFF763FD94F8E3
:10CF70002420EBB29A4207D90633013554F8230036
:10CF800003689B689847F2E77DF00EFA0027224677
:10CF900004F5BA7140F2F315D2F8A0307C32C31A0E
:10CFA000AB428CBF0023012302F83B3C914247EA8D
:10CFB0000307F1D194F92830032B07D194F84033BB
:10CFC000002B3BD0D4F83C03002849D167B1636BF8
:10CFD000013309D047F098FC616B47F0B3FA18B100
:10CFE00047F092FC46F0ACFA94F93032002B3AD17B
:10CFF00094F93132CBBB94F9323213B1022384F865
:10D00000463394F846132046FFF778FF86420546DC
:10D0100011D047F079FC4FF6FF7147F093FA50B109
:10D02000002D14BF00220422019247F06DFC019AEA
:10D03000032147F019FA284603B0F0BD012304206C
:10D0400084F84033FFF776F9054610B1214607F022
:10D050007FFA94F92830C4F83C53032BB2D0B5E7DB
:10D0600007F084FAB2E70023C9E70123C7E700000D
:10D0700070B504460E46FFF7A7F90546C8B131461C
:10D080002046FFF75FFBC0B2022812D87C239FED39
:10D090000A7A03FB0044D4ED1B7AF4EEC77AF1EE72
:10D0A00010FA06D4B7EE087AF4EEC77AF1EE10FA69
:10D0B00000DD0025284670BDABAA2A3F70B5D0F828
:10D0C0000C5304460E4615F400350DD190F8443348
:10D0D0005BB90A78072A07D8012303FA02F290F80D
:10D0E0004333134380F8433370BD94F82420EBB2EC
:10D0F0009A42F9D906333146013554F823000368C2
:10D10000DB689847F1E7000038B5054670242B59D5
:10D110001BB10021281940F039FF7C34B4F5F27FAF
:10D12000F5D138BD014B1868704700BF748E0030D0
:10D1300010B50446006810B103685B689847204644
:10D1400010BD000010B50446006810B103685B68AC
:10D150009847204610BD000010B50446006810B185
:10D1600003685B689847204610BD00006D4B2DE9B1
:10D17000F04F1E68044689B0002570684FF0010921
:10D18000DFF8ACA103689B689847804609FA05F36D
:10D1900013EA080F52D10135202DF7D17068002510
:10D1A0004FF00109DFF888A10368DB6898478046E3
:10D1B00009FA05F313EA080F7BD10135202DF7D1C9
:10D1C0000025594AB16805A8FFF7E2F8059B2A46F1
:10D1D000294607A80793CDE9055505F02FFB102137
:10D1E00002462046FFF7E8FA07A8FFF7B5FF06A8B2
:10D1F000FFF7B2FF05A8FFF79BFF94F82730052B38
:10D2000048D0B16805A8494AFFF7C2F8059B2A46ED
:10D21000294607A80793CDE9055505F00FFB102116
:10D2200002462046FFF7C8FA07A8FFF795FF06A8B1
:10D23000FFF792FF05A8FFF77BFF2BE05FFA85FB66
:10D240000E2220465946FFF797FA074628B30023D7
:10D25000CDE90433059A0023012107A807920A2289
:10D26000CDE9053303F026FF072102462046FFF7EC
:10D27000A3FA07A8FFF770FF06A8FFF76DFF05A840
:10D28000FFF760FF17B104A8FFF75CFF94F82730A1
:10D29000052B80D109B0BDE8F08F0423CDF800A0A4
:10D2A0005A46CDE901030E23716805A8FFF77AF805
:10D2B000D0E75FFA85FB0E2220465946FFF75CFA5D
:10D2C000074618B30023CDE90433059B00210A2249
:10D2D00007A80793CDE9051103F0ECFE07210246EC
:10D2E0002046FFF769FA07A8FFF736FF06A8FFF701
:10D2F00033FF05A8FFF726FF17B104A8FFF722FFA9
:10D3000094F82730052B7FF458AFC3E70423CDF8FA
:10D3100000A05A46CDE901030E23716805A8FFF766
:10D3200041F8D2E7088E0030B82F1108C12F11083C
:10D33000801A06002DE9F04FD0F80C538DB004464A
:10D340000F4615F4807B164698469DF858909DF838
:10D350005CA060D1FFF710FA054600283FD0CDE968
:10D3600006BB069B4FF0000B42463946204604930D
:10D37000CDE905BBFFF700FA064600283DD0CDE910
:10D380000ABB0A9A002308A904A808924A46CDE9D4
:10D390000933534600F0DEFF074608A8FFF7DCFE1E
:10D3A00009A8FFF7D9FE0AA8FFF7CCFE16B10BA813
:10D3B000FFF7C8FE04A8FFF7CFFE05A8FFF7CCFED5
:10D3C00006A8FFF7BFFE15B107A8FFF7BBFE3A4658
:10D3D000082120460DB0BDE8F04FFFF7EDB904235A
:10D3E0000E493A460968CDE901030D4B06A80093A2
:10D3F00033464968FEF7D6FFB3E7042307493A46A8
:10D400000968CDE90103064B0AA800934346496821
:10D41000FEF7C8FFB5E70DB0BDE8F08F088E00300D
:10D42000801A06002DE9F04F01249146D0F80C2314
:10D430008BB08C40984606460F4614409DF85030FD
:10D440009DF854A09DF858B035D11A464146059331
:10D45000FFF792F9059B054600B3CDE90844089A09
:10D460000023514606A806925A46CDE90733C8471D
:10D47000044606A8FFF770FE07A8FFF76DFE08A890
:10D48000FFF760FE15B109A8FFF75CFE224639469A
:10D4900030460BB0BDE8F04FFFF78EB904220749C4
:10D4A000CDE90102096808A8054A00924246496888
:10D4B000FEF778FFD3E70BB0BDE8F08F088E0030A1
:10D4C000801A0600B34B2DE9F04F1D68044689B061
:10D4D000002668684FF001084FF0080ADFF8BC9298
:10D4E00003689B689847074608FA06F33B4240F0FA
:10D4F0007A820136202EF7D1686800264FF00109A4
:10D500004FF006080368DFF894A2DB6898470746E7
:10D5100009FA06F33B4240F078820136202EF7D11B
:10D52000686800264FF001084FF0080A0368DFF82A
:10D5300070929B689847074608FA06F33B4240F012
:10D5400075820136202EF7D1686800264FF0010859
:10D550004FF0080A0368DFF84C929B68984707462B
:10D5600008FA06F33B4240F071820136202EF7D1D3
:10D570006868002601274FF01A0903689B689847DE
:10D58000804607FA06F313EA080F40F06F8201366F
:10D59000202EF6D1686800264FF0010A4FF01A09D4
:10D5A0000368B046DB68984707460AFA06F33B4231
:10D5B00040F077820136202EF7D1686800264FF0C0
:10D5C000010ADFF8E4910368B046DB689847074634
:10D5D0000AFA06F33B4240F07F820136202EF7D153
:10D5E000686800264FF0010ADFF8BC910368B04676
:10D5F000DB68984707460AFA06F33B4240F07C8214
:10D600000136202EF7D1686800264FF001084FF050
:10D61000020A0368DFF890919B689847074608FA6A
:10D6200006F33B4240F078820136202EF7D168683D
:10D6300000264FF001084FF0020A0368DFF86891F6
:10D640009B689847074608FA06F33B4240F0808201
:10D650000136202EF7D1686800264FF00108DFF868
:10D660004C910368B2469B689847074608FA06F350
:10D670003B4240F07D820136202EF7D168680026BB
:10D680004FF0010ADFF824910368B046DB68984741
:10D6900007460AFA06F33B4240F07A820136202E12
:10D6A000F7D1686800264FF001084FF0060A0368BA
:10D6B000DFF8FC909B689847074608FA06F33B4260
:10D6C00040F076820136202EF7D1686800264FF0B0
:10D6D000010ADFF8DC900368B046DB68984707462C
:10D6E0000AFA06F33B4240F073820136202EF7D14E
:10D6F000294B07AF0426DFF8BC904FF00C0A0793C4
:10D7000068684FF000084FF0010B03689B6898476A
:10D7100005900BFA08F3059A134240F0698208F16C
:10D720000108B8F1200FF4D168684FF000084FF0FD
:10D73000010B0368DB68984705900BFA08F3059A1C
:10D74000134240F0668208F10108B8F1200FF4D1CD
:10D75000013E013716F0FF06D2D168684FF001088C
:10D76000B146DFF854A003689B689847074608FA5B
:10D7700006F33B4240F060820136202EF7D1686804
:10D7800000264FF00109DFF830A00368B046DB68DF
